:100000005446495300010000A84C0200E70C1A10A6
:10001000101701041610261444315930101702002D
:100020001610261444313030101701121610261401
:100030004431594C030000000000000000000000A3
:1000400054464353002000000C240200000000002E
:100050000080011001210000252100004122000044
:10006000292100002B2100002D2100003D2100004E
:100070003D2100003D2100003D2100002F21000016
:10008000312100003D21000033210000A55A00006D
:100090008B5B0000372100003D210000094B001060
:1000A000372100009F3E0000A53E00003D210000DA
:1000B0003D210000CF5600002D4E0000AB3E000059
:1000C00055540000372100003D2100003D21000073
:1000D0000000000000000000000000000000000020
:1000E0000000000000000000000000000000000010
:1000F0000000000000000000000000000000000000
:1001000000000000000000000000000000000000EF
:1001100000000000000000000000000000000000DF
:1001200000000000000000000000000000000000CF
:1001300000000000000000000000000000000000BF
:1001400000000000000000000000000000000000AF
:1001500000F003F800F020F8FEE70D480168890878
:100160008900002001C101C101C101C17047000027
:1001700088590010FEE7FEE7FEE7FEE7FEE7FEE730
:10018000FEE7FEE7FEE703480047FEE7FEE7000064
:10019000202100003D21000000F002F800F068F886
:1001A0000AA090E8000C82448344AAF10107DA45D2
:1001B00001D100F05DF8AFF2090EBAE80F0013F0BC
:1001C000010F18BFFB1A43F001031847F8CD0100D7
:1001D00048CE01000A444FF0000C10F8013B13F028
:1001E000070408BF10F8014B1D1108BF10F8015B90
:1001F000641E05D010F8016B641E01F8016BF9D183
:1002000013F0080F1EBF10F8014BAD1C0C1B09D1D9
:100210006D1E58BF01F801CBFAD505E014F8016B4B
:1002200001F8016B6D1EF9D59142D6D370470000DD
:10023000103A24BF78C878C1FAD8520724BF30C812
:1002400030C144BF04680C607047000000230024E4
:1002500000250026103A28BF78C1FBD8520728BFD6
:1002600030C148BF0B6070471FB51FBD10B510BD32
:10027000DFF80CD0FFF7F8FF04F0B8FF1CF00AF825
:100280000080011003B4FFF7F1FF03BC1CF00AF873
:100290001EF0040F0CBFEFF30880EFF3098009F0A4
:1002A00005BF000008B5002103200B460A46009157
:1002B0001AF0CAFD08BD38B5FC4D0024AC80EC80B6
:1002C0002C811AF09EFD2861FF20A870F848234673
:1002D00022460460446004720120E8700320214635
:1002E00000941AF0B1FD012038BD38B5EF4D022859
:1002F000AC7822460DD0052810D0A24208BF38BDE8
:10030000002003460246214600901AF09DFDAC7085
:1003100038BD022914BF01240224EEE7022914BFCC
:1003200064246524E9E738B513460A464FF0010C0A
:1003300000240146604600941AF086FD38BDDB4873
:1003400000697047D949012008707047D748007884
:100350007047D6490020087070472DE9F0410446E7
:100360000127002503F00700D04E8846012804BF6E
:100370000020308146D0022844D1308904280BD295
:10038000002818BFF06802D11AF07FFDF06010F865
:10039000011B2170F0602EE0062808D21AF077FDCC
:1003A0003189C1F10501C900C840207023E0082847
:1003B00008D21AF070FD3189C1F10701C900C840A7
:1003C000207018E00C2808D21AF01BFD3189C1F109
:1003D0000B01C900C84020700DE00E2808D21AF0A9
:1003E00012FD3189C1F10D01C900C840207002E041
:1003F000FF20207000273089401C80B230810E28F9
:1004000028BF012588F800503846BDE8F08130B497
:1004100003F007000024DFF894C201280BD06046E7
:10042000BCF808308088022B0CD2120242EA10205D
:10043000ACF8040010E0ACF80440ACF80640ACF8AE
:1004400008400CE01844851EB5F5806F04DADCF82E
:100450001050284400F8022C581CACF808000C700E
:1004600030BC00207047F0B40746002003F00704BA
:100470008E4D0646012C08BF2E811AD0DFF82CC203
:10048000022CBCF806C003D013F0070F0DD010E00B
:100490002A890CEB0203B3F5806F0AD22869C05C8D
:1004A0003870501C2881012003E0120242EA1C220D
:1004B000EA800E70F0BC704738B503F007000024E6
:1004C0000D4601280AD1794821460B4604818480D3
:1004D000C48002200A4600941AF0B6FC2C7000205A
:1004E00038BD2DE9F04182B00446DDE908061F461B
:1004F0000D464FF0010804EB061C002818BF022827
:1005000018D0002101287CD003281CBF02B0BDE810
:10051000F0810F202070032060706180A180E18055
:1005200021816181A181A07B20F00100A07302B034
:10053000BDE8F0810CF8106C0CF80F0CB5F8B400A5
:100540002CF80E0CB5F8B6002CF80C0C95F89000B1
:100550002CF80A0C95F891002CF8080C95F89200EC
:100560002CF8060CA88A2CF8040C92F848101CF8F9
:10057000020C61F300000CF8020C95F8EE00012863
:100580001CBF02B0BDE8F08104F038FE05281CBF96
:1005900002B0BDE8F08109F020FE042804BF02B0DB
:1005A000BDE8F081C0208DF8000095F899008DF825
:1005B000010095F8990004EB001030F80E0C000AC9
:1005C0008DF8020095F8990004EB001010F80E0C5D
:1005D0008DF8030095F8990004EB001030F80C0C2E
:1005E000000A8DF8040095F8990004EB001010F84B
:1005F0000C0C8DF805000CF0BBFE9DF800100909ED
:1006000000E00FE008FA01F1084204BF02B0BDE8C3
:10061000F08101230622694607200CF0DFFE02B0BC
:10062000BDE8F0810CF8106C0CF80F8C2CF80E1C47
:100630002CF80C1C2CF80A1C2CF8081C2CF8061C96
:100640002CF8041C1CF8020C20F001000CF8020C21
:1006500004F0D4FD05281CBF02B0BDE8F08109F00C
:10066000BCFD042804BF02B0BDE8F081C1208DF8B4
:1006700000008DF801607888000A8DF80200B878D3
:100680008DF80300B888000A8DF8040038798DF8D9
:1006900005000CF06DFE9DF80010090908FA01F143
:1006A0000842B6D102B0BDE8F0810000008400101D
:1006B000388700102B49002048707047294840783F
:1006C00070472849012048707047274A11547047E5
:1006D000244800B5006983B04FF00001407810F065
:1006E000020F0AD000918DF80410012305226946FB
:1006F00000200CF09AFE03B000BD10F0040F12D0E1
:1007000001208DF800008DF801108DF802108DF891
:1007100003108DF8041003460522694600200CF0F2
:1007200084FE03B000BD10F0C00F4FF001034FF086
:10073000000206D003B0012103205DF804EB0CF0A9
:100740001DBE03B0632107205DF804EB0CF016BE5C
:1007500070470449002818BF0120C870704701483D
:10076000C078704700840010388700107047FE483A
:10077000D0F8500300F00100704770B5FA4D040046
:100780000AD001F020FB38B9D5F8500310F0010F62
:100790001CBF0020A86005D10120A860002C08BF64
:1007A000002000D00120286270BDEF48006A0028B8
:1007B00018BF01207047C00000F1804000F5A04044
:1007C00041637047C00000F1804000F5A040006B1D
:1007D00000F4807070471021C00000F1804000F5E7
:1007E000A04041637047E049D1F8402160F30D22F9
:1007F000C1F840217047DC48D0F84001C0F3052023
:10080000704700F00F0202EB42029201C0F30310A6
:1008100002EB801000F1804000F5A0400029D0F8E4
:10082000401114BF41F0010121F00101C0F8401155
:10083000704700F00F0101EB41018901C0F3031083
:1008400001EB801000F1804000F5A040D0F840019D
:1008500000F001007047C44900230B6202680A607F
:1008600042684A6082688A60C268CA60426A0A64F2
:10087000826A4A6402698A614269CA61826B0A6655
:10088000826C0A67C26C4A67026D8A67426DCA67EA
:10089000826DC1F88020C26DC1F88420026EC1F85B
:1008A0008820426EC1F88C20426FC1F8B020C26F20
:1008B000C1F8B820C26EC1F8A820D0F89422C1F8BF
:1008C0005023D0F89822C1F85423D0F89C22C1F8C4
:1008D0005823D0F8A022C1F85C23D0F88420C1F8B6
:1008E000F020D0F88820C1F8F420D0F88C20C1F88E
:1008F000F820D0F89020C1F8FC2021224A63CA6376
:10090000C2694A62C26A8A64026BCA64026FC1F831
:10091000AC20026ACA62426B0A65C26B4A66026C0C
:100920008A66426CCA66826FC1F8B420D0F8802013
:10093000C1F8BC20D0F8A422C1F86023D0F8A822C6
:10094000C1F86423D0F8AC22C1F86823D0F8B022F3
:10095000C1F86C23D0F8B422C1F87023D0F8B822C3
:10096000C1F87423D0F8BC22C1F87823D0F8C02293
:10097000C1F87C23D0F88C2222F48032C1F84023C5
:10098000D0F89022C1F84C23D0F89420C1F800216F
:10099000D0F89820C1F80421D0F89C20C1F8082193
:1009A000D0F8A020C1F80C21D0F8A420C1F8102163
:1009B000D0F8A820C1F81421D0F8C820C1F83421FB
:1009C000D0F8AC20C1F81821D0F8B020C1F81C2113
:1009D000D0F8B420C1F82021D0F8B820C1F82421E3
:1009E000D0F8BC20C1F82821D0F8C020C1F82C21B3
:1009F000D0F8C420C1F83021D0F8CC20C1F8402173
:100A0000D0F8D020C1F84421D0F8D820C1F84C212A
:100A1000D0F8E420C1F86021D0F8E820C1F86421C2
:100A2000D0F8EC20C1F86821D0F8F020C1F86C2192
:100A3000D0F8D420C1F84821D0F8DC20C1F85021EA
:100A4000D0F8E020C1F85421D0F8F420C1F870218A
:100A5000D0F8F820C1F87421D0F8FC20C1F8782132
:100A6000D0F80021C1F87C21D0F83C21C1F8C02188
:100A7000D0F84021C1F8C421D0F84421C1F8C821E0
:100A8000D0F84821C1F8CC21D0F84C21C1F8D021B0
:100A9000D0F85021C1F8D421D0F87021C1F8F42148
:100AA000D0F85421C1F8D821D0F85821C1F8DC2160
:100AB000D0F85C21C1F8E021D0F86021C1F8E42130
:100AC000D0F86421C1F8E821D0F86821C1F8EC2100
:100AD000D0F86C21C1F8F021D0F87421C1F80022BF
:100AE000D0F87821C1F80422D0F88021C1F80C2276
:100AF000D0F88C21C1F82022D0F89021C1F824220E
:100B0000D0F89421C1F82822D0F89821C1F82C22DD
:100B1000D0F8AC21C1F84022D0F8B021C1F844226D
:100B2000D0F8B821C1F84C22D0F8C421C1F8602215
:100B3000D0F8C821C1F86422D0F8CC21C1F86822CD
:100B4000D0F8D021C1F86C22D0F87C21C1F808225D
:100B5000D0F88421C1F81022D0F88821C1F81422DD
:100B6000D0F89C2102E0000000500040C1F8302283
:100B7000D0F8A021C1F83422D0F8A421C1F838223D
:100B8000D0F8A821C1F83C22D0F8B421C1F84822FD
:100B9000D0F8BC21C1F85022D0F8C021C1F85422AD
:100BA000D0F8D421C1F87022D0F8D821C1F874222D
:100BB000D0F8DC21C1F87822D0F8E021C1F87C22FD
:100BC000D0F8E421C1F88022D0F8E821C1F88422CD
:100BD000D0F8EC21C1F88822D0F8F021C1F88C229D
:100BE000D0F8F421C1F89022D0F8F821C1F894226D
:100BF000D0F81822C1F8B422D0F8FC21C1F898220C
:100C0000D0F80022C1F89C22D0F80422C1F8A0221A
:100C1000D0F80822C1F8A422D0F80C22C1F8A822EA
:100C2000D0F81022C1F8AC22D0F81422C1F8B022BA
:100C3000D0F81C22C1F8C022D0F82022C1F8C4226A
:100C4000D0F82822C1F8CC22D0F83422C1F8E02212
:100C5000D0F83822C1F8E422D0F83C22C1F8E822CA
:100C6000D0F84022C1F8EC22D0F85422C1F8002379
:100C7000D0F85822C1F80423D0F86022C1F80C2320
:100C8000D0F86C22C1F82023D0F87022C1F82423B8
:100C9000D0F87422C1F82823D0F87822C1F82C2388
:100CA000D0F82422C1F8C822D0F82C22C1F8D022D2
:100CB000D0F83022C1F8D422D0F84422C1F8F02272
:100CC000D0F84822C1F8F422D0F84C22C1F8F8221A
:100CD000D0F85022C1F8FC22D0F85C22C1F80823D9
:100CE000D0F86422C1F81023D0F86822C1F8142388
:100CF000D0F87C22C1F83023D0F88022C1F8342308
:100D0000D0F88422C1F83823D0F88822C1F83C23D7
:100D1000FE4A126832F0FF0C05D1D1F890C062F3A0
:100D2000030CC1F890C0FA4A5370D0F8943213F013
:100D3000010F1CBF01235370D1F8503323F001037E
:100D4000C1F85033D0F8A43213F0010F03D0537818
:100D500043F002035370D1F8603323F00103C1F86C
:100D60006033D0F8B43213F0010F03D0537843F05E
:100D700004035370D1F8703323F00103C1F87033CA
:100D8000D0F8AC0210F0010F03D0507840F008000A
:100D90005070D1F8680320F00100C1F86803704773
:100DA000DB4800787047DA4880787047D849C870C7
:100DB0007047D748C0787047D649D1F8542360F3BC
:100DC0000902C1F854237047D248D0F85403C0F345
:100DD00009007047CE4948607047CE48C0687047E8
:100DE0002DE9F047DFF82893054615F4003F99F800
:100DF000010099F8031000EA010418BF24F001046F
:100E000015F4802F18BF24F0020415F4002F18BF2A
:100E100024F00404DFF8FC82D8F8400320F480308A
:100E2000C8F8400314F0070F59D0D9F80460D8F877
:100E30004803002740F00100C8F84803D8F84803E9
:100E400020F00100C8F84803D8F8400340F480308F
:100E5000C8F840034FF0630A0DE002F0B4FE5046BC
:100E6000D8F8481311F0010F01D0012703E0011E4B
:100E7000A0F10100F4DC301EA6F1010601DD002F17
:100E8000EBD067B3D8F8500314F0010F0CBF20F07B
:100E9000010040F00100C8F85003D8F8600314F0D6
:100EA000020F14BF40F0010020F00100C8F86003F9
:100EB000D8F8700314F0040F14BF40F0010020F0C4
:100EC0000100C8F8700389F80240012089F8000089
:100ED000D8F8400340F48030C8F8400333E0D8F835
:100EE000500320F00100C8F85003D8F8600320F048
:100EF0000100C8F86003D8F8700320F00100C8F8BA
:100F00007003002089F80200ACB1022089F80000CB
:100F1000D8F8400340F48030C8F84003D8F84803BC
:100F200040F00100C8F84803D8F8480320F0010059
:100F3000C8F8480307E0D8F8401321F48031C8F816
:100F4000401389F80000D8F8400115F0020F20F096
:100F50000D0018BF40F0010015F0080F18BF40F059
:100F6000040015F0040F18BF40F00800C8F8400155
:100F700015F0010F21D001F05AF9044601F05AF999
:100F80000146D8F80C0000280EBF2046084621462E
:100F90000028D8F8000214BF40F0010020F0010042
:100FA000C8F80002D8F84002002914BF40F0010040
:100FB00020F00100C8F840020BE0D8F8000220F051
:100FC0000100C8F80002D8F8400220F00100C8F87B
:100FD000400215F0200F18BF002417D0204601F062
:100FE00030F900284FEA841000F1804000F5A0405D
:100FF000D0F8C01214BF41F0010121F00101C0F886
:10100000C012641C022CE9D3BDE8F087D8F8C002F6
:1010100020F00100C8F8C002D8F8000320F0010059
:10102000C8F80003BDE8F0872DE9F003024602F09E
:101030000F01002001EB41018C01C2F3031104EB0D
:10104000811101F1804101F5A041D1F8401111F069
:10105000010F11D142F01001C1F3031104EB811112
:1010600001F1804101F5A041D1F8401111F0010FCB
:1010700004BFBDE8F003704702EB42018E0106F1A8
:10108000804101F5A041D1F82431C3F30809214B77
:10109000DB69D1F8001103F008071FFA81F800217D
:1010A00042EA0113C3F3031304EB831303F18043F8
:1010B00003F5A043D3F8403113F0010F18D006EB2D
:1010C000811303F1804303F5A043D3F844C1CCF36B
:1010D000080517F1000C1CBFD3F844C1CCF3023C47
:1010E000D3F8403105FA0CFCC3F3054360441844BF
:1010F000491C0229D4D309EBC90100FB08F001EB1C
:101100000911BDE8F00300EB41007047E0FE030069
:10111000148400100050004010B50120FFF784FF38
:1011200004460220FFF780FF044400F03CFC20440A
:101130004FF47A7148434CF25031B0FBF1F010BDDE
:101140002DE9F041FA4E0546306810F01F0408BF43
:1011500001240120FFF768FF07460220FFF764FF24
:10116000074400F020FC3918F24F002D18BF002969
:101170004ED0D6F85003002210F0010F36D0782060
:10118000B0EB151F08D9D6F85C0320F00F0040F033
:101190000100C6F85C032EE0D6F85403E64BC0F31A
:1011A000090060436FF0180C00FB0CF003EB4003E8
:1011B000E248A0FB05C04FEA502CB3FBF1F0102829
:1011C00028BF0F20844598BF6046002808BF012033
:1011D00005D0012884BF00FB1132B2FBF0F2D6F833
:1011E0005C3360F30303C6F85C3304E0B7FBF5F04F
:1011F000884288BF421A32206043B2FBF0F0B0F55B
:10120000005F28BF41F6FF70726860F30C027260E5
:101210007068C0F30C00604300EBC00202EB0010EA
:1012200001EB4000B7FBF0F0BDE8F081C048D0F81A
:10123000501311F0010F07D0D0F85C0300F00F003D
:10124000C0EB00108001704770B50168406801F084
:101250001F05C0F30C060120FFF7E6FE044602203E
:10126000FFF7E2FE044400F09EFB06FB05F132228C
:1012700001FB02410844AF49B1FBF0F070BDAC483E
:10128000D0F85C0300F00F007047A9494A684B682A
:10129000C2F30C0260F30C034B6010467047A44885
:1012A0004068C0F30C00704700EB4000800100F183
:1012B000804000F5A040D0F80001A14980B2B1FB08
:1012C000F0F0401C4008704730B49D4B31B1B3FB87
:1012D000F1F1491C4A08B2F5804F01D343F6FF7281
:1012E000B3FBF2F1491C4D0800EB400189015308A2
:1012F00001F1804101F5A041002807BF981FA3F12B
:101300000C0CD1F8040180B218BFA2F1060C2CF02D
:10131000010CD1F8004162F30F04C1F80041D1F88B
:10132000002163F31F42C1F80021D1F8042160F3CA
:101330000F02C1F80421D1F818016CF30F00C1F8B5
:101340001801284630BC704700EB4000800100F1D6
:10135000804000F5A040D0F80001000C704700EB81
:101360004002920102F1804202F5A042D2F800311F
:1013700061F31F43C2F80031002818BF70478A1F6D
:10138000901F20F001016A48D0F8043162F30F0386
:10139000C0F80431D0F8182161F30F02C0F8182109
:1013A000704700F00F0101EB41018901C0F3031008
:1013B00001EB801000F1804000F5A040D0F844011E
:1013C000C0F30800704700F00F0202EB42029201E6
:1013D000C0F303105B4B02EB801000F1804000F57E
:1013E000A0409B58D0F84421CB1A61F30802C0F802
:1013F0004421D0F844119B1E63F31841C0F84411F6
:1014000070474B49C969504A11F0100F00F00F01A5
:1014100001EB41014FEA8111C0F3031001EB801091
:1014200000F1804000F5A0405258D0F84401D2B2FB
:10143000C0F3080008BF0022801A0004000C08BF97
:101440000120704703091B0203EB810101F14051A8
:1014500001F540410007C00E0B6802FA00F0184386
:10146000086070470209120202EB810101F140514C
:1014700001F5404100070968C00E21FA00F000F0B4
:101480000300704700F00F0303EB43039B01C0F31D
:10149000031003EB801000EB810000F1804000F5A9
:1014A000A040C0F85021704700F00F0202EB42024A
:1014B0009201C0F3031002EB801000EB810000F1F9
:1014C000804000F5A040D0F850017047184A002134
:1014D000D26912F0080F10D000F00F0101EB4101AA
:1014E0008901C0F3031001EB801000F1804000F58A
:1014F000A040D0F84401C0F30231084670470C4ABE
:10150000D36943F00803D36100F00F0202EB4202FB
:101510009201C0F3031002EB801000F1804000F54F
:10152000A040D0F8442161F30E32C0F84421704746
:10153000005000400008AF2FD8810C0089888888AF
:10154000A08601001C51004028510040F84A0021AB
:10155000D26912F0080F10D000F00F0101EB410129
:101560008901C0F3031001EB801000F1804000F509
:10157000A040D0F84801C0F302410846704700F08F
:101580000F0202EB42029201C0F3031002EB801043
:1015900000F1804000F5A040D0F8482161F31242EC
:1015A000C0F848217047042988BF704710B4002351
:1015B000DF4CE26912F0080F00F00F0202EB42026A
:1015C0004FEA8212C0F3031002EB801000EB04021A
:1015D0001CBFD2F84401C0F302330020D4F81CC071
:1015E0001CF0080F1CBFD2F84801C0F30240C91A12
:1015F0000844042803DD081A011D042003E0002824
:10160000BCBF014400201944E36943F00803E361CF
:10161000D2F8443161F30E33C2F84431D2F84811A4
:1016200060F31241C2F8481110BC7047C04900284D
:10163000886914BF40F0080020F0080088617047F6
:10164000BB488069C0F3C000704700F00F0202EB96
:1016500042029201C0F3031002EB801000F18040BF
:1016600000F5A040C0F84C11704700F00F0101EBED
:1016700041018901C0F3031001EB801000F18040AB
:1016800000F5A040D0F84C017047A94AD2F85C138D
:10169000022903D110F0010F18BF7047D2F84001A2
:1016A00010F0010F0BD0D2F84C01D2F844110028F1
:1016B000C1F302311EBF0029C043C2F84C01012111
:1016C00001EB410100204FEA811C0CEB801101F17C
:1016D000804101F5A041D1F8402112F0010F0BD05B
:1016E000D1F84C21D1F84431002AC3F302331EBF94
:1016F000002BD243C1F84C21401C0228E5D370478F
:101700008B4A0021D26912F0080F10D000F00F01AF
:1017100001EB41018901C0F3031001EB801000F1DE
:10172000804000F5A040D0F84801C0F300510846C1
:1017300070470120704710B4022ADDF804C026BFAC
:10174000921E52080022022B26BF9B1E5B0800231C
:10175000784CA4FB0C4C4FEA1C1400F00F0C0CEB63
:101760004C0C4FEA8C1CC0F303100CEB801000F102
:10177000804000F5A040D0F864C161F31B6C62F3B7
:10178000144C63F30C2C64F3070CC0F864C110BC58
:10179000704770B400F00F0404EB4404A401C0F3DC
:1017A000031004EB801000F1804000F5A040DDF84C
:1017B0000CC0D0F864010029C0F30366C0F30444F0
:1017C000C0F30425C0B218BF0E6012B16100891CBD
:1017D000116013B16900891C1960BCF1000F04BFCE
:1017E00070BC704700EB80008000CCF8000070BC3B
:1017F000704770B491B000224FF480456C10EC46F5
:1018000001E0082A05D2531C03EB8303B5FBF3F375
:1018100004E0D31F03EB8303B4FBF3F35B1A48BF6D
:101820005B424CF82230521C102AEAD30026009B5F
:1018300001215CF821209A42BCBF13460E46491C88
:101840001029F6D300F00F0101EB41018901C0F32B
:10185000031001EB801000F1804101F5A041D1F8A7
:101860006801D1F8682100F00F0066F30302C1F8A7
:101870006821082807D2401C00EB8000B5FBF0F07F
:1018800011B070BC7047C01F00EB8000B4FBF0F0DB
:1018900011B070BC704700F00F0101EB41018901EC
:1018A000C0F3031001EB801000F1804000F5A04070
:1018B000D0F8680100F00F00082834BF401CC01F9A
:1018C00000EB800034BF4FF480414FF40051B1FB76
:1018D000F0F0704710F00F0F08BF704700F00F00D6
:1018E00000EB4000800100F1804000F5A04000299D
:1018F000D0F82C110CBF21F4803141F48031C0F8B4
:101900002C117047002110F00F0F0ED000F00F00C7
:1019100000EB4000800100F1804000F5A040D0F8CD
:101920002C0110F4803F18BF0121084670470000C9
:1019300000500040CDCCCCCC00F00F0000EB4000BC
:10194000800100F1804202F5A042D2F83401C2F8D1
:10195000341170472F4B58679967DA6770472D49E4
:101960000028D1F8AC0014BF40F0020020F00200C3
:10197000C1F8AC00704727490028D1F8AC0014BF6B
:1019800040F0010020F00100C1F8AC007047214890
:10199000D0F8E00070471F49C1F8E40070471D48C7
:1019A000D0F89800704770B41A4E0020D6F8401155
:1019B00011F0010F04BF70BC704711F0040FD6F88E
:1019C000242101F00805D6F800C1C2F308021FFA6D
:1019D0008CF4D6F844C1CCF3080C18BFC1F307400F
:1019E000F369C1F3052113F008031CBFD6F8443195
:1019F000C3F30233002D18BF491C0CFA03F301FB9B
:101A00000300604302EBC20170BC01EB021100EB6A
:101A10004100704700500040FEF7C7BE10B5FEF70A
:101A2000C4FE012818BF10BD0020FEF7A6FE21212C
:101A30000020FEF7C0FE2121BDE810400120FEF786
:101A4000BABE10B5FEF792FEFEF7AFFE01280AD12E
:101A50000020FEF792FE21210020FEF7ACFE21219E
:101A60000120FEF7A8FE0121052001F0EEFB012177
:101A7000052001F0EAFBFF490020087110BD10B5F8
:101A80004FF4066001F037FCBDE810404FF40660EB
:101A900001F022BCF74A0146107B002818BF012044
:101AA000002918BF012111737047F24A516A506230
:101AB00008467047EF490020C87288704870704728
:101AC000EC490020C87288704870704770B50007F4
:101AD000C00E0D46801E00EB400101EB0014E648ED
:101AE0004FF4987200EBC40029461AF0E1FBE3487A
:101AF00005F5987100EBC400BDE870404FF4987292
:101B00001AF0D6BB2DE9F0410546FEF774FEDC4F16
:101B1000DFF870830446EDB14C2004FB00F216465A
:101B2000294638461AF0C4FB324605F500614046A6
:101B30001AF0BEFB04EB440000EB041407EB840036
:101B40004C211AF0BAFB08EB8400BDE8F0414C21AF
:101B50001AF0B3BB4C21401C41430C4638461AF0E6
:101B6000ACFB21464046BDE8F0411AF0A6BB10B5DB
:101B7000C04CE061FFF734F9FFF712F9A1696FF388
:101B80000F01A161A269C1B242EA0121A16102284B
:101B900018BF10BDA06940F00100A06110BDBA4897
:101BA0008168BA4A114381600168521C1143016087
:101BB00000F061BE2DE9F041B34A0C46054693683A
:101BC000B248184390601068B1490843106000F0B3
:101BD00052FE0026002C76D00020FEF7CEFD2068B5
:101BE00020B1FEF738FE0020FEF7C7FD2846FFF7BC
:101BF000BEFF0020FEF71DFE70B36068FFF782FF96
:101C0000A448E16819B102151AF052FB1DE0A24D7B
:101C10004FF440711AF051FB00200123295600298E
:101C200010DB0A09120202EB800202F1405202F5B7
:101C300040420907C90ED2F800C003FA01F14CEA8C
:101C400001011160401C2628E8D39448616959B10C
:101C50004FF400721AF02CFB0120FEF7EAFDDFF8CA
:101C60001882864F48B904E04FF400711AF025FB42
:101C7000F2E71120FEF7DDFD70B1A56865B14046C1
:101C80004FF4987229461AF013FB38464FF49872B5
:101C900005F598711AF00CFB0220FEF7CAFD18B981
:101CA0001220FEF7C6FD70B1246964B17C484FF480
:101CB000987221461AF0FCFA7A484FF4987204F5AB
:101CC00098711AF0F5FA6B48C672867046704662D3
:101CD000017B002101734FF4066001F00CFBBDE8AD
:101CE000F0414FF4066001F0F7BA10B50020FEF79E
:101CF00044FD00F0ADFD5F48C078002808BF10BD6E
:101D00006148016821F0030141F00D7141F08051FB
:101D10000160816821F0020141F00D7141F08051B4
:101D2000816010BD4FF4066001F0DBBA10B54FF4CE
:101D3000066001F0D6FAFEF738FD01280AD100202E
:101D4000FEF71BFD21210020FEF735FD212101209A
:101D5000FEF731FD5448D0F8401321F48031C0F82B
:101D600040130020FEF709FD00F072FD4148C078E5
:101D7000002808BF10BD4448016821F0030141F06C
:101D80000D7141F080510160816821F0020141F044
:101D90000D7141F08051816010BD10B501F0A6FABF
:101DA00010F0600018BF012010BD3248C0697047B4
:101DB00030488069704772B62E498A6922EA00006D
:101DC000886162B670472B480078002818BF012050
:101DD000704770B5FEF7E9FC002818BF70BD0024FD
:101DE000244DEC72AC706C7021212046FEF7E3FCB0
:101DF00021210120FEF7DFFC2C70BDE8704001209E
:101E0000FEF7BBBC70B50446FEF7CFFC002818BF38
:101E100070BD0021174DE972A97069702121002061
:101E2000FEF7C9FC21210120FEF7C5FC022C3CBFB6
:101E30000120FEF7D0FC012028702C62BDE8704024
:101E4000FEF79BBC10B5FEF7B0FC002818BF10BD14
:101E50000020084CE072A07060702121FEF7ABFCFE
:101E600021210120FEF7A7FC0120FEF7B4FC012090
:101E700020701BE01C840010189D003018BD00303D
:101E80000080003000A000300080004002003412CA
:101E90000300341200C000304487001000D000302E
:101EA000489E003048BE0030005000402062BDE82F
:101EB0001040FEF762BC0020FEF75FBCFE49002028
:101EC000887048700120FEF758BCFB498862704753
:101ED000F948806A7047002818BF0120F649C86297
:101EE0007047F548C06A002818BF012070470020DD
:101EF00000F0CEBB012000F0CBBB10B5FFF747FDD3
:101F00000446FFF748FDED48044208BF10BDEA480B
:101F1000816941F0040181610E2101EAD43104F0AC
:101F200001020A43816962F31F418161E44801684B
:101F300041F02001016010BD002818BF0120DE49DA
:101F4000C8707047DF487047DF487047DA48006B59
:101F50007047D948406B7047D748806B70472DE970
:101F6000F04FD84F4FF0000C8DB007F14C04E6460F
:101F70004FF0FF3807F80C8004F80CE00CF1010C6E
:101F8000BCF1260FF6DB4FF0000C002807DD12F83D
:101F90000C5007F80C500CF1010C6045F7DC0022E6
:101FA0000126CDF804E06D46CDF800E0002816DDEE
:101FB00017F902C0BCF1000F0EDBBCF1260F0BD2EB
:101FC0004FEA5C190CF01F0C55F829A006FA0CFC1E
:101FD0004AEA0C0C45F829C0521C8242E8DB002278
:101FE00094460DF108094FEA521A02F01F0B55F8FA
:101FF0002AA006FA0BFB1AEA0B0F1ABF09F802C057
:102000000CF1010C09F80280521C262AEBDB00229D
:10201000002810DD17F902C0BCF1000F08DBBCF18D
:10202000260F3ABF19F80CC004F802C004F8028069
:10203000521C8242EEDBDFF880A200220028CAF8A0
:1020400030E009DD14F902C0944502D0CAF83040EE
:1020500002E0521C8242F5DBDFF870B20020ABF1E7
:10206000720404F14C0704F8008007F800E00BF854
:1020700000E0401C2628F6DB0020002904DD1A5C65
:102080002254401C8142FADC0020CDF804E0CDF857
:1020900000E0002912DD2256002A0CDB262A0AD293
:1020A000530902F01F0255F823C006FA02F24CEA67
:1020B000020245F82320401C8842ECDB0020024647
:1020C000430900F01F0C55F8233006FA0CFC13EA04
:1020D0000C0F1ABF09F80020521C09F80080401CA0
:1020E0002628EDDB002000290BDD2256002A05DB27
:1020F000262A3CBF19F802200BF80020401C884219
:10210000F3DB0020CAF838E0002909DD1BF90020C4
:10211000824202D0CAF838B002E0401C8842F5DBA7
:1021200011F0010F18BF252015D0420900F01F0340
:1021300055F8222006FA03F31A420AD1420900F0A8
:102140001F0055F8223006FA00F0184345F8220027
:1021500001E0401EE9D500200246430900F01F0CB3
:1021600055F8233006FA0CFC13EA0C0F1ABF09F8D5
:102170000020521C09F80080401C2628EDDB0020BE
:1021800000290ADD2256002A04DB262A3CBF19F862
:1021900002203A54401C8842F4DB0020CAF834E0A4
:1021A0000029DCBF0DB0BDE8F08F3A56824204D062
:1021B000CAF834700DB0BDE8F08F401C8842F4DBE3
:1021C0000DB0BDE8F08F40F2DB114843404901EB10
:1021D000800070473F49C0EB001001EBC000704722
:1021E000DFF8D4C0012B8CF805008CF8061003D959
:1021F000401C20F0010011468CF807008CF80810F4
:1022000000FB01F24FF6FF7101EA4202ACF8122026
:1022100001EA4000ACF8140070472748007A704784
:102220002548C0797047244A5072917270472248FD
:10223000807A70472048407A7047274A1070517062
:1022400070472549085C70472DE9F047DFF8689032
:10225000044699F80C00002804BF99F801001AF010
:1022600031F899F80B00002808BFBDE8F0874FF05F
:102270000008D9F81C0047464646454610F0020FB4
:102280001CBFDFF84C8010F0040F05D0B9F8121015
:102290000F4A21F001018F1810F0010F18BF0D4EE9
:1022A00010F0200F18BF0D4DD9F828002060FEF760
:1022B0007AFD10F0010F13E01C84001001000700EC
:1022C0005C840010448700106A870010DC870010CF
:1022D00004880010708F0010298400106090001096
:1022E00006D0FEF7CCFF022828BF99F8020000D2E2
:1022F0000020E760C4E90108C4E904650120BDE8E5
:10230000F087FF490020C872704770B50546FEF798
:1023100072FA4C2100FB01F21446FA49284619F0E2
:10232000C7FF224605F50060BDE87040F64919F088
:10233000BFBFF0B583B0FEF75EFA04460021084641
:10234000FFF7B2F8009001210020FFF7ADF800225E
:102350000190002C2AD96E464FF0010C4FF6F07513
:1023600002EB4200002100EB02104B0901F01F07B5
:1023700056F823300CFA07F73B4211D0CB079B0CE1
:1023800003EB80034F0803EB870303F1405303F58E
:1023900000431B889BB2AB4202D903B00020F0BDC2
:1023A000491C2629E1D3521CA242D9D303B00120F3
:1023B000F0BD70B50D460107C80E811E01EB41004E
:1023C00000EB0114D1484FF4987200EBC401284689
:1023D00019F06EFFCE484FF4987200EBC40105F57A
:1023E0009870BDE8704019F063BF2DE9F04F00F020
:1023F0000F07780083B0A0F1020B0025E9464FF0EB
:1024000001084FF6F07647EA051A5046FEF711FA32
:10241000002843D05046FFF759F808FA00F4022C80
:1024200088BF022400215046FFF73EF800900121AA
:102430005046FFF739F800210190002C2ED90BEB04
:102440000500982200FB02FA01EB4102002002EB9A
:10245000011C420900F01F0359F8222008FA03F377
:102460001A4215D000F001020AEB423202EB8C0254
:10247000430802EB830202F1405202F51042B2F827
:10248000182D92B2B24203D903B00020BDE8F08FFC
:10249000401C2628DDD3491CA142D5D36D1C022D3A
:1024A000B1D303B00120BDE8F08F2DE9F041002643
:1024B000934D00280C4640D000F00F01C0F30310EC
:1024C00001290EBF00210229BDE8F081022828BFA2
:1024D000BDE8F0810F18FEF768F95FEA00081CBF3D
:1024E0000020FEF74AF90023982007FB00FC03EBCD
:1024F0004300002200EB031702F001000CEB403018
:10250000510800EB870000EB810000F1405000F51E
:102510001040521CC0F8184D262AEDD35B1C022B2C
:10252000E5D3B8F1000F08BFBDE8F081AE706E7062
:10253000BDE8F0410120FEF720B9FEF736F95FEA69
:1025400000081CBF0020FEF718F9002303EB43002E
:10255000002200EB031CD007800C510800EB8C001C
:1025600000EB810707F1405707F50047521C3C601C
:10257000262AF0D35B1C312BE8D3B8F1000FD5D15C
:10258000BDE8F08110B5FEF73CFF5D49088210BD43
:102590005B4AC1B200F47F43128A914288BF114660
:1025A0004FF0640C01FB0CF1B1FBF2F11A0A02FBD3
:1025B0000C1110F4803F12BF08B2484200B27047BD
:1025C00010B54FF44071534C534819F076FE00207B
:1025D00001232156002910DB0A09120202EB8002B6
:1025E00002F1405202F540420907C90ED2F800C07C
:1025F00003FA01F14CEA01011160401C2628E8D3DE
:1026000010BD10B5434C4FF44071434819F055FECE
:10261000002001232156002910DB0A09120202EBD7
:10262000800202F1405202F540420907C90ED2F879
:1026300000C003FA01F14CEA01011160401C262898
:10264000E8D341F678712F4819F037FEBDE8104005
:1026500041F678712C4819F030BE294810B5808BAE
:1026600000F48170FFF783FA4FF440712A4819F0A3
:1026700024FE41F61851234819F01FFE41F6185167
:10268000214819F01AFEBDE810400020FEF7FDBDFC
:1026900070B51B4C0546A06A401CA062E16A002987
:1026A00018BFFEF7F2FF207850B1206A10B1206AFF
:1026B000401E2062206A002804BF0020FEF75DF85B
:1026C00020212846FEF777F8616A00291CBF2846BA
:1026D0008847FEF765FB022826D11048D0F848133A
:1026E00011F0010F20D0D0F8481341F00101C0F8DB
:1026F0004813D0F8481321F00101C0F848130FE047
:102700001C8400100080003000A00030189D0030B4
:1027100018BD00304487001000C000300050004059
:10272000A06940F00200A0610248016841F0200168
:10273000016070BD5C840010F0B40024634E01237E
:1027400082B0002808BF33701CD00128347018BF35
:10275000747017D05E4D28685E4908432860317850
:102760005D4A002914BF49F608305C48D06014BFA8
:102770005B484FF0BB7090605A48006830F0FF0C27
:1027800008D101E07370E5E7D2F80CC060F3030CE8
:10279000C2F80CC040F2E24CA9B1906840F01800B9
:1027A00090600120009004E00198471E0197FBD241
:1027B0000098471E009728BFCDF804C0F4D2906857
:1027C00040F4805090600120009004E00198471E82
:1027D0000197FBD20098471E009728BFCDF804C090
:1027E000F4D2707818B1D06840F03000D060D2F8E0
:1027F000B00040F00100C2F8B0000120009004E0F9
:102800000198461E0196FBD20098461E009628BFEE
:10281000CDF804C0F4D2D3674FF4E0601061C2F881
:102820008840002918BFC2F89430D06820F03000EA
:10283000D060906820F480509060286820F00400F8
:1028400040F00D7040F08050286002B0F0BC70473E
:102850002148C16821F03001C160816821F48051B4
:1028600081601B48016821F0040141F00D7141F0C5
:102870008051016070471648026816491143016093
:10288000124915480A783AB1826842F0180282600B
:10289000826842F480528260497819B1C16841F07F
:1028A0003001C160D0F8B01041F00101C0F8B010A3
:1028B00070470D49C0B241EA0020074908647047DB
:1028C00005494FF02040086470470000588400100C
:1028D00000800040040034120060004005F4010054
:1028E00020009B00D0FE0300130000A04248414995
:1028F0008161891CC1614A1E4263036823F003039E
:1029000043F00D7343F080530360436923F00103E8
:1029100043F00D7343F08053436103691A4302612E
:10292000364A8260364AC260C2681143C160354986
:1029300000200860704710B501F03DF93148046887
:10294000002C08BF30BFFAD00021016001F037F938
:10295000204610BD10B501F02EF92648294B264916
:10296000421C1C682CB10020186001F028F9204698
:1029700010BD72B648638A6120BF88614A6362B63F
:10298000BFF36F8FBFF34F8FEBE71B48016821F058
:10299000030141F00D7141F0805101601A498160DD
:1029A00001691A4A1143016130BF704772B611497B
:1029B00011484163C91CC161891E816162B67047BB
:1029C0000D480168124A1143016070470A480168C6
:1029D00021F0030141F00D7141F080510160704719
:1029E00072B6044904488161891CC161491E416372
:1029F00062B6704700003412008000403C00341280
:102A0000280034125C8400100800341201003412D3
:102A100003003412704770470022B2EBD10F26D268
:102A20000368B3F1FF3F04BF4368B3F1FF3F17D121
:102A30008368B3F1FF3F04BFC368B3F1FF3F0FD119
:102A40000369B3F1FF3F04BF4369B3F1FF3F07D10F
:102A50008369B3F1FF3F04BFC369B3F1FF3F01D006
:102A6000002070472030521CB2EBD10FD8D3012088
:102A7000704710B40023B3EBD20F30D2D0F800C0AF
:102A80000C68A44522D1D0F804C04C68A4451DD1DF
:102A9000D0F808C08C68A44518D1D0F80CC0CC6818
:102AA000A44513D1D0F810C00C69A4450ED1D0F8BC
:102AB00014C04C69A44509D1D0F818C08C69A4454C
:102AC00004D1D0F81CC0CC69A44502D010BC0020B1
:102AD0007047203020315B1CB3EBD20FCED310BC3B
:102AE000012070472DE9F041054601F06CF8002007
:102AF00021264FF4825784464FF4E0221660C5F831
:102B000000C0116841F004011160116811F0040F58
:102B1000FBD1176080232C460021D4F80080B8F147
:102B2000FF3F04BFD4F80480B8F1FF3F1DD1D4F8B3
:102B30000880B8F1FF3F04BFD4F80C80B8F1FF3F24
:102B400013D1D4F81080B8F1FF3F04BFD4F814803B
:102B5000B8F1FF3F09D1D4F81880B8F1FF3F04BFA6
:102B6000D4F81C80B8F1FF3F08D0C2F800C0401C68
:102B7000C0B20828C2D30220BDE8F081491C20342D
:102B8000B1EBD30FC9D3C2F800C00120BDE8F0817A
:102B90002DE9F041054601F016F80020092684468B
:102BA0004FF4E0231E60C5F800C0196841F004012D
:102BB0001960196811F0040FFBD12C464FF48062A4
:102BC00000212768B7F1FF3F04BF6768B7F1FF3FF7
:102BD00017D1A768B7F1FF3F04BFE768B7F1FF3F20
:102BE0000FD12769B7F1FF3F04BF6769B7F1FF3F16
:102BF00007D1A769B7F1FF3F04BFE769B7F1FF3F0E
:102C000008D0C3F800C0401CC0B20328CAD30220B9
:102C1000BDE8F081491C2034B1EBD20FD1D3C3F809
:102C200000C00120BDE8F0812DE9F05F88468146B3
:102C300004274FF07F0A4FF0020B4FF4E02600F01C
:102C4000C2FF4946424653464FF0060CC6F800B054
:102C500052F8040B41F8040BC6F800C0306810F0BD
:102C6000040FFBD15B1EF1D2002030604C4645467C
:102C70001F20D4E900C3D4E90221D5F800E0E645DD
:102C800004BFD5F804C09C4505D1AB68934204BF8E
:102C9000EA688A4208D07F1E03D34846FFF722FF26
:102CA000CDE70220BDE8F09F10341035401EE0D281
:102CB0000120BDE8F09F70B50D46044600F083FF8B
:102CC0004FF400722146284619F0F2FA012070BD37
:102CD0002DE9F0410546C005ADF5007D14460E46D0
:102CE000C00D25D0A8466FF308086F4600F06BFFB3
:102CF0004FF400724146384619F0DAFAC5F308007D
:102D0000C0F50077A74288BF274668443A46314657
:102D100019F0DDFA4046FFF7E5FE022844D0694687
:102D20004046FFF781FF022843D03D443E44E41B68
:102D3000B4F5007F19D34FF400723146684619F09C
:102D4000C6FA2846FFF7CEFE02282DD0694628464F
:102D5000FFF76AFF02282CD0A4F5007405F5007572
:102D600006F50076B4F5007FE5D2C4B16F4600F0F9
:102D70002AFF4FF400722946384619F099FA224684
:102D80003146684619F0A3FA2846FFF7ABFE022841
:102D90000AD069462846FFF747FF022809D00DF5FB
:102DA000007D0120BDE8F0810DF5007D0A20BDE821
:102DB000F0810DF5007D0B20BDE8F0812E49086003
:102DC000086100F010B82C490860486100F00BB8A9
:102DD0002949486770472849886770472648012174
:102DE0000166016570474FF04022116B10F0010F32
:102DF00018BF21F4404110F0020F1CBF21F44051D4
:102E000041F4805110F0040F18BF21F4406110F01C
:102E1000080F18BF41F4407110F0100F18BF41F0B7
:102E2000C00110F0200F18BF41F0300110F0400F2A
:102E300018BF41F00C0110F0800F18BF41F00301E2
:102E400041F4BE0141F020411163D2F8901010F41A
:102E5000807F1CBF21F0030141F0020110F4007FCC
:102E60001CBF21F00C0040F0080141F4BE0040F00E
:102E70002040C2F890007047001000407047D048D2
:102E80008268D0490A438260C2681143C1604169C7
:102E9000CD4A114341617047C948416921F00101A0
:102EA00041F00D7141F080514161C16821F0400154
:102EB00041F00D7141F08051C160816821F0400105
:102EC00041F00D7141F080518160704710B5BC4CEC
:102ED000A168BC480143A160E1680843E060606903
:102EE000B94908436061B94843F63F71C1600021A8
:102EF00081638164C0F8B01003210A2000F0A5F9B5
:102F00000A2000F0C5F9606920F0010040F00D7062
:102F100040F080506061E06820F0400040F00D70AB
:102F200040F08050E060A06820F0400040F00D705C
:102F300040F08050A06010BDA44A1060516048432A
:102F400090607047A14A10605160484310F0010F33
:102F500018BF401C906070479C49C1F8B000704792
:102F60009A49002818BF01208864704797498863F0
:102F7000C86840F00200C8607047DFF850C2CCF863
:102F80002000CCF82410CCF82820CCF82C300120DC
:102F9000CCF83000DCF8340010F0010F05D020BF71
:102FA000DCF8340010F0010FF9D110F0020018BF66
:102FB0004FF0FF3070478548C16821F00201C160C1
:102FC00070478248C16841F00101C16070477F4B82
:102FD000186259629A6201201864586C10F0010F4F
:102FE00004D020BF586C10F0010FFAD110F0060089
:102FF00018BF4FF0FF3070477448C16821F00101DD
:10300000C16070477148C16841F00401C1607047F8
:10301000027C017B02F03F0241EA02416B4A91656A
:1030200001685162416891628168D1620121116534
:10303000516D11F0010F04D020BF516D11F0010F3F
:10304000FAD1D36D8382D36D1B0CC382136E0383BD
:10305000136E1B0C4383536E8383526EC2F30E4276
:10306000C28311F0020018BF4FF0FF30704757487D
:10307000C16821F00401C16070475448C16841F043
:103080000801C1607047DFF844C1CCF87820CCF863
:103090002000CCF82430CCF828100120CCF87000A7
:1030A000DCF8740010F0010F05D020BFDCF87400CC
:1030B00010F0010FF9D110F0060018BF4FF0FF30EB
:1030C00070474248C16821F00801C160704701683B
:1030D0004FEA31423D49C1F89C204068C1F8A00048
:1030E000C86840F02000C860704701684FEA31426C
:1030F0003649C1F89C208088C1F8A000C86840F01B
:103100002000C8607047314B18625A6299620120F2
:10311000C3F89400D3F8980010F0010F05D020BF39
:10312000D3F8980010F0010FF9D110F0060018BF85
:103130004FF0FF307047254A106251620120C2F8FB
:103140009000D2F8980010F0010F05D020BFD2F8FF
:10315000980010F0010FF9D110F0060018BF4FF0E1
:10316000FF3070471948C16821F02001C1607047E5
:103170001648C16841F01001C1607047A3F1050C09
:10318000124BC3F888C018625A6299620120C3F8D2
:103190008000D3F8840010F0010F05D020BFD3F8D1
:1031A000840010F0010FF9D110F0060018BF4FF0A5
:1031B000FF3070470548C16821F01001C1607047B9
:1031C00000800040400034120100341200900040A2
:1031D0001B4810B5022140F8501F01210161102148
:1031E000416241F206014161002181610421816354
:1031F00090214163416B41F0010141634FF48171C2
:1032000001610161032000F043F80021032000F078
:103210001CF8002010BD10B5032000F045F8084848
:103220004FF480710166002101661021816702213F
:103230004165002010BD0349002008707047000060
:103240000030004060840010704700F00303DA0093
:103250004FF0FF0C0CFA02F24FF0050C0CEBC3031D
:1032600001FA03F300F00C0101F1E021002807DA74
:10327000D1F8140D90431A401043C1F8140D704753
:10328000D1F8000490431A401043C1F8000470477D
:1032900000F01F01012202FA01F14009800000F153
:1032A000E020C0F80011704700F01F01012202FA6F
:1032B00001F14009800000F1E020C0F88011704762
:1032C00000F01F01012202FA01F14009800000F123
:1032D000E020C0F8801270474FF0E021C1F80001F3
:1032E00070474FF0E021C1F8800170474FF0E020B7
:1032F000D0F8000170474FF0E021C1F8800270471C
:10330000084800687047074A11681060084670470F
:10331000044A126800F1100352F8230042F8231007
:103320007047000008ED00E002210C20FFF78DBF80
:10333000B8488268B8490A438260C2681143C160D4
:103340007047B448816821F4805141F00D7141F01B
:1033500080518160C16821F4805141F00D7141F0CC
:103360008051C1607047AD4881B0016F11F4007F9A
:10337000FBD1816E11F0010F1CBFD0F884100091B9
:1033800004D0D0F88410009A9142FAD0016F11F461
:10339000007F04BF4CF27101016642F24131816647
:1033A00001B070479D4981B04FF40D528A660A6F93
:1033B000CA66012898BF012005D9401EB0F5803F9C
:1033C00028BF4FF6FF7082B24FF05C5040EA0220F7
:1033D00048664FF01140C1F88000086F10F4007F7C
:1033E000FBD1886E10F0010F1CBFD1F88400009053
:1033F00004D0D1F88400009A9042FAD0086F10F4FB
:10340000007F04BF4CF27100086642F241308866CA
:1034100001B07047814881B0016F11F4007FFBD18A
:10342000816E11F0010F1CBFD0F88410009104D000
:10343000D0F88410009A9142FAD04FF40D51816671
:1034400001B070477348806810F4805008BF70471F
:103450007248806E00F0010070477048406EC0F303
:103460000F2070476D48D0F88400704710B50C20CD
:10347000FFF726FF0C20FFF70BFF68490220486783
:1034800010BD664910B5032088670C20FFF70CFFBC
:10349000BDE810400C20FFF713BF614A11681060AF
:1034A000084670475D4810B5016FC1665C4800680A
:1034B000002818BF80475B48016841F480510160D3
:1034C00010BD574840687047524810B5826852494D
:1034D0000A438260C2681143C16050490320886773
:1034E0000C20FFF7E1FE0C20FFF7EAFE00F05CF98C
:1034F0004D4B0420C3F888004FF6FF70C3F88C00D2
:1035000072B66033FFF74EFF4FF40070186062B67A
:1035100010BDF8B572B64148016F11F4007FFBD1C0
:10352000816E11F0010F1CBFD0F88410009104D0FF
:10353000D0F88410009A9142FAD04FF40D51816670
:1035400039494FF400320A6662B6D1F80412314D9F
:10355000002946D0324C4FF6FF73591AA160AA6970
:10356000D5F81CC002F00F020CF00F0C6244121DC3
:1035700001FA02F2A2F54341DFF8B0C051396145CA
:103580002FD2D0F88400191AE160B1F5803F28D21B
:10359000274B4FF0000CA1FB03070CFB037301FB4F
:1035A0000C31634618F098FE401C40082061B0F5CD
:1035B0007A7F38BF4FF47A701E4B9968002908BF94
:1035C00098605A681A609968C3E901108A421BD949
:1035D000824205D9814201D9616002E0606000E069
:1035E000626000F0EDF8A86820F4805040F00D70A3
:1035F00040F08050A860E86820F4805040F00D70E2
:1036000040F08050E860F8BD8242E9D88142E5D8B8
:10361000E2E70000008000400010341200C00040CB
:10362000648400105C84001000A000404F622500FC
:1036300000E1F505D89000100F4881680F4A11434A
:1036400081600F48016841F404710160001F016846
:1036500041F004010160016841F010010160704710
:10366000084908607047BFF34F8F08490648086053
:10367000BFF34F8FFEE700000080004004003412CB
:1036800014ED00E008ED00E00400FA050CED00E0A8
:1036900015488168154A114381601003416941F062
:1036A00001014161016A21F00F0211490A430262DE
:1036B000104B8A1EC3F8C420016570474FF04020AC
:1036C000006900F0700070474FF040200A4940F850
:1036D000301F0A4941600A4901660A49416670473C
:1036E0004FF04020406870470080004004003412D2
:1036F00003005FA000600040C0845FA095995FA0B8
:103700000A005FA000005FA0022824BF00207047CD
:10371000E04B53F8202043F820101046704770B556
:10372000DD4C206FDB4D10F0010F05D00120E0666D
:103730002868002818BF8047206F10F0020F08BFCC
:1037400070BD0220E0666868002808BF70BDBDE853
:1037500070400047D14810B58268D1490A43826061
:10376000C2681143C160CC4902220A6501230B667D
:103770000323CB664A65816821F0800141F00D7119
:1037800041F080518160C16821F0800141F00D71EC
:1037900041F08051C1600920FFF77AFD0221BDE8A8
:1037A00010400920FFF751BDBC488268BC490A435C
:1037B0008260C2681143C160B74902200865704742
:1037C000B54902204865B548816821F0800141F083
:1037D0000D7141F080518160C16821F0800141F09C
:1037E0000D7141F08051C1607047AC488068C0F3F2
:1037F000C0107047A848016F11F4007F14BF4FF448
:1038000040714FF480710166704710B5A24CE06FB3
:1038100010F0020F4FF0010018BF0320606700F0A6
:103820006EF99E498A69C96902F00F02D04001F021
:103830000F01C8400521B0FBF1F04FF405710009FC
:10384000C4F8801018F04DFD964A974B18F04EFDC5
:1038500018F051FDC4F88400206F10F4007F14BFED
:103860004FF440704FF48070206610BD8A48016F9D
:1038700011F4807F14BF4FF440714FF40071016662
:103880007047854B30B4DA6F12F0010F14BF03227A
:1038900002225A6700EB4005C5EBC010C1EBC00027
:1038A0004FF4FA744C43C0EB001000EB40007F492A
:1038B00004EBC000A1FB0010784900224FF0020C7D
:1038C0008C69C008C96904F00F0401F00F0121449C
:1038D000C8400521B0FBF1F0B0F5803F05D3511C85
:1038E0004008CAB2B0F5803FF9D242EA0C2141F05B
:1038F0001001C3F88810C3F88C00186F10F4807F93
:1039000014BF4FF440704FF40070186630BC70471D
:103910006148016F11F4003F14BF4FF440314FF480
:103920008031016670475C48016F11F4803F14BF1D
:103930004FF440314FF40031016670475648006F34
:10394000C0F3002070475448006FC0F34020704718
:1039500052498968C1F3C011002904BF0020704793
:103960004D4900280CBFD1F80002D1F8040270477D
:103970004A4B9A68C2F3C012002A04BF0020704765
:10398000454A00280CBFD2F88000D2F88800C0F366
:103990000A200CBFD2F88020D2F8882002F00F0253
:1039A000D3F818C0DB690CF00F0C03F00F0363446D
:1039B0001A449140012202EB400048433C49A1FBDC
:1039C0000010000970473B4901200870704770B42F
:1039D000324B322251439A69D3F81CC002F00F02D5
:1039E0000CF00F0C6244121DD14008BF012104D01D
:1039F000B1F5803F28BF4FF6FF719A68C2F3C0123D
:103A0000002A1CBF70BC7047D3F808C0244A4CEA97
:103A1000020CC3F808C0D3F80CC04CEA0202DA600A
:103A20001D4A4FF0020CC2F850C04FF40034146627
:103A30000425C2F88850C2F88C101F4DD566C2F814
:103A400074C01E4902283CBF124E46F820100021C7
:103A5000184801704FF400711166017819B920BF40
:103A600001780029FBD014669567D566C2F854C06A
:103A7000986820F0800040F00D7040F08050986011
:103A8000D86820F0800040F00D7040F08050D86081
:103A900070BC70477C84001000A000400080004093
:103AA000800034127B14AE47E17A843FCDCCCCCC7D
:103AB0001F85EB5178840010020002027759000044
:103AC0004FF0E0210020886108611F49486070477D
:103AD00010B54FF0E02460610020A0610221401E7B
:103AE000FFF7B3FB0720206110BD4FF0E02100205D
:103AF0000861704714480188491C018070471248CA
:103B0000806870472DE9F0410F4C0027054627805B
:103B1000A0684FF47A71B0FBF1F04FF0E026401E40
:103B20007061B7610221C81EFFF78FFB072030616B
:103B30002188A942FCD33761BDE8F081034948439D
:103B400001498860704700008484001040420F00E3
:103B5000704770B505464FF40D500406A06603206B
:103B6000E066264860664CF2710020662448C4F87E
:103B7000800042F24630A06602210020FFF765FB7C
:103B80000020FFF785FB002D08BF70BDA06E42F23C
:103B900041310843A06670BD012110B588078167D7
:103BA0004FF40D5181660020FFF77EFBBDE8104009
:103BB0000020FFF785BB012081074867704701207F
:103BC0008107886770474CF271008107086670476B
:103BD0000C4A11681060084670470A4808B500682A
:103BE00018B18047002818BF08BD4CF27101880742
:103BF0000166016FC166006F009008BD075E5F3708
:103C000000AF2F919084001070B5FD4C00254FF44B
:103C1000E46125706570E570FA4818F04EFB4FF4CA
:103C2000E461F94818F049FBA56025714C21F7487B
:103C300018F043FB4C21F64818F03FFB65717421E6
:103C4000F44818F03AFB7421F34818F036FBE560AD
:103C5000A5717421F14818F030FB7421F04818F078
:103C60002CFB256170BDE649002048707047E44890
:103C700040787047E2480079002818BF012070475B
:103C8000DF488079002818BF01207047DC48407960
:103C9000002818BF01207047D948C078002818BFF5
:103CA00001207047DD48704770B5DE4A0546107840
:103CB00051784218520014462946D84818F007FB9C
:103CC00022462946D64818F002FBCD4901208871CA
:103CD00070BDCB4800697047C948407800EB40018F
:103CE000C1EB4010CB4901EB800070472DE9F0415A
:103CF000C34D0446C7496A78CB4F02EB4200C0EB84
:103D00004210CA4E01EB80033A78307821461044C5
:103D10004200184618F0DBFA6A78BF4902EB42000D
:103D2000C0EB421001EB80033A7830782146104412
:103D30004200184618F0CBFA01206871BDE8F08106
:103D4000AF48C0687047AE484078C0EBC001C1EBD7
:103D50008010AC4901EB401070472DE9F041A84EAE
:103D600007463078002814BFB148B248047814BF21
:103D7000B148B248057804FB05F8FFF780F82946FA
:103D80002046FFF7D9F870789F4CC0EBC001C1EB1B
:103D9000801004EB4012A4F5E46101EB40103B46B7
:103DA0000146FFF7EAF8FFF777F870784FEA480224
:103DB000C0EBC001C1EB801004EB4010394618F095
:103DC00086FA0120F070BDE8F0812DE9F0478C4DB6
:103DD00004468C496A78DFF85882C2EBC200C0EB17
:103DE000821001EB40132878DFF84892924E934FEF
:103DF000002815BF98F8000099F8000032783A784A
:103E000000FB02F04FEA40022146184618F05FFA24
:103E10006A787D49C2EBC200C0EB821001EB401C06
:103E200028782146002815BF98F8002099F800202E
:103E300033783B7802FB03F04FEA4002604618F00B
:103E400046FA0120E870BDE8F0876D488068704749
:103E500070B57B4C0546014622786C48520018F03C
:103E600036FA227829465200694818F030FA644937
:103E70000120087170BD2DE9F04FDFF88481ADF2AB
:103E8000647D98F80300CDF8440798F80400CDF855
:103E9000400798F80500CDF83C0798F80600CDF8E3
:103EA000380701F0ABF90446FDF7B6FDCDF85C0725
:103EB000FDF789FFCDF85807FDF7F1F9CDF8540764
:103EC000FCF771FFCDF84807FCF76AFF0746FDF7DE
:103ED000A5FDDDF8480710F0010F02D0FDF779FFCE
:103EE00004E00020FDF7D1F9FDF7ACFF98F80200DF
:103EF0001E250026002804BF0420C8F8180007D09B
:103F0000022C18BF0A2008D0C8F8180088F80260F0
:103F10004FF0010A022F19D109E00FF032FE10F420
:103F2000817F14BF0F20C8F81850EDD1EEE7022CA6
:103F300018BF052C0AD1FDF779F908300009022CC9
:103F400018BFC8F818503AD088F802A0D8F818005E
:103F50000428BCBF0420C8F8180098F80200B8F87C
:103F60001810000240EA014040F0010200239121B4
:103F7000072009F003FA37464FF0000B05F045F82B
:103F8000012826D00DF5E460FEF75EF9002800F068
:103F9000A3820DF5E46005F00BFF002088F8010016
:103FA000D8F81800C01E8642CABF874201240024E8
:103FB000DDF82C0718B3DDF8400770B15BE04FF473
:103FC0007A7141434FF47A7091FBF0F0C8F8180011
:103FD000BAE74FF0010B00F068BADDF82C978CB30C
:103FE000174D494628784200084818F070F928789B
:103FF00049464200064818F06AF988F804A03AE0F9
:1040000094840010E49000100498001044A600105E
:1040100090A60010DCA6001050A7001038A80010D1
:10402000ACA80010D4840010D1840010D2840010F9
:10403000CF840010CC840010D0840010CD840010F8
:10404000D3840010FFE7FEF71AFFFF4D0121287807
:10405000FEF772FFFD4A4B46A2F14C010846FEF7FF
:104060008CFFFEF719FF287849464200F74818F000
:104070002EF988F804A0DDF82807002800F0D78082
:10408000DDF84407002840F0D28098F80000DDF801
:104090002857E0BBD8F80890B9F1000F24D0EC48BD
:1040A0000078CDF85007EB480078CDF84C07FEF7C4
:1040B000E6FEDDF84C17DDF85007FEF743FF294612
:1040C0004A460846FEF783FFFEF7E6FEE248007820
:1040D000022804BF484605F03EFBDF480078092867
:1040E00004BF284605F037FBDC480078012816D9C4
:1040F000DFF8649399F80000042804BF284605F00F
:104100002AFB2946684618F0FBF8054600E006E061
:1041100099F80000052804BF284605F01CFBCCB325
:1041200098F8010098F80020C0EBC001C1EB8011A5
:10413000CB48002A00EB411029460CBFC94AC44AAB
:10414000137814BFC34AC84A127803FB02F24FEA3D
:10415000420218F0BCF898F80100C0EBC001C1EBB6
:104160008011C24800EB411398F80000294600284E
:1041700014BFB748BB48007814BFB64ABA4A127891
:1041800000FB02F04FEA4002184618F0A0F888F849
:1041900003A03DE0FFE7CDF84C5798F80000002859
:1041A00014BFAB48AF4890F8009014BFA948AE4880
:1041B000057809FB05F0CDF85007FEF760FE2946AB
:1041C0004846FEF7B9FE98F80100A84DC0EBC001C3
:1041D000C1EB801005EB4012A5F5E46101EB401046
:1041E0000146DDF84C37FEF7C8FEFEF755FEDDF858
:1041F0005007420098F80100C0EBC001C1EB8010ED
:1042000005EB4010DDF84C1718F061F888F803A0B2
:104210009148007803280AD198F80100C0EBC0014A
:10422000C1EB80118E4800EB411005F094FADDF8E7
:10423000300700287DD0DDF83C07002879D198F8B8
:104240000000DDF8305748BBD8F80C90B9F1000FEA
:1042500024D087480178874800780844401C4008EB
:10426000019002200090FEF70AFEDDE90010FEF743
:1042700069FE29464A460846FEF7A9FEFEF70CFEEF
:104280007D480078022804BF484605F06FFB7A4855
:104290000078092804BF284605F068FB4CB398F85D
:1042A0000100DFF8D09100EB4001C1EB40117348F1
:1042B00000EB81036E482946027899F8000010440B
:1042C0004200184618F003F898F80100684A00EB1D
:1042D0004001C1EB40116A48127899F8003000EBB8
:1042E00081001A442946520017F0F1FF88F805A012
:1042F00030E05F48009501785E4800780D18FEF7C1
:10430000BEFD681C40080221FEF716FE98F8010069
:10431000DFF86C9100EB4001C1EB4010A9F1740192
:1043200009EB800201EB80010846009BFEF725FEA9
:1043300000E01EE0FEF7B0FD98F801006A0000EB17
:104340004001C1EB401009EB8000009917F0BFFF5E
:1043500088F805A04848007803280AD198F8010099
:1043600000EB4001C1EB4011444800EB810005F037
:10437000FDFADDF83407002863D0DDF8380700289F
:104380005FD198F80000DDF8345740BBD8F81090A2
:10439000B9F1000F23D03B48017840780844401C15
:1043A0004008019002200090FEF769FDDDE9001051
:1043B000FEF7C8FD29464A460846FEF708FEFEF706
:1043C0006BFD31480078022804BF484605F0E8FB41
:1043D0002D480078092804BF284605F0E1FB29484C
:1043E0000178407874B108444400224629462748A1
:1043F00017F06DFF22462946254817F068FF88F818
:1044000006A017E00C18FEF73AFD601C40080221D8
:10441000FEF792FD1E4A2B46A2F174010846FEF7F4
:10442000ACFDFEF739FD62002946194817F04FFF31
:1044300088F806A014480078032804BF134805F044
:10444000AFFBFDF75EFF25E0D384001090A60010BF
:10445000CF840010D08400103D850010CE84001061
:10446000E4900010CC840010CD840010049800105B
:10447000D1840010D284001042850010DCA6001008
:1044800050A70010D48400104785001038A80010F1
:10449000ACA80010D8F81800761C7F1C8642A8BF74
:1044A000874211DBD8F8140070B1FDF7B7FADDF8D8
:1044B0005407FCF7EAFEDDF85C0790B1DDF8580719
:1044C00068B1FDF7BFFC0CE0DDF8480710F0010F04
:1044D00008BFFDF7B7FC51E500F0DDFE4EE5FDF746
:1044E00078FCBBF1000F04BF0420C8F818000FD0FF
:1044F000DDF8440788F80300DDF8400788F8040079
:10450000DDF83C0788F80500DDF8380788F8060074
:10451000B8F818104FEA0B2040EA0142002391211D
:10452000072008F02BFF0DF2647D5846BDE8F08FA0
:1045300010B50024FDF739FCFF4910F0020F0AD036
:10454000CA78002A08BF012410F0040F03D00A79AA
:10455000002A08BF012410F0010F03D04A79002A75
:1045600008BF012410F0200F03D08879002808BF6D
:1045700001240020002C08BF10BD00200870BDE8F9
:10458000104078E408B50F2100F03AFF012804D16B
:10459000FFF7CEFF009001F0A2F8E748C1780029AC
:1045A0001CBF4179002906D0817900291FBF0079FD
:1045B0000028012008BD002008BD08B50F2100F02B
:1045C0001FFF012804D1FFF7B3FF009001F087F827
:1045D000D948C17800291CBF4179002906D08179CA
:1045E00000291FBF00790028012008BD002008BD58
:1045F0007047D14900220028CA700A714A718A7135
:104600001CBF0120887000F011BD10B54FF4E461AB
:10461000CA4817F052FEBDE810404FF4E461C848A4
:1046200017F04BBE2DE9F041C34D069A29780029B9
:1046300014BFC449C4490978D21A4A4303FB01F4A0
:1046400069785200C1EBC103C3EB8111BB4B164625
:1046500003EB411101EB440300EB44010F46184604
:1046600017F035FE68783246C0EBC001C1EB801010
:10467000B34901EB401000EB4400394617F027FE28
:104680000120E870BDE8F0812DE9F047AA4F80468F
:1046900008983978002914BFAA49AB490D78A0EBD6
:1046A000030905FB09F603FB05F4FEF7E8FB4946A1
:1046B0002846FEF741FC7878A14DC0EBC001C1EB64
:1046C000801005EB401101EB4402A5F5E46101EB1C
:1046D000401000EB440008EB440843460146FEF757
:1046E0004CFCFEF7D9FB78787200C0EBC001C1EB3F
:1046F000801005EB401000EB4400414617F0E7FD49
:104700000120F870BDE8F087002818BF01208A4911
:10471000C870704710B5884C002804BFA06010BD59
:10472000DFF828C287490B7889490A7801465A433D
:104730005200604617F0CBFD8448A06010BD10B554
:104740004C21844817F0B9FDBDE810404C21824847
:1047500017F0B3BD7F487047002818BF0120764985
:104760000871704710B574217C4817F0A6FDBDE8AC
:10477000104074217A4817F0A0BD002818BF01200E
:104780006D494871704710B56B4C002804BFE0605C
:1047900010BD74220146734817F099FD7148E0601E
:1047A00010BD10B57421704817F087FDBDE81040AA
:1047B00074216E4817F081BD002818BF01205E49A2
:1047C0008871704710B55C4C002804BF206110BD93
:1047D00067490A78497811444A000146654817F04C
:1047E00076FD6448206110BD70B5534C002105462C
:1047F000E17021716171A17100F018FC002D14BFEE
:10480000012000202070BDE87040FFF734BB2DE987
:10481000F04F89B04FF4E4614C4817F04EFD74211D
:10482000504817F04AFD7421524817F046FDFDF735
:10483000BCFA0446FDF7F0F80890FDF7C4FA0190C1
:10484000FCF72DFD0090FDF7E9F80020FCF71DFDB9
:10485000FDF7F8FA00252E4604F0D7FB012868D0B2
:1048600002A8FDF7F1FC002864D002A805F0A0FA28
:1048700014F0020F1CD03348DFF8D0B0DDF81090F0
:1048800090F800803248DA460778FEF7F8FA0120FF
:10489000FEF766FB39464046FEF754FB5246494652
:1048A0005846FEF794FB0020FEF75AFBFEF7F4FA99
:1048B00014F0010F20D03048DFF8A8B04FF0020804
:1048C00001782E48DA46DDF8189000780844401C3C
:1048D0004708FEF7D4FA0120FEF742FB414638466E
:1048E000FEF730FB524649465846FEF770FB002063
:1048F000FEF736FBFEF7D0FA14F0200F47D01C4825
:10490000DFF870904FF0020B01784078C8460844F9
:10491000401C4FEA500A079FFEF7B1FA0120FEF74C
:104920001FFB59465046FEF70DFB424639464846A6
:1049300026E034E040E0000094840010E490001091
:1049400004980010CF840010CC840010249F001025
:10495000D084001044A6001090A60010DCA6001021
:1049600050A70010C4A7001038A80010ACA8001071
:10497000D484001020A90010D1840010D28400102B
:10498000FEF725FB0020FEF7EBFAFEF785FAFDF7B0
:10499000B8FC6D1C102D03D2FDF754FA5CE701261C
:1049A000FDF73CF80098FCF770FC089848B10198B6
:1049B00028B1FDF747FA04E000F06DFC4CE7FDF785
:1049C00008FA96BBF84D14F0020F4FF001070DD016
:1049D000F648009710230178F548007801FB00F2B3
:1049E000F449084617F091FCF248A86014F0010F52
:1049F0000CD0F148009710230178F04800780A188D
:104A0000EF49084617F081FCED48E86014F0200FEC
:104A10000BD0EC4800971023017840780A18EA4937
:104A2000084617F072FCE848286109B03046BDE836
:104A3000F08F012070472DE9F0414FF43F300027FF
:104A4000D0E90015D0E903464BF6BB38ADF5007D43
:104A500041452BD04FF40071684617F02EFCFF2221
:104A60004FF40071684617F055FCFF2060F307050E
:104A70002D2060F3070460F30F24282060F317440F
:104A8000CDF80080CDE90346CDE901574FF43F341E
:104A90002046FEF727F869462046FEF7C5F80128AC
:104AA0001EBF00200DF5007DBDE8F08101200DF551
:104AB000007DBDE8F0814FF43F3070474FF43F3147
:104AC000042804BFC87A704710DC002804BF0879A6
:104AD0007047012804BF087A7047022804BF487A4B
:104AE0007047032804BF887A70470BE0142804BF7E
:104AF000087B7047152804BF487B7047162804BF01
:104B0000887B7047FF2070472DE9F0434FF43F3C0E
:104B1000ADF5017DDCE9015461F3070462F30F2474
:104B2000DDF82092DCE9037860F3070563F31744AE
:104B300069F31F64FF224FF400716846DCF80060DF
:104B400017F0E8FB0096CDE90154CDE903784FF466
:104B50003F342046FDF7C6FF69462046FEF764F85D
:104B6000012818BF00200DF5017DBDE8F0832DE977
:104B7000F04F4FF43F33ADF5017DD3E90274D3E933
:104B80000056904689468246FF224FF400716846DF
:104B9000D3F810B017F0BEFB6AF3070469F30F24D3
:104BA00068F31744CDE90274CDE900564FF43F3461
:104BB000CDF810B02046FDF795FF69462046FEF778
:104BC00033F80DF5017DBDE8F08F2DE9F04F00279A
:104BD000ADF5017D7D4C42F20F783D461420FFF784
:104BE0006DFF40B202901520FFF768FF4FFA80F981
:104BF0001620FFF763FF40B201901620FFF75EFF1B
:104C0000404240B20090FDF7D0F8DFF89CA1834607
:104C100000208AF803008AF804008AF805008AF860
:104C2000060000F003FA00208AF80000FFF723F9DD
:104C30001BF0010F04D017F072FB012808BF0127F9
:104C40001BF0020F7ED062489AF80110002690F8FF
:104C500000C06048C1EBC102C2EB811100785E4A1E
:104C6000002802EB4112C8BFACF1010A1DDD002192
:104C7000BAF1000F16DD01F1010B01FB00630BFB24
:104C8000006B32F8133032F81BB0A3EB0B031BB2EE
:104C9000002BB8BF5B421BB2AB42C8BF1D46491CCC
:104CA0005145E8DB761C8642E1DBA945B8BF47F0F9
:104CB00002070026B146BCF1000FC8BFA0F1010AEF
:104CC0001BDD0021BAF1000F13DD09FB001332F8E0
:104CD00013B002EB43035B88ABEB03031BB2002B67
:104CE000B8BF5B421BB2B342C8BF1E46491C514508
:104CF000EBDB09F10109E145E3DB0299B142B8BF01
:104D000047F002074FF00009BCF1000F13DD00234C
:104D100000280CDD09FB003132F91110A142C8BF97
:104D20000C464145B8BF88465B1C8342F2DB09F163
:104D30000109E145EBDB0198A04202DB0098404508
:104D400003DD00E001E047F002074FF43F32C8F115
:104D50000001D2E9018066F3070065F30F20D2E974
:104D600003AB64F3174061F31F600446D2F8009070
:104D700067F30708FF224FF40071684617F0CAFA7C
:104D8000CDF80090CDE901844FF43F342046CDE9C1
:104D900003ABFDF7A7FE69462046FDF745FF0DF57D
:104DA000017DBDE8F08F000094840010CF840010D6
:104DB000D0840010249F0010D1840010D2840010F1
:104DC000C4A70010D484001020A90010F1D8FFFF60
:104DD000CD840010CC840010E4900010FA48808943
:104DE0007047F948C089704770B515460E460446AD
:104DF00008F0BAFE002C18BF70BD042806D0F34896
:104E0000006890F82400A84288BF70BD3046BDE815
:104E1000704017F089BADDF800C0084312BF52EAAB
:104E2000030000208CF800007047E7484069704795
:104E3000E549012048617047E34900204861704717
:104E40000143E14818BF142AD4BF01210021416168
:104E50007047DD480021C171018270472DE9F0479C
:104E600090468946044608F0FDFD0027D64E0028EE
:104E700002BFF7713782BDE8F087B6F910008442AF
:104E8000C8BF3482204617F054FA04460D46B6F9DE
:104E9000100017F04EFACE4ACE4B17F027FA2246F2
:104EA0002B4617F083FB13D2B9F1010F10D0F07924
:104EB000401CC0B2F071032898BFBDE8F087F771BD
:104EC000378201203071801EC8F80000BDE8F087ED
:104ED000F771BDE8F0872DE9FF5F0546BE480A2659
:104EE000002490F80090BD48B74FDDF838B090F836
:104EF00000809246012B08BFBBF1000F1BD008F0C9
:104F0000B1FD01281DD0B889012888BF1E2336D9DC
:104F100079890020A1421CBF7C81B871002119EB66
:104F200008021FD035F911C09C4517DDB87104B0D7
:104F30000020BDE8F09FB879052828BF05201ED3C2
:104F40001CE0BBF1010F08BF4123E1D03C23012449
:104F50000526BAF1000FC8BF3323D9E7491C89B22F
:104F60008A42DFD8B979491CC9B2B971B14206D9B0
:104F700001994FF0FF320A6001213971B87104B014
:104F80000020BDE8F09F70B51E4615460C4608F09F
:104F900069FD01281AD10021DFF82CC2002DC2BF03
:104FA0008CF80510002070BD012E0FD09CF8050074
:104FB000401CC0B28CF805000A2807D94FF0FF301A
:104FC000206001208CF804008CF80510002070BDD2
:104FD00000207D4A034601291CBF137070471078DA
:104FE000401CC0B21070042826BF1370022001209C
:104FF000704708B502237A490A787A490978891EE8
:1050000000910021FFF70EFB012008BD744908B58F
:105010000A78744902230978891E00910021FFF75C
:1050200033FB012008BD6848007A704710B508F0CE
:1050300019FD002808BF10BD08F017FD002301214D
:10504000BDE810401A46022008F098B9664A02806E
:10505000428000218280C18001815342438181814D
:10506000C18101824182017501834183C2827047FF
:105070002DE9FF4F83B01446DDE910A70546DDF8A2
:1050800048B008F071FD0195DFF83C8100252E46FF
:1050900088F8085008F0F4FC4FF0010948BB08F00C
:1050A000BBFE014601AA1398FFF7D8FE3B465246C5
:1050B00001A9CDF800B00498FFF70DFF08F0D2FC6D
:1050C000012816D1BAF1000FC8BF88F8056010DCBE
:1050D000012F0ED098F80500401CC0B288F80500DA
:1050E0000A2806D94FF0FF30019088F8049088F81C
:1050F000056008F0E5FE012808D1D8F8140028B1B1
:105100000025012F18BF88F800600CD00198344AA0
:105110003449B0F1FF3F04BF98F8040001280FD0D4
:10512000022D2DD036E098F80000401CC0B288F85F
:105130000000042826BF88F8006002250125E5E765
:1051400088F8046088F80890012D18BF022D08D057
:10515000002C04BF07B0BDE8F08F2046FEF735FEF7
:1051600018E0002C04BF07B0BDE8F08F2046097896
:105170001278891E009102230021FFF753FA09E0FB
:1051800044B109781278891E00912046022300213B
:10519000FFF77AFA0198002807BF98F80200012863
:1051A00007B0BDE8F08F88F8026088F80890002CFE
:1051B0001CBF2046FEF7D1FD0698002818BF17F047
:1051C000BDF807B0BDE8F08FB0840010D4850010A2
:1051D000CDCCCCCCCCCCE43FD1840010D284001018
:1051E000CC840010CD840010F1D8FFFF10B505F07D
:1051F00097FD05F042FE002010BD0000FE4800783B
:105200007047FD4840787047FB480078022805D079
:1052100005281CBF0020704704F0DFBF08F0A4BCC5
:10522000F5490870704770B5F34E04460D46307866
:10523000A04212D002281AD0052814BF002004F082
:10524000CCFF44EA05213278002341EA024141EAD9
:1052500000626121072008F091F87570072C28BFC3
:1052600070BDDFE804F016070B13160F160008F0E8
:105270007BFCE6E7284600F03FFA0AE0284608F003
:105280006EFC06E0284604F09DFF02E0284608F088
:105290001DF9347070BDD94900200968B1F8641057
:1052A00011F4807F08BF7047FDF745BBD34900204C
:1052B0000968B1F8641011F4807F08BF7047FDF7EA
:1052C00049BBCE4900200968B1F8641011F4007F91
:1052D00008BF704717F037B8C84900200968B1F80F
:1052E000641011F4806F08BF704717F031B8C249DD
:1052F000887800281CBF401E8870704770B5C04970
:10530000D1F8CC00BC4C10F0030F0AD040F4BE0022
:1053100040F02040C1F8C800A078002804BF012058
:10532000A070B8488068B54D10F0020F296807D109
:105330004FF04020406910F0010F01D0A07840B13B
:10534000B1F86410002011F4807F18BFFDF702FB54
:1053500007E0B1F86410002011F4806F18BF16F058
:10536000F7FFA949084208BF70BD2968496E090CBA
:10537000A17070BD10B572B6FEF70EFCBDE810400E
:10538000FEF771B910B5012802D0022805D008E057
:105390004FF44330FDF7A6FB03E04FF040219B485C
:1053A000086772B6FEF7F8FBBDE81040FEF75BB980
:1053B0009149002818BF0120C87070478E48C078F6
:1053C000002818BF012070478B48406970478A4801
:1053D00000697047884988617047874880697047CD
:1053E0008549C86170478448C0697047834802682E
:1053F00002F5C073118A508A02F5A072FCF7AFBDA6
:105400002DE9F04FDFF8F09197B08A46C9F8140003
:1054100005F0B6FBC9F81000002800F0A58090F850
:1054200000C089F804C0417889F8051083780446E3
:105430000CF1010089F8063000F0FE0089F8070041
:10544000E27889F80820207989F80900607989F8DC
:105450000A0009F10C05A0792870E07968702078BD
:1054600089F80B006046FCF7BBFE99F80A1099F822
:105470000900FCF7D8FE69782878FCF7DEFE69465B
:10548000204605F0A0FB608AD9F8185000281CBF00
:105490006843050BB4F81A80D9F81C60B8F1000F06
:1054A00008BF4FF48058678C002F08BF4FF4805717
:1054B00000201AF0040F18BF4FF485701AF0080F7F
:1054C00018BF40F004001AF0020F1CBF40F2012187
:1054D00008431AF0010F18BF40F48460616A6FF34B
:1054E0000F0A08406FF30F0108434AEA000A0098C8
:1054F000109004981190089812900C9814900198AC
:1055000013900798159010A95046FCF753FB1AF01A
:10551000020F65D005F045F85FEA000B31D005F0C9
:1055200057F86843050B59460020FBF7CDFE218A4A
:1055300000291CBF0020FBF746FF05F069F8704307
:10554000000B00F50060010A0820012202FA00F3B6
:105550000B4201D1401EF9D5061FA07B002818BFC1
:10556000A0F1010B17D112E024480068B0F86400E4
:1055700010F4807F18BFFDF7EDF9002017B0BDE8EB
:10558000F08FB4F80CB0BBF1000FCCD1CFE7002006
:10559000FBF79CFF8346E07B002814BF401EFBF70F
:1055A000D5FF0BEB0601042903DD711A0E1D042142
:1055B00003E00029BCBF761A00210644042E03DD57
:1055C000301FC540042604E0002E02DA70428540F8
:1055D00000260020FBF793FF31460020FBF7CFFFAA
:1055E0001AF0010F30D0A18A00291CBF0120FBF75F
:1055F0006BFE268BA6B10BE0C8840010D48500108A
:10560000006000400080004008000300AD2007B0AB
:1056100031460120FBF7D7FE31461120FBF7D3FEC0
:10562000A67D3EB1711E0120FBF769FF711E11209E
:10563000FBF765FFE67D3EB1711E0120FBF79FFF82
:10564000711E1120FBF79BFF1AF0200F23D0A18BB6
:1056500000291CBF0220FBF737FE268C3EB13146E5
:105660000220FBF7B0FE31461220FBF7ACFEA67F0E
:105670003EB1711E0220FBF742FF711E1220FBF7A4
:105680003EFFE67F3EB1711E0220FBF778FF711EE0
:105690001220FBF774FFE07A00281CBF0001FBF723
:1056A0004FFD029804F059FF039830B12B4699F84A
:1056B000052099F8041016F050FE3A464146284657
:1056C00016F050FE0598FFF725F80998FFF75BF8EC
:1056D0000D98FFF777F817B00120BDE8F08F10B5EF
:1056E000FCF724FB04F041FF02490020086101207F
:1056F00010BD0000C8840010FE4908707047FD48C6
:1057000000787047FC4810B4FC4A0168914218D1F7
:105710004168B1F5887F14D80022D0F808C003464C
:105720001146B2EB9C0F24BF10BC704753F82140C8
:10573000491C2244B1EB9C0FF8D3002A04BF10BCD3
:105740007047002010BC7047EB48FDF7CBB9E94922
:105750000120087070472DE9F34FE5B00020459017
:105760008A465590549072B6FCF71FFB0646FEF72A
:105770003CF848B1FEF7E2F85590FEF7C9F8FEF79D
:10578000E2F85490FEF7CFF8FCF709FAFCF744F979
:105790005C90FCF718FB5B90FCF740F9FCF7A1FB71
:1057A0005D900020FCF797FBFDF74CFE5A90FDF74B
:1057B00031FE4FF49350FDF79EFD62B60020074680
:1057C00036AD45F82070401C0628FAD3DFF8308348
:1057D00016F0020F4FF001040AD041F6185140466E
:1057E000369416F06AFD41F61851C64816F065FD6C
:1057F000DFF8149316F0010F15D04FF41871C34859
:1058000016F05BFD4FF41871484616F056FD012066
:10581000FBF70FF8002818BF38941120FBF709F8A0
:10582000002818BF399416F0200F15D04FF41871C6
:10583000B64816F042FD4FF41871484616F03DFD8B
:105840000220FAF7F6FF002818BF3A941220FAF760
:10585000F0FF002818BF3B94DFF8B492A54E3698AD
:105860004FF0405B68B300210846FBF71DFE009037
:1058700001210020FBF718FE019099F800008DF837
:105880000800A4480078012894BFA348A3480078E2
:105890008DF809000020FBF733FF002818BF4FF0F8
:1058A000FF3004908DF80AA07088ADF80C0000203D
:1058B000FBF7A7FDADF80E009948CDF81880CDE9AB
:1058C00007B037984FF0FF0A68B300210846FBF78E
:1058D000EBFD099001210020FBF7E6FD0A9099F805
:1058E00000008DF82C008DF82D400D978DF82EA01E
:1058F0007088ADF830000020FBF783FDADF8320072
:105900009DF8090000EB400101EB001108EB81015B
:105910000F919DF8081048430BEB4001109180490E
:1059200001EB400011907F4FDFF8FC81389870B395
:1059300000210120FBF7B8FD012112900846FBF77A
:10594000B3FD1390FBF749FA00280CBF98F800004C
:1059500038788DF850000120FBF7B8FD04FA00F00C
:105960008DF851000120FBF780FEC04316908DF8A2
:1059700052A0B088ADF854000120FBF742FDADF80D
:105980005600624818906948199069481A903998E9
:1059900070B300211120FBF787FD1B90012111201E
:1059A000FBF782FD1C90FBF718FA00280CBF387833
:1059B00098F800008DF874001120FBF787FD04FAB9
:1059C00000F08DF875001120FBF74FFEC0431F90CB
:1059D0008DF876A0B088ADF878001120FBF711FDA6
:1059E000ADF87A00534821905348229053482390B1
:1059F000534F3A9840B300210220FBF755FD249005
:105A000001210220FBF750FD259038788DF8980091
:105A10000220FBF75BFD04FA00F08DF899000220EC
:105A2000FBF723FEC04328908DF89AA0B088ADF80C
:105A30009C000220FBF7E5FCADF89E0041482A904F
:105A400041482B9041482C903B9840B300211220B4
:105A5000FBF72AFD2D9001211220FBF725FD2E904A
:105A600078788DF8BC001220FBF730FD04FA00F0C6
:105A70008DF8BD001220FBF7F8FDC04331908DF882
:105A8000BEA0B088ADF8C0001220FBF7BAFCADF89C
:105A9000C2002F4833902F4834902F4835909DF8FE
:105AA00051000227022888BF8DF851709DF87500BB
:105AB000022888BF8DF875704FF055361F9601206B
:105AC0001696FBF7D2FD18B171000120FBF7BDFD62
:105AD0001120FBF7CAFD20B14FF0AA311120FBF7CE
:105AE000B4FD9DF89900022888BF8DF899709DF843
:105AF000BD0033E0E884001000FE0200544352462B
:105B00000080003000A0003018BD0030189D00302B
:105B1000CF840010CE840010CD840010D0840010FB
:105B200000400030D1840010D2840010CC09003035
:105B3000CC490030B09D0030CC0E0030CC4E00304F
:105B4000D4840010489E00304C1800304C5800306F
:105B5000E09E00304C1D00304C5D0030022888BFB4
:105B60008DF8BD70319602202896FBF77EFD20B19E
:105B70004FF0AA310220FBF768FD1220FBF775FDFC
:105B800020B14FF0AA311220FBF75FFDBDF85400A1
:105B900000F58060ADF85400BDF8780000F5806035
:105BA000ADF87800BDF89C0000F58060ADF89C0071
:105BB000BDF8C00000F58060ADF8C000FBF740FD07
:105BC0005E900120FBF732FD0120FBF7B2FD6190F2
:105BD0000020FBF76AFF60900020FBF75BFF5F90FF
:105BE0000020FBF752FB6290FCF72CF90020539049
:105BF00052903D9044904598002840F0988303F0DF
:105C000004FA012800F093835398802800F28F83D0
:105C100046A8FCF719FB002800F0838346A804F08F
:105C2000C7F85298401C529000F0728300205290A6
:105C30005398401C539000203EAA012142F82010A6
:105C4000401C0628F8D33D98002808BF3C9013D08C
:105C5000012804BF00203C9000F0E480022804BF2B
:105C600000203C9000F00782032804BF01204590EB
:105C700000F02D8300F05BBB3C9936A850F8210062
:105C800000287DD001EBC101684600EB81000021B6
:105C9000449A4D9101684E9141684F91077A417A3B
:105CA0004C91D0E90681B0F90C600069C2F1080599
:105CB0005090FAB1002D7DDB4C984FF0000A00287F
:105CC00061D905F10800012202FA00FBE81D02FA81
:105CD00000F056900123509803FA0AF2104018BFC2
:105CE0000120002257900AEB4A0000EB0A1094466C
:105CF00051907EE04C980024002888BF4FF0010EA0
:105D00007FD950980EFA04F2024214BF4FF0010BF3
:105D10004FF0000B002004EB440202EB0412844617
:105D2000519228E043094EAA52F8232000F01F03A5
:105D30000EFA03F31A421BD000F0010208EB4233C3
:105D4000519A4FEA500903EB820A31F9023B5AF8A3
:105D500029209B1B0CF1010CBBF1000F18BF5B420B
:105D6000002BC8BF42F4803242F400424AF8292096
:105D7000401C262801D2BC45D4D3641C4C9800E0BA
:105D800048E08442BDD33CE053094EA802F01F0412
:105D900050F823300120A040034227D002F0010038
:105DA00008EB403351984FEA520903EB800454F852
:105DB000290000E029E031F9023BDDF85CE19B1BA2
:105DC0000CF1010CBEF1000F18BF5B4210F4803FD4
:105DD00002D0002B04DA01E0002B01DD20EA0B00E9
:105DE000002DC4BF569B184344F82900521C262A94
:105DF00001D2BC45C8D34C980AF1010A8245FFF490
:105E000069AF002D04BF01204D903EA93C9A4D98EA
:105E100041F822003C98401C3C900628FFF42CAF2F
:105E200000F055BA3C9936A850F82100002800F03F
:105E30001A813C98449900EBC002684600EB82004E
:105E40000022509202684C9242684D92037A457A41
:105E5000847A4F94D0E906C2B0F90C800469519459
:105E6000C0894F9CC1F1080600EA0407E9B1002E81
:105E700075DB4FF0000A002D70D9012000FA06FBF7
:105E8000701E012101FA00F059900124519804FA82
:105E90000AF1084018BF012000214E900AEB4A0089
:105EA00000EB0A108946589092E04FF0000A002D4E
:105EB00054D90124519804FA0AF1084018BF01206E
:105EC00000214E900AEB4A0000EB0A1089465790D9
:105ED0003EE04C094CA801F01F0B50F82440012073
:105EE00000FA0BF0044230D001F001000CEB40341A
:105EF00057984FEA510B04EB8000569032F9024B51
:105F0000DDF838E150F82B00A4EB080409F1010991
:105F1000BEF1000F18BF644210F4803F09D0002C7E
:105F20000EDA10F47F4018BFA0F5807040F4803086
:105F300006E0002C04DD10F47F4018BFA0F580704F
:105F400040F08000569C44F82B00491C262901D2C1
:105F50009945BED30AF1010AAA45AAD33FE042E01F
:105F60004C094CA801F01F0E50F82440012000FA03
:105F70000EF0044229D001F001000CEB4034589897
:105F8000DDF838E104EB80004C08CDE9564050F8CC
:105F9000240032F9024B09F10109A4EB0804BEF117
:105FA000000F18BF644210F4803F02D0002C04DAC6
:105FB00001E0002C01DD20EA0B00002EC4BF599C3B
:105FC0002043DDE9564E4EF82400491C262901D213
:105FD0009945C5D30AF1010AAA45FFF456AF002E30
:105FE000C8BF50983BDC0026002D36D94F98C0F52D
:105FF000807A40F4807E002006EB4601024601EBE9
:10600000061B25E044094CA900F01F0851F8244064
:10601000012101FA08F10C4217D000F001010CEB4C
:10602000413101EB8B094FEA5008521C59F82840C6
:10603000E1B201EB5A0101EA0E01B94288BF3946CB
:1060400024F0FF04214349F82810401C262801D2DF
:106050009A42D7D3761CAE42CDD3012050903C9AC1
:106060003EA941F822003C98401C3C900628FFF4D1
:10607000D9AE00F02CB93C9936A850F82100002880
:1060800000F01F8144984F9001EBC101684600EB7E
:10609000810000214E91016850914168519190F822
:1060A00008A0417A4C91817AB0F90C90826957929C
:1060B000D0E90784C289006956904F98C1F580766F
:1060C00002EA010710F0010F14D04C984FF0000BBA
:1060D000002870D90122569802FA0BF1084018BF27
:1060E000012000214D900BEB4B0000EB0B108C4678
:1060F0006390D4E00020FBF71CFB05464C9800FBA6
:106100000AF1032000EB410020F003024146204643
:1061100016F0DDF82846FBF70CFB4C984FF0000B0F
:10612000002848D90122569802FA0BF1084018BFFE
:10613000012000214D900BEB4B0000EB0B100D46A6
:1061400059904BE04A0950A801F01F0350F8222053
:106150000120984002423ED038F9020B6D1CA0EBA2
:1061600009034D98002818BF5B4201F001025798BF
:106170004FEA510E00EB4232599802EB80005890E2
:1061800050F82E20C2F3072002F0FF0C12F4803FDB
:1061900002D0002B02DB04E0002B02DDACEB060496
:1061A00001E00CEB0604BC4206DDFF283ABF0024E8
:1061B000401C3C4607E07AE0002C04DA0028C6BF09
:1061C0003C46401E002402F4803242EA0020589AE5
:1061D000204342F82E00491C262901D25545B1D34F
:1061E0004C980BF1010B83459CD360E04A0950A801
:1061F00001F01F0350F822200120984002424BD0AA
:1062000034F9020B4D9AA0EB09000CF1010C002AA5
:1062100018BF404238F9022BA2EB090218BF5242C4
:106220000028B4BF43420346002AB8BF52429A42F4
:1062300032D9579A01F0010302EB4333639A03EB1F
:1062400082024B08CDE9583252F82330C3F30722BB
:10625000DDB213F4803F02D0002802DB03E0002807
:1062600001DD354400E0AD1BBD4205DDFF2A3ABF2C
:106270000025521C3D4606E0002D04DA002AC6BF68
:106280003D46521E002503F4803040EA0220DDE93D
:106290005823284343F82200491C262901D2D4451B
:1062A000A4D34C980BF1010B8345FFF413AF4F9827
:1062B000032826BF01204E904E983EA93C9A41F8F3
:1062C00022003C98401C3C900628FFF4D4AE0123E9
:1062D00000203EA951F82020EAB1401C0628F9D33D
:1062E000CBB13D981F2811D2401C012101FA00F2C8
:1062F0003D906598024209D13D98401C3D9003288D
:1063000004D801FA00F265980242F5D000204490CA
:10631000459818B10BE04498401CF8E7FBF792FD54
:106320006DE4FEF7C3FF459800283FF468ACFBF727
:1063300075FB5D98FBF7CFFD5E98FBF777F96198E9
:10634000FBF7F7F96098FBF7B0FB5F98FBF7A2FB50
:106350006298FAF79AFF5C9830B15B9810B1FBF73E
:1063600071FD01E0FBF735FDFDF73FFA48B15598A7
:10637000002818BFFDF73EFA5498002818BFFDF713
:1063800075FA5A98002818BFFCF7EDFF45980028C9
:106390000CBF0120002067B0BDE8F08F2DE9F05F51
:1063A000ADF5A85D0646002001AF054607F580580B
:1063B00007F5935900909EE0284604F0E1FB002881
:1063C0007ED0008900EA060424F0CC0030F47C4042
:1063D00076D00F212846FFF713F8002870D0FBF77E
:1063E000E4FC009900296CD1FBF7C1FBFF210F20D1
:1063F000FFF7B1F90090FBF711FB0098002877D167
:1064000014F0010F0DD0FEF7E2FF82464FF0040BAF
:106410003846FBF77AFF9AF92C103A46584604F0B2
:10642000FDFB14F0100F0ED0FEF7D1FF82464FF0A7
:10643000080B41460120FBF7BCFF9AF93010424699
:10644000584604F0EBFB14F4807F0ED0FEF7BFFF3C
:1064500082464FF00C0B49460220FBF7AAFF9AF93F
:1064600034104A46584604F0D9FB009848BB24F043
:10647000990030F4794006D0FEF7C9F90090FBF797
:10648000CDFA0098E8B914F0020F0DD0FDF7DDFC4D
:106490008246FEF79CFF05235FEA0A0204D090F9CA
:1064A0002D10184604F0BAFB14F0200F10D0FDF7A1
:1064B00047FC8246FEF78BFF09235FEA0A0201E0F0
:1064C00018E015E004D090F93110184604F0A6FB4E
:1064D00014F4007F0CD0FDF7FCFB0446FEF777FFB9
:1064E0000D23220004D090F93510184604F096FBD5
:1064F000FFF7F5F86D1C04F03FFBA842009803D9A4
:1065000000283FF459AF06E0002802BF01200DF536
:10651000A85DBDE8F09F00200DF5A85DBDE8F09FE7
:106520002DE9F04F9C48ADF50D7D0478FEF766FE31
:10653000012840F0CB8099480068B0F93610B0F9D6
:10654000340015F014FF14F0020F7DD00DF5007B20
:10655000FFF7D8F83026924F4FF488784FF0500963
:106560004FF0FF3A002578B1B0E80E108BE80E101E
:10657000B0E80E100DF5047B8BE80E100FC80DF57A
:10658000087B8BE80F0013E0FF223021584615F0FE
:10659000C1FECDE98495CDE98265CDF82CA2CDF878
:1065A00028A2CDF824A28695CDE9875ACDE9807836
:1065B000DFF8F0B15846FCF795FA8598401C8590B5
:1065C00040F27770FFF7EAFE012803D1FEF731FAB7
:1065D00001281FD087980023401C87901A4621214C
:1065E000CDF81092072006F0C9FE00231A4619467E
:1065F000FE200095FEF788FA0DF5007904F0A0FA68
:1066000090B181698891C169899141698A91C06815
:106610008B9011E014F0080F14BFA220A1208490E9
:106620008698401C8690E7E7CDF82CA2CDF828A2EA
:10663000CDF824A2CDF820A2CDE98265CDE98078FD
:1066400000214A46084600E029E0D9F8083052F80F
:1066500020C0401C6144B0EB930FF8D34D42FF22A1
:106660004FF400716846C9F80C5015F053FED9F884
:106670000820F9E804018DE82700B9E80F0004AD0F
:1066800085E80F0099E80F0008AD85E80F0058462F
:10669000FCF728FA69465846FCF7C6FA0DE014F0F4
:1066A000100F0AD04FF4E060FFF778FE28B90023FE
:1066B00001222121072006F061FE0020FDF799FF4D
:1066C000002322464021072006F058FE0DF50D7DDF
:1066D000BDE8F04F02F052BC2F49488070472E4968
:1066E0008880704770B50126FFF70CF820B100696B
:1066F000A12818BFA22801D0002070BD002404F0FA
:106700003BFA002842D9204604F03AFA00281EBF7E
:10671000058925F0CC0030F47C4032D00F21204692
:10672000FEF76EFE68B315F0010F0AD0FBF701FE0D
:1067300038B944F4807200232021072006F01EFEA1
:10674000002615F0100F0BD00120FBF74EFE38B9D4
:1067500044F4805200232021072006F00FFE00267B
:1067600015F4807F0BD00220FBF73FFE38B944F4CC
:10677000803200232021072006F000FE0026FEF7CD
:10678000AEFF641C04F0F8F9A042BCD8304670BDDE
:106790000020704700207047E8840010D485001066
:1067A0005443524600FE020070470020704710B567
:1067B00003F00700042808BFFEF7DCFD002010BD31
:1067C00070B503F007020025F84CF94B012A02D0FE
:1067D000022A14D011E0052018709D60FCF780FF9C
:1067E0002268532111702268452151702268010AE4
:1067F00091702168C87020680571002070BD1A78FA
:10680000052A13D19A68052A28BF104607D2D4F862
:1068100000C01CF802C080F800C0501C9860052819
:1068200004D101209D60087003201870012070BD04
:106830002DE9F04103F0070201260025DB4CDC4B7B
:10684000012A02D0022A3BD037E0052018709D6053
:10685000FCF746FF2168AC270F702268010A5170CF
:106860002168887004F022F9DFF8488380B1D8F8F5
:10687000000004F017FA58B1D8F8000090F8200092
:1068800010F0020F04D02068477021684320887000
:106890002068C6702068057104F008F950B1D8F876
:1068A000000004F0FFF928B1D8F800002168007E4C
:1068B000487102E02168FF2048710020BDE8F081A6
:1068C0001A78052A12D19A68062A28BF104607D2DC
:1068D000D4F800C01CF802C080F800C0501C9860BA
:1068E000062803D19D600E70032018700120BDE8BA
:1068F000F08103F00702022A1CBF0020704720220B
:1069000002700120087070472DE9F041A84F0D4634
:10691000064613F0070F04D003F00700022808D042
:1069200004E012F0040F1CBF0020B8700020BDE886
:10693000F08102F01DFB002814BF0124002402F0A6
:106940001AFB002814BF0222002242EA0403B8788E
:10695000002814BF0422002242EA03003070012004
:106960002870BDE8F08170B503F0070C0026904C4C
:106970008E4DBCF1010F0AD0204613F0070F0078AE
:106980000DD0BCF1040F08BF062818D029E0A6607E
:1069900028680670286846700520207021E00528C8
:1069A0001FD1A068022803D22B681A54401CA06093
:1069B000022816D10120A6600870062010E0286881
:1069C000007855280BD128684078AC2818BFBC281F
:1069D00005D128680122411C062002F0AFFA0320ED
:1069E0002070002070BD70B503F0070200256F4CC9
:1069F0006F4B012A02D0022A24D021E00520187012
:106A00009D6002F070FA41F6E8710144B0F53C3F38
:106A100010D8CA78086862F31F60674A904208BFBE
:106A2000002007D10A18236812791A54401C142830
:106A3000F8D305E0002021680D54401C1428FAD337
:106A4000002070BD1A78052A13D19A68142A28BF2D
:106A5000104607D2D4F800C01CF802C080F800C06D
:106A6000501C9860142804D101209D6008700320F8
:106A70001870012070BD70B503F0070200254B4C63
:106A80004B4B012A02D0022A3FD03CE0052018706F
:106A90009D6002F028FA41F6E8710144B0F53C3FF0
:106AA0002BD8CA78086862F31F60434A904224D109
:106AB0002268087C10702268487C50702268887CAC
:106AC00090702068CA7CC27020680A7A02712268BD
:106AD000487A50712268887A90712268C87AD07199
:106AE0002268087D10722268487D50722268887D75
:106AF0009072C87D2168C87205E0002021680D549D
:106B0000401C0C28FAD3002070BD1A78052A13D136
:106B10009A680C2A28BF104607D2D4F800C01CF887
:106B200002C080F800C0501C98600C2804D10120DD
:106B30009D60087003201870012070BD70B503F0CF
:106B400007020025194C1A4E012A02D0022A3FD012
:106B50003CE003F0F5FF40B3D0E906212368C068AC
:106B60001A70D4F800C0130A8CF80130D4F800C0B1
:106B7000130C120E8CF802302368DA70226811713F
:106B800023680A0A5A7123680A0C090E9A7122684E
:106B9000D171216808722268010A51722268010CC1
:106BA0009172010E2068C1720DE007E098E90100C2
:106BB000F8840010D485001034CD12AB21680D5438
:106BC000401C0C28FAD305203070B560002070BD41
:106BD0003278052A10D1B2680C2A28BF104604D298
:106BE00023689B5C0370501CB0600C2804D101200A
:106BF000B560087003203070012070BD70B503F0DF
:106C000007020024F84DF94B012A02D0022A3ED097
:106C10003BE00520187000269C6002F064F900F546
:106C20000051B0F53C3F98BF11F0030F27D1F04A57
:106C30000868904204BF0022104620D151F820304D
:106C4000401C1A440728F9D302B1C6B128680A7C4F
:106C500002702A68487C50702A68887C90702A6884
:106C6000C87CD0702A68087D10712A68487D5071F0
:106C70002A68887D9071C87D2968C87105E0002068
:106C800029680C54401C0828FAD3002070BD1A78DB
:106C9000052A13D19A68082A28BF104607D2D5F8CA
:106CA00000C01CF802C080F800C0501C9860082882
:106CB00004D101209C60087003201870012070BD71
:106CC0002DE9F04103F0070C0027C84E4FF00508EE
:106CD000BCF1010F0DD013F0070F0FD03246BCF1FD
:106CE000020F127810D0BCF1040F08BF062A26D07C
:106CF00058E086F800807770B76053E07270BD4846
:106D0000B062062030704DE0052A15D1B268042A21
:106D100028BF104609D2C2F10303D6F828C0DB0011
:106D20002CFA03F30370501CB060042804D1012036
:106D3000B7600870032030700120BDE8F0817078E2
:106D40000125002410F0010F11D002F0CCF8B0F5AD
:106D50003C3F23D86A030021B1EB900F07D252F8D1
:106D6000043B491C1C44B1EB900FF8D3B5B17078CB
:106D700010F0020F0ED003F0E3FE78B1826800211C
:106D8000B1EB920F06D250F8043B491C1C44B1EB06
:106D9000920FF8D3002D18BFB46200D1B76277709C
:106DA00086F800800020BDE8F081F0B503F0070C04
:106DB00000268D4D8D4C83B0BCF1010F0ED013F029
:106DC000070F1DD0224603271278BCF1020F26D0F0
:106DD000BCF1040F08BF062A36D03CE002AA01A984
:106DE000684602F0E3FB05202070296801980870CE
:106DF000296800984870296802988870A6602AE07F
:106E0000A068032803D229680A54401CA060022805
:106E100021D306212170032808BFA6601BE0052AA4
:106E20000FD1A268032A28BF104604D22B689B5CAE
:106E30000370501CA060032803D10120A6600870D5
:106E4000277003B00120F0BD28688278017840786F
:106E500002F09FFB277003B00020F0BD08B503F0DF
:106E6000070001280AD103F021FE38B101208DF876
:106E70000000024669460D2002F060F8002008BDBF
:106E800008B503F0070001280AD103F00FFE38B15E
:106E900000208DF80000012269460D2002F04EF816
:106EA000002008BD08B503F00700012809D103F050
:106EB000FDFD30B103208DF800000122694602F08B
:106EC0003DF8002008BD0020704708B503F007001A
:106ED00001280AD103F0EAFD38B10B208DF800003B
:106EE00001226946032002F029F8002008BD1FB5E1
:106EF00013F0070F0ED103F0D9FD58B19DF808002B
:106F0000F0280AD003F0D2FD20B1012202A9092005
:106F100002F014F804B0002010BDFEF715FCF9E7EC
:106F200008B503F0070001280AD103F0BFFD38B10E
:106F300010208DF8000001226946032001F0FEFFB9
:106F4000002008BD70B503F00700274C274D01282D
:106F500008D013F0070F12D0042804BF28780628A1
:106F600016D01FE00020A8602168087021684870D2
:106F7000216888702168C8700520287012E0A86810
:106F800004280FD221680A54401CA860062008E09B
:106F900003F08CFD30B104221046216801F0CEFFD1
:106FA00003202870002070BD10B503F007000128F1
:106FB00004D102F0D1FF0D4900200871002010BD5E
:106FC00010B503F0070C094CBCF1010F06D013F00B
:106FD000070F11D0BCF1020F20D01DE00020A060EF
:106FE00006F0C3F9A06117E098E90100F8840010E9
:106FF00054464953EFBEADDEA068002804BF10021E
:10700000A06106D0012804D1A0691043A06106F058
:10701000ABF9A068401CA060002010BDA26812B1AE
:10702000012A04D007E0218B090A017003E0237EC6
:10703000037001200870501CA060012010BD10B525
:1070400003F0070CFE4CBCF1010F06D013F0070F44
:1070500009D0BCF1020F18D015E00020A06006F0A6
:1070600087F9A0610FE0A068002804BF1002A061AA
:1070700006D0012804D1A0691043A06106F07BF975
:10708000A068401CA060002010BDA26812B1012AB7
:1070900004D007E0218B090A017003E0237E03700E
:1070A00001200870501CA060012010BD70B506467C
:1070B00003F00700E24C0D46012808BF00200DD068
:1070C00013F0070F02D002280BD008E0A0680028B8
:1070D00004BF104611F047FEA068401CA0600020CD
:1070E00070BD11F03DFE30700120287070BD70B58C
:1070F00003F0070CD24D0E460446BCF1010F06D03A
:1071000013F0070F07D0BCF1020F18D015E00020D4
:10711000A860E86011E0A868002804BF1002A86118
:1071200008D0012806D1A869104381B2A861E88877
:107130000CF035FDA868401CA860002070BDE86810
:1071400002280ED2E8880CF02EFDEB6882B2002BEC
:1071500004BF100A207004D0012B02D1227001203C
:107160003070E868401CE860012070BD10B403F086
:10717000070CB34CBCF1010F08BF00200BD013F07B
:10718000070F03D0BCF1020F09D005E0A06800286A
:1071900008BFE280401CA06010BC00207047A268BD
:1071A0001AB9A379037001200870501CA06010BCAC
:1071B000012070472DE9F047064603F00700A04F75
:1071C0008946012808BF002039D0DFF878829E4D1B
:1071D00013F0070F02D0022835D031E0B86800283C
:1071E00008BF7A7029D0012804BF1002B86124D0EA
:1071F000022822D1B8691043B8617E7884B203F0C6
:1072000055FCD0B1062E18D2DFE806F00306090CB3
:107210001014A8F80E4010E0A8F80C400DE0286803
:1072200084860AE02868A0F80C4106E02868A0F8E7
:10723000504002E02868A0F85240B868401CB8608E
:107240000020BDE8F087F86802282CD297F801A04A
:10725000002403F02BFCD8B1BAF1060F18D2DFE8F6
:107260000AF00306090C1014B8F80E4010E0B8F844
:107270000C400DE02868848E0AE02868B0F80C41C4
:1072800006E02868B0F8504002E02868B0F85240A4
:10729000F868002804BF200A307004D0012802D109
:1072A000347089F80000F868401CF8600120BDE8DF
:1072B000F0872DE9F0411C4615460E46074603F0BF
:1072C000F5FB80B15F4814F0070F04D004F007010C
:1072D00002290BD007E0002D1ABF90F86C00C008FF
:1072E000002009F0DAFC0020BDE8F08190F86C0085
:1072F000C008387001203070BDE8F0812DE9F04100
:107300001C4615460F46064613F0070F08D103F03A
:10731000CDFB28B1022D3CBF284607F09EFB03E0C1
:1073200004F00700022802D00020BDE8F08107F039
:107330008DFB307001203870BDE8F08170B503F02E
:1073400007020026414C3E4D012A02D0022A15D0E8
:1073500012E006F027FC21680870FDF74FFF216856
:10736000487003F01BF921688870FDF74DFF216814
:10737000C87005202870AE60002070BD2A78052AEC
:1073800010D1AA68042A28BF104604D223689B5C47
:107390000370501CA860042804D10120AE6008705E
:1073A00003202870012070BD70B503F00702274C40
:1073B0000025234E012A02D0022A4BD03FE0FEF7DF
:1073C000A1F9002828D04169FF292CBFFF21C9B2AB
:1073D000226811708169FF2934BFC9B2FF21226878
:1073E0005170C169FF2934BFC9B2FF212268917071
:1073F0002268017CD170226890F820101171018CF4
:107400002268090A5171016A2268090C9171006AA7
:107410002168000EC87111E0206805702068457071
:107420002068857021685020C8702168FF2008718D
:1074300021684871216888712168C871B56007E0CA
:10744000F8840010E8FC0010D485001098E90100D1
:10745000002070BDB268082A28BF104604D22368F5
:107460009B5C0370501CB060082802D10120B560FD
:107470000870012070BD03F00702FC4B4FF0000CB8
:10748000012A08BFC3F808C001D0022A01D0002099
:1074900070479A68022A3DBF80F800C0501C98606F
:1074A0001046022803D10120C3F808C0087001204B
:1074B00070472DE9F047064603F00700EB4F894679
:1074C0004FF00008012808BFC7F8088001D0022843
:1074D00002D00020BDE8F087B86880BB00242546B4
:1074E00001F001FD00F50051A1F1180340214FF416
:1074F0000052B0F53C3F1ED893F803A0D3F800C06B
:107500006AF31F6CDFF868A3D44514D1001FB4EBF5
:10751000900F07D252F804CB641C8CEA0505B4EB3B
:10752000900FF7D3DA7D586962F31F60A84204BF59
:107530008020307000D03170B868401CB8600128DD
:1075400003D1C7F8088089F800000120BDE8F08762
:107550002DE9F04103F007020026C64CC34D012A75
:1075600002D0022A56D052E0FCF7BAF80520287063
:1075700003F09CFA002849D0BF4F386803F092FB13
:10758000002843D00CF0F5FA80460CF0F6FA396882
:107590000A7E12F0040F11D0C98A2268090A1170FC
:1075A00039682268897D517039682268898A090A98
:1075B000917039682268097DD17010E0898A22684B
:1075C000090A117039682268097D5170396822688A
:1075D000C98A090A917039682268897DD170226848
:1075E0004FEA18211171216881F805802268010A8B
:1075F00091712168C87138682268817C1172226893
:10760000017C5172008B2168000A8872AE600020F4
:10761000BDE8F0812A78052A10D1AA680B2A28BF74
:10762000104604D223689B5C0370501CA8600B2892
:1076300004D10120AE600870032028700120BDE84D
:10764000F0812DE9F04703F007020026894D874BB2
:10765000012A02D0022A5DD059E0052018700024CA
:107660009E6001F040FC00F50053B0F53C3F98BF30
:1076700013F0030F45D1814A1968914204BF0022DB
:10768000114608D153F821C0491C62440729F9D397
:10769000002A08BF01249F7C93F8138084B341F62D
:1076A000E8710144B0F53C3F07D8CA78086862F336
:1076B0001F606F4A904208BF012491F8129091F820
:1076C00013A0002C08BF002014D003F039FA296859
:1076D000806981F80090296881F801A02A68010C6E
:1076E000000E91702968C87028680771286880F8B2
:1076F00005800CE029680E54401C0628FAD306E0E9
:10770000FFE7002029680E54401C0628FAD3002009
:10771000BDE8F0871A78052A13D19A68072A28BF8E
:10772000104607D2D5F800C01CF802C080F800C08F
:10773000501C9860072804D101209E600870032027
:1077400018700120BDE8F08710B503F0070C474C16
:10775000BCF1010F06D013F0070F0AD0BCF1020FE5
:107760001AD017E00020A060E0600CF076FAA0616B
:1077700010E0A068002804BF1002A06107D0012813
:1077800005D1A0691043A06180B20CF063FAA06833
:10779000401CA060002010BDE268022A0BD212B18A
:1077A000012A04D007E0218B090A017003E0237E3F
:1077B000037001200870501CE060012010BD70B5FE
:1077C00003F007010026294D0446012908BFEE6297
:1077D00001D0022901D0002070BDE86A002804BF52
:1077E000274814F0C9FDE96A082928BF267002D28B
:1077F0002348405C2070481CE862012070BD2DE9E0
:10780000F04103F007010026184D0746012908BF83
:10781000EE6201D0022902D00020BDE8F08195F887
:107820002C0000F007042879204304D1144814F0F8
:10783000A3FD01202871052C28BF2E711048005D82
:107840003870E86A401CE8620120BDE8F08170B53C
:10785000044603F007000D4602281CBF002070BD3F
:1078600014F08FFD20700120287070BDF884001086
:1078700034CD12AB98E90100D48500105446495329
:107880002885001070B503F007020025F94C012A85
:1078900002D0022A12D00FE00520207000221146EB
:1078A0001046A56001F082FE4FF6FF7101EA40002C
:1078B000206101F08EFE6062002070BD2278052AF2
:1078C00017D1D4F810C0A268624528BF104607D26D
:1078D00012F0010F1CBF637803700CD0501CA06025
:1078E000604506D10120A56008700320207001F0DA
:1078F0007DFE012070BD666A22F00103F35A1E0A64
:1079000006706370EAE770B503F007020025D94CF2
:10791000012A02D0022A11D00EE0D74805220068C1
:10792000B0F91210B0F91000227008444000A560B0
:10793000206101F0CEFF6062002070BD2278052A30
:1079400017D1D4F810C0A268624528BF104607D2EC
:1079500012F0010F1CBF637803700CD0501CA060A4
:10796000604506D10120A56008700320207001F059
:10797000BEFF012070BD666A22F00103F35A1E0AA1
:1079800006706370EAE7F8B503F007020025B94C0A
:10799000012A02D0022A13D010E000216A460846CC
:1079A00001F004FE05202070A56000984FF6FF71DD
:1079B00001EA4000206102F0BEF860620020F8BDDC
:1079C0002278052A17D1D4F810C0A268624528BFD2
:1079D000104607D212F0010F1CBF637803700CD061
:1079E000501CA060604506D10120A56008700320EE
:1079F000207002F0AEF80120F8BD666A22F00103A3
:107A0000F35A1E0A06706370EAE77FB51C460E46FD
:107A1000054613F0070F08D103F048F828B10122FA
:107A200002A90C2001F08AFA03E004F00700022802
:107A300002D004B0002070BD06F0B4F82870012018
:107A4000307004B070BD7FB51C460E46054613F07D
:107A5000070F08D103F02AF828B1012202A90F204C
:107A600001F06CFA03E004F00700022802D004B031
:107A7000002070BD10F076FF00F00F0040F0100005
:107A800028700120307004B070BD10B503F00702FB
:107A9000784C012A02D0022A0DD00AE003F09DFAA8
:107AA0000021E06100281ABF4FF4056020622162C6
:107AB000A160002010BD236AA2689A4228BF104628
:107AC00007D2D4F81CC01CF802C080F800C0501CBB
:107AD000A060984204BF01200870012010BD10B4BE
:107AE00013F0070F4FF0402C04D003F00702022AD6
:107AF00013D00FE0012A04BFDCF8140040F00100AD
:107B000006D0002A04BFDCF8140020F0010001D1E7
:107B1000CCF8140010BC00207047DCF8142002F0F0
:107B2000010202700120087010BC704770B5144645
:107B30000E46054613F0070F04D003F00700022895
:107B400013D010E0002C14BF0120002002F0F6F941
:107B50004CB14FF04020016B21F4405141F4BE0183
:107B600041F020410163002070BD02F0EEF90028D1
:107B700014BF012200222A700120307070BD70B540
:107B800003F007003B4D1446012808BF002015D024
:107B900013F0070F13D1A868002808BF6A700BD034
:107BA000012809D16878FBF709F96878334900EAB8
:107BB00004020A63A0434863A868401CA860002030
:107BC00070BD70B5044603F007000D4602281CBFC7
:107BD000002070BD05F046FF20700120287070BDA8
:107BE00070B50D46044613F0070F04D003F00700EC
:107BF000022805D002E0104605F03CFF002070BDD1
:107C000005F03BFF20700120287070BD70B50D4657
:107C1000044613F0070F04D003F00700022805D034
:107C200002E01046F9F7C2F8002070BDF9F7C1F87C
:107C300020700120287070BD10B403F007020024EA
:107C4000DFF830C0012A08BFCCF808400FD0022A64
:107C500003D013F0070F05D009E00470012008706D
:107C600010BC7047DCF80800401CCCF8080010BCC1
:107C700000207047F8840010D485001000100040E8
:107C800070B5044603F00700FE4D0E46012804BF00
:107C90000020A86014D013F0070F02D0022811D0E2
:107CA0000EE0A868F84904283CBF0B681A54401C31
:107CB000A860042804D104220968112001F03EF9CB
:107CC000002070BD0AF0E8F9AA68002A04BF000E7F
:107CD00020700FD0012A08BF000C06D0022A08BF6E
:107CE000000A02D0032A02D004E0207002E02070D3
:107CF00001203070501CA860012070BD70B503F0E9
:107D0000070CE04D0E460446BCF1010F04BF0020F5
:107D1000A86015D013F0070F03D0BCF1020F11D0EB
:107D20000EE0A868D84902283CBF0B681A54401CD2
:107D3000A860022804D102220968122001F0FEF88E
:107D4000002070BD0AF080F9AA68002A04BF000A6A
:107D5000207004D0012A02D1207001203070501C04
:107D6000A860012070BD70B5044603F00700C54D42
:107D70000E46012804BF0020A86014D013F0070F9E
:107D800002D0022811D00EE0A868BF4904283CBFE9
:107D90000B681A54401CA860042804D10422096806
:107DA000132001F0CBF8002070BD0AF0A8F9AA68F2
:107DB000002A04BF000E20700FD0012A08BF000C5B
:107DC00006D0022A08BF000A02D0032A02D004E02B
:107DD000207002E0207001203070501CA86001204B
:107DE00070BD70B5044603F00700A64D0E4601288D
:107DF00004BF0020A86037D013F0070F02D002287C
:107E000034D031E0A868A04C002804BF21680A7073
:107E100021680978012901D039B11BE0002818BF79
:107E200004283CBF21680A5414E00AF086F921684E
:107E3000000948700AF072F9C0F303260AF07DF9D0
:107E4000216846EA001088700AF068F92168C87055
:107E50000320A860A868401CA860042804D104225C
:107E60001420216801F06AF8002070BD0AF071F951
:107E7000AA68002A04BF000E20700FD0012A08BF94
:107E8000000C06D0022A08BF000A02D0032A02D042
:107E900004E0207002E0207001203070501CA860C7
:107EA000012070BD10B503F00702764C012A02D004
:107EB000022A27D024E003F090F80023002804BF12
:107EC000E36123621BD000F15001E1614168B1F52B
:107ED000887F90F820100CD390F8212001EB020C41
:107EE00001FB02C190F8222090F8230010440844BE
:107EF00004E090F822000A1801FB00202062A36031
:107F0000002010BD236AA2689A4228BF104607D2FB
:107F1000D4F81CC01CF802C080F800C0501CA0603F
:107F2000984204BF01200870012010BD03F0070231
:107F3000012A02D0022A05D002E0524900208860BE
:107F400000207047012202700A701046704710B579
:107F500013F0070F04D003F00702022A05D002E055
:107F6000104601F050FB002010BD484A1278027004
:107F70000120087010BD10B513F0070F04D003F0F6
:107F80000702022A05D002E0104601F0D5FC0020CD
:107F900010BD3F4A127802700120087010BD10B564
:107FA00013F0070F04D003F00702022A05D002E005
:107FB000104601F0DBFD002010BD364A1278027039
:107FC0000120087010BD1FB513F0070F07D102F094
:107FD0006DFD20B1012202A90B2000F0AFFF04B01B
:107FE000002010BD70B503F00700264C154601288F
:107FF00004BF0020A06024D013F0070F21D102F0AD
:1080000055FDF0B1A068204E03283CBF31680D54E7
:10801000401CA060032814D1F9F7C1FD3068B0F806
:10802000010045BAF9F7F8FC040018BFF9F743FF5F
:10803000306829460078F9F747F9002C18BFF9F79E
:108040003DFF002070BD70B503F007000D4C1646D3
:10805000012804BF0020A06034D013F0070F31D1F5
:1080600002F024FD70B3A068074D02283CBF2968C8
:108070000E54401CA060022824D1F9F790FDF9F7B6
:10808000CBFC09E0F884001098E901003D85001060
:108090004285001047850010040018BFF9F70BFF58
:1080A0002868007880B129684978F9F78CF9286840
:1080B0004178007840F01000F9F785F9002C18BFDE
:1080C000F9F7FCFE002070BD286841780020F3E736
:1080D0007FB51C460E46054613F0070F08D102F087
:1080E000E5FC28B1012202A9182000F027FF03E0D7
:1080F00004F00700022802D004B0002070BD05F093
:1081000029FD002814BF012200222A7001203070AE
:1081100004B070BD7FB51C460E46054613F0070F30
:1081200008D102F0C3FC28B1012202A9192000F0F5
:1081300005FF03E004F00700022802D004B000208D
:1081400070BD05F0F4FC28700120307004B070BDE3
:1081500070B503F00700FB4C1546012804BF002052
:10816000A06019D013F0070F16D102F09FFC98B150
:10817000A068F54903283CBF0A681554401CA0605C
:10818000032809D108680968B0F80100097840BAE5
:1081900000B219B1FEF7A3FA002070BDFEF79CFAF9
:1081A000FAE770B503F00700E64C1546012804BF56
:1081B0000020A06017D013F0070F14D102F076FC56
:1081C00088B1A068E04B03283CBF19680D54401CDF
:1081D000A060032807D11868B0F8010041BA1868F8
:1081E0000078FAF762F9002070BD10B503F00702BD
:1081F000D44C012A02D0022A07D004E00020A0605B
:10820000FBF75FF9A061002010BDA268042A07D225
:10821000C2F10303D4F818C0DB002CFA03F3037097
:10822000501CA060042804BF01200870012010BD6C
:1082300010B503F00700012807D102F037FC20B188
:10824000002211461D2000F079FE002010BD2DE90E
:10825000F04103F00705BB4E174688460446012D42
:1082600004BF0020B0601BD013F0070F16D102F03E
:108270001DFC98B1B068B44B03283CBF19680F547B
:10828000401CB06003280BD1186890F9022090F9C7
:10829000011090F90000FCF76AFC01E0022D02D009
:1082A0000020BDE8F081B06820B1012807D0022885
:1082B0000AD010E01420FCF701FC20700BE0152020
:1082C000FCF7FCFB207006E01620FCF7F7FB2070A3
:1082D000012088F80000B068401CB0600120BDE8B3
:1082E000F08170B50D46044613F0070F04D003F07B
:1082F0000700022805D002E0924900208860002093
:1083000070BD0020FCF7DAFB20700120287070BDE2
:1083100070B503F0070C00268B4C8A4DBCF1010FA1
:1083200006D013F0070F0CD0BCF1020F1FD01CE0D9
:1083300005F04CFDAE60216808702168000A4870A5
:1083400013E0A868022803D221680A54401CA860E0
:1083500002280AD1AE602068007810F0010F04D026
:1083600002221A20216800F0E9FD002070BDAA68F1
:10837000022A28BF104604D223689B5C0370501C5D
:10838000A860022804D10120AE6008700320287084
:10839000012070BD7FB51C460E46054613F0070F41
:1083A00008D102F083FB28B1012202A9222000F0AB
:1083B000C5FD03E004F00700022802D004B000204D
:1083C00070BD0BF039FC28700120307004B070BD16
:1083D0007FB51C460E46054613F0070F08D102F084
:1083E00065FB28B1012202A91F2000F0A7FD03E0D0
:1083F00004F00700022802D004B0002070BD0BF08A
:1084000026FC28700120307004B070BD7FB51C467A
:108410000E46054613F0070F08D102F047FB28B1BE
:10842000012202A9212000F089FD03E004F00700E9
:10843000022802D004B0002070BD444800782870A3
:108440000120307004B070BD7FB51C460E46054655
:1084500013F0070F0ED102F029FB58B19DF8080068
:10846000002818BF0BF0FCFB012202A91E2000F01F
:1084700065FD03E004F00700022802D004B00020EC
:1084800070BD0BF0F0FB28700120307004B070BD9F
:10849000002070472DE9FF412A4E1C460F46054635
:1084A00013F0070F1CD102F001FBC8B19DF80800C2
:1084B000002818BF012802D0022807D014E0F0706D
:1084C000012202A9082000F039FD0DE0F07004201F
:1084D0008DF80800012202A9082000F02FFD03E01A
:1084E00004F00700022803D004B00020BDE8F081AA
:1084F000F07828700120387004B0BDE8F0817FB5B5
:108500001C460D46064613F0070F08D102F0CEFABE
:1085100028B1012202A9082000F010FD03E004F0B8
:108520000700022802D004B0002070BDFCF766FEF0
:10853000801E052814D2DFE800F0030D0F0B110098
:1085400000200EE0F884001098E90100308500104A
:10855000012006E0022004E0032002E0042000E005
:10856000FF2030700120287004B070BD2DE9F0416B
:108570001C4617460E46054613F0070F0BD102F0B6
:1085800095FA40B1384605F067FA002211460120FD
:1085900000F0D4FC03E004F00700022802D0002021
:1085A000BDE8F08105F05BFA287001203070BDE86D
:1085B000F08110B5104613F0070F08BF05F0E0FA80
:1085C000002010BD10B5104613F0070F08BF05F0CE
:1085D000DEFA002010BD70B5044603F007000D461A
:1085E00002281CBF002070BD05F0D9FA20700120C0
:1085F000287070BD03F0070230B4FF4B4FF0000C41
:10860000012A05D0022A04BF1A78022A0BD01EE0E4
:1086100002201870F948C3F808C06FF07F41006865
:10862000081A986113E09A68042A28BF104606D2F7
:108630009D69D40025FA04F40470501C9860042845
:1086400005D10120C3F808C008700320187030BCA1
:108650000120704713F0070F04BFE94802700020A3
:10866000704710B503F00700E349012804BF00205C
:10867000886013D013F0070F10D18868E14B0428ED
:108680003CBFD3F800C00CF80020401C88600428D0
:1086900004D104221020196800F050FC002010BD05
:1086A0002DE9F047164603F007020024D24F012AB5
:1086B00004BFBC60FC6064D0DFF84C8313F0070F8C
:1086C00007D0022A33D0042A04BF387806284FD0B6
:1086D00058E0BD68002D08BFFE6125D0012D06D0F1
:1086E000D7F81090AC1E4C4516D284B908E0701C27
:1086F0003861F9690844B0F5007F88BF3C6113E038
:108700004FF400724FF43E31C04813F0D1FDBD4923
:10871000F869096820440E54601C484504D1BB48E0
:10872000C0F8FC8106203870681CB8602AE0FF227F
:1087300002703B69CBB1D7F81CC0FA689444BCF511
:10874000007F10D2B24D2D68454518BF047005D189
:108750000CF53C3C9CF800C880F800C0501C9842C6
:1087600004BF01200870501CF8600120BDE8F087AC
:108770004FF43E30FAF7B6F9A4494FF43E30FAF719
:1087800053FA3C700020BDE8F08770B503F0070095
:10879000994C1546012804BF0020A06014D013F0A6
:1087A000070F11D102F082F970B1A0689549022833
:1087B0003CBF0A681554401CA060022804D1022264
:1087C0000968052000F0BAFB002070BD2DE9F041DA
:1087D000054603F007008B4C874E0F4601280AD050
:1087E00013F0070F14D002281BD0042804BF3078E0
:1087F000062834D03FE00020B0602168087021686E
:108800004870216888702168C8700520307032E097
:10881000B06804282FD221680A54401CB06006209A
:1088200028E0B06860B905F00EF921680870226888
:10883000010A51702268010C000E91702168C87005
:10884000B06804283ABF2168095CFF21297024BF61
:1088500001213970401CB0600120BDE8F08102F0B8
:1088600025F940B12068C178006861F31F6005F008
:10887000E5F8032030700020BDE8F08170B503F00A
:1088800007015D4C064601290BD05E4D13F0070F22
:108890000CD0022914D0042904BF207806281DD04A
:1088A00025E00020A0600520207020E0A068B0F541
:1088B000007F1CD229680A54401CA060062015E0E5
:1088C000A06818B90021286813F060FD2868A16825
:1088D000405C3070481CA060012070BD02F0E6F8DA
:1088E00028B1A168286813F056FD032020700020ED
:1088F00070BD1FB513F0070F04D1012202A91B2080
:1089000000F01CFB04B0002010BD03F007003A4942
:10891000012806D013F0070F04BF0878012806D0FD
:1089200014E0012008700020886048610DE088682C
:10893000042805D24B69401C42EA03224A61886040
:10894000042803D1032008704869C86100207047DB
:1089500003F00700DFF8A0C0012807D013F0070FCD
:1089600004BF9CF80000022809D01EE002208CF809
:1089700000000020CCF80800CCF8180015E0DCF866
:108980000800022808D2DCF81810401C42EA012135
:10899000CCF81810CCF80800022806D1DCF8180032
:1089A000CCF8200003208CF800000020704770B441
:1089B00003F007020025104C012A02D0022A06D03B
:1089C00002E002202070A56070BC00207047227871
:1089D000022A2BD1D4F820C0A268624528BF1046D5
:1089E0001DD212F0030F04D1E36953F8046BC4E9FC
:1089F0000663237E03700DE0F88400108884001065
:108A00002084001098E90100554E564D94A900109D
:108A1000FCF90200A069000AA061501CA06060453A
:108A200004D10120A56008700320207070BC0120D3
:108A3000704770B503F007000025FF4C0E46012873
:108A400006D013F0070F04BF2078022805D02BE0D2
:108A500002202070A560A56126E0216AA0688842F6
:108A600019D2A169090A41EA0262401CA26110F010
:108A7000030FA0600FD1E069B0F5443F28BF02604A
:108A800006D2B0F5005F03D30422EC49FAF720F9CF
:108A9000E069001DE061216AA068884204D10120DC
:108AA000A560307003202070002070BD30B403F04A
:108AB00007040025DFF880C3012C08BFCCF808505C
:108AC00035D013F0070F02D0022C33D02FE0042A48
:108AD00008BF4FF4403028D013DC002A08BF4FF401
:108AE000005022D0012A08BF4FF443301DD0022A83
:108AF00008BF4FF41C3018D0032A08BFD04814D048
:108B000010E0052A08BF4FF43E300ED0CD48102AA1
:108B100000680AD0112A08BFCB4806D0202A08BF17
:108B2000B43002D0CCF8145001E0CCF8140030BCC2
:108B300000207047DCF80820042A07D2C2F10303A2
:108B4000DCF81440DB0024FA03F30370501CCCF86B
:108B50000800042824BF01200870012030BC7047A1
:108B600070B403F0070CB44DBCF1010F07D0B74C43
:108B700013F0070F07D0BCF1020F21D01DE0002039
:108B8000A860E86019E0A86805283CBF21680A547D
:108B9000042810D123682268D4F800C0D3F801302B
:108BA000696912781BBA9CF804C023F0FF0343EAFA
:108BB0000C0341F82230401CA86070BC00207047B4
:108BC000EB6873B1042B07D22268032B1A44527846
:108BD000027004BF01200870581CE86070BC0120BE
:108BE00070472268D5F814C012785CF822202668F5
:108BF0004FEA126C86F801C026684FEA124C86F8DC
:108C000002C026684FEA122C86F803C0D4F800C0D0
:108C10008CF80420D8E710B503F00700012804D130
:108C2000002211460E2000F089F9002010BD2DE928
:108C3000F04103F00704804E174688460546012C94
:108C400004BF0020B06017D013F0070F12D101F05D
:108C50002DFF78B1B0687D4902283CBF0A681754DF
:108C6000401CB060022807D102220968072000F0EA
:108C700065F901E0022C02D00020BDE8F081B26865
:108C800012B1012A04D009E0FCF7B8FA287005E017
:108C9000FCF7BAFA2870012088F80000B068401C80
:108CA000B0600120BDE8F08170B503F00700002539
:108CB000614C012808D013F0070F0BD0042804BF23
:108CC0002078062825D02DE06561A5616570A56036
:108CD000257027E0A068022807D2616942EA0121D5
:108CE000616161781144617010E0042807D2A169C4
:108CF00042EA0121A16161781144617006E0052812
:108D000004D261788A4204BF06212170401CA06011
:108D100008E0D4E9050101F003FA002804BF0120AE
:108D2000A0702570002070BD10B5434C13F0070FE4
:108D300007D003F00700042804BF2078062822D0BB
:108D40002BE0A068022807D2616942EA0121616133
:108D500061781144617013E03D49091808D23B491C
:108D60000968014401F8022C61781144617007E040
:108D70003849091804D261788A4204BF062121705B
:108D8000401CA06009E03449606901F0EBF900285B
:108D900004BF0120A07000202070002010BD03F04F
:108DA000070CBCF1010F00D0BEE723490020486149
:108DB000487088600870704730B403F007050024DD
:108DC000DFF874C0012D07D013F0070F0DD0022D6E
:108DD00050D0042D68D083E0CCF81440CCF8184073
:108DE000CCF808408CF800407AE0DCF80800022853
:108DF0000BD2DCF8141042EA0121CCF814109CF8D4
:108E0000011011448CF801102DE004282BD2DCF85D
:108E10001810032842EA0121CCF818109CF8013000
:108E20001A448CF801201ED106228CF80020DCF8B0
:108E30001420114312E00000F88400101085001087
:108E400000FE0200D4850010E8FC001098E9010043
:108E5000FEFDFFFFFDFDFFFF94A9001004BF4FF4CE
:108E6000C471CCF818102849401CCCF82810CCF854
:108E7000080035E0DCF80820042A28BF10460AD292
:108E8000C2F10303DCF82850DB0025FA03F303707A
:108E9000501CCCF80800042803D10120CCF808406D
:108EA000087030BC012070479CF80000062815D1DE
:108EB000DCF8140000224102DCF8180043021046DE
:108EC000B2EB930F06D251F8045B401C2A44B0EB7E
:108ED000930FF8D3CCF828208CF80040CCF8084049
:108EE00030BC002070474FF443300168880A42428A
:108EF00011EB822218BF401C404201EB8000C01CD5
:108F000020F0030070470000EFBEADDEF9480022FC
:108F100042708270C270427182710271DFF8D8C3F0
:108F2000114601EB410300200CEB43031A54401C93
:108F30000628FBD3491C2029F3D3704713F030BA1D
:108F40002DE9F04115460E460746FAF7CFF900F035
:108F500008040820FAF7C5F92A463146384613F0C6
:108F60001FFA05462046FAF7B7F92846BDE8F08112
:108F7000E048C0787047DF4880787047DD490020BE
:108F800088707047DB490820C871704770B50026AB
:108F9000F8F70EFF044610F00F0531D02846F8F719
:108FA0000AFF012D18D0FCF72FF944EA00640023D2
:108FB00022460321072004F0E1F914F0060F1FD028
:108FC0000126FCF71BF9044604F0CEFD0546022CF1
:108FD00018BF052C09D013E0FCF710F9C549CA7970
:108FE000904218BFC871DED1E7E70120FBF701FB13
:108FF000022D05D0022C4FF0020003D001F0E2F860
:10900000304670BD04F0ABFDFAE72DE9F84F0027BC
:10901000FAF7D9FD04F0F4FD002818BF0127FCF78A
:10902000EDF8022804D101F00DFD002818BF01273A
:10903000FFF7ACFF002818BF0127AE4EF0780028DC
:1090400000F05A82B0686D464FF0FF344FF00008D0
:1090500038B1B26800230121084604F08FF9C6F840
:109060000880FAF743F900F0080A0820FAF739F9FE
:109070003079DFF884B2F0B1B07900EB4001401CE8
:10908000C0B20BEB4101B071202828BF86F80680E2
:109090003079401E30714C7891F800900020002CFF
:1090A00005DD0A1892782A54401C8442F9DC81F8C4
:1090B000008081F801805046FAF70EF9002CC0F2CA
:1090C0000C8209F0FF000024232880F0C881DFE82B
:1090D00000F0D132F81B25351241F948D17F859A2D
:1090E000DC8AF6F5F4F3F2D1D1D1AFBFC5CAD1F124
:1090F000F0EFD1EEED009DF80000AC280CBF012090
:109100000220FCF73FF916E09DF800100120FCF763
:109110008AF80120B070044600F0A1B99DF8031050
:10912000009861F31F6001F055FF01210320FCF757
:109130007AF80120B070012400F091B9BDF8000068
:1091400040BA04F083FC02210320FCF76CF80120F4
:10915000B070F0E79DF801109DF80000FCF763F88F
:10916000E9E74FF0010A86F802A0707860BBF8F7D3
:1091700014FE48B39DF8005086F801A015F0040FC6
:1091800018BFFDF705FB15F0020F07D0FF210F20D8
:10919000FCF7E1FAFBF73BFB45F0010515F0010F89
:1091A00010D0FCF72BF8022802D104F0DDFC48B106
:1091B000FCF724F8052802D101F00FF810B10020C7
:1091C000FBF712FB86F8018086F8028000F047B9B1
:1091D0009DF80000401E01F06BFAACE79DF800001E
:1091E00004F0E3FCA7E79DF8000000F00F000FF08B
:1091F000BCFB9DF8000010F00F0018BF01200FF01D
:10920000B7FB00F02CB99DF8000060B1FBF7F6FF4A
:10921000022818BF012404F0ADFC01460220FCF72F
:1092200002F800F01CB900210620FBF7FCFF82E7E2
:109230009DF80000002818BF012004F081FC9DF873
:109240000000002818BF012000F0B2FF00F007B9AD
:109250009DF8000004F060FC00F001B9BDF80000CA
:1092600004F054FD67E79DF8000020B1012801D00B
:10927000022805D0F3E04FF44330F9F733FCEEE079
:1092800001F057FC00210420CFE7FAF72FF800F097
:1092900008040820FAF725F83079002808BF86F876
:1092A00003802046FAF718F80121BDE7D1E0A4E0D9
:1092B00083E075E02DE05BE04CE045E02CE01DE054
:1092C00000E076E09DF80000012804BF022105209F
:1092D000ABD0022804BF00210320A6D0032804BF7E
:1092E00000210420A1D004281CBF022108469AD0E6
:1092F0009BE700003085001094AB00109DF8030040
:10930000009A002360F31F626221072004F036F800
:10931000A5E0FBF75AFC0EE79DF800009DF8011050
:10932000000140EA111008F09EFE9DF801109DF822
:10933000020001F00F0140EA012008F09AFE9DF8BA
:10934000030008F0A2FE8AE0BDF8000040BA08F071
:109350007EFE84E09DF8000008F0AAFE9DF8010062
:1093600008F0B5FEBDF8020040BA08F0BFFE76E096
:109370009DF8000008F0CFFE9DF801009DF8021056
:10938000000140EA111008F0DBFE9DF802109DF884
:10939000030001F00F0140EA012008F0C2FE5EE088
:1093A0009DF800000AF05CFC9DF8000000287FF4A6
:1093B000C2AE0020FBF71DF9BDE60AF048FC0546E9
:1093C0009DF8004004F002FD012C0AD0022C08BFD9
:1093D00040F4807005D0042C14BF082C40F40070B9
:1093E00001D104F066FC20460AF02CFC082D12BFC7
:1093F000082C022004F0EEFB9DE69DF80050F6F7E5
:109400009EFF027815F0010F114614BF41F00201D2
:1094100021F00201337814BF43F0020323F002036A
:10942000337015F0020F14BF41F0040121F0040164
:10943000337814BF43F0040323F0040333709142E4
:109440000DD001700022012311461046F7F734F8C1
:1094500005E09DF800000AF0ECFB04F016FB0CB1EF
:1094600001273AE0B0686D464FF0FF3438B1B2687A
:1094700000230121084603F081FFC6F80880F9F7B0
:1094800035FF00F0080A0820F9F72BFF3079F0B11A
:10949000B07900EB4001401CC0B20BEB4101B07150
:1094A000202828BF86F806803079401E30714C781D
:1094B00091F800900020002C05DD0A1892782A54BB
:1094C000401C8442F9DC81F8008081F8018050461C
:1094D000F9F702FF002CBFF6F4ADF9F707FF00F033
:1094E00008040820F9F7FDFE3179002908BF86F845
:1094F00003802046F9F7F0FE002F14BF0120002062
:10950000BDE8F88F02460020022928BF704772B1DB
:1095100001EB4103C3EB4111012A08BFFA4803D014
:10952000022A0CBFF948704700EB8100704740F2F7
:10953000DB104843F64901EB8000704770B5F9F73E
:10954000D5FE00F008060820F9F7CBFEF14C002507
:109550006078FF2806D240F6D861ED4812F0ADFEE3
:10956000A570E570A079FF2805D2E821E64812F041
:10957000A4FEE5712572E07AFF2805D2E821E348D0
:1095800012F09BFE257365733046BDE87040F9F715
:10959000A3BEDFF884C300FB01F31CEB030C88BF00
:1095A0007047DC4B9A61C3E904017047DFF864C37C
:1095B0000028DCF8103018BF0360D6480029406945
:1095C00018BF0860002A1CBFDCF81810116058434F
:1095D0007047D04801210171007840F2DB1180F022
:1095E00001004843CA4901EB80007047C9488278AE
:1095F000002132B1C27822B9027882F001020270F1
:10960000817001717047C3491E284A78487008BFAD
:10961000002003D01F2808BF012000D10870104689
:109620007047BC48007840F2DB1180F001004843ED
:10963000B74901EB80007047F0B4B64E96F800C011
:1096400040F2DB140CFB04FCB14C356904EB8C0CD0
:1096500003FB05F40CEB440C8D4234BF2C460C4646
:109660007669F31A934238BF1A460026002A9CBF37
:10967000F0BC70470023002C06D930F813702CF88A
:1096800013705B1C9C42F8D8761C0CEB450C00EB6D
:1096900041009642EED3F0BC70472DE9F0419D4F5A
:1096A00014468C4601467A7806981D468A4218BFB1
:1096B000BDE8F0810121F970012802D0022824D0F0
:1096C00029E0387840F2DB11484391493E6901EBCB
:1096D0008001A64234BF324622467869A84238BF8C
:1096E00005460023002D16D90020002A06D91CF8B3
:1096F000007021F81070401C8242F8D85B1C01EB0E
:109700004601A444AB42EFD305E000232A4621469C
:109710006046FFF791FFBDE8F04100F0A1BB0028D3
:1097200008BF70477B497D4B4A787D491B78002AEA
:10973000097818BF022A05D0042A18BF092A01D0C7
:10974000012279E7774A1278012A84BF764A137892
:10975000012200F09FBB2DE9F04FDFF8B8A183B0E4
:1097600001218AF8031071496E4C6F4D0F786B49D7
:109770000E789AF80110112930D00EDC002918BF9C
:1097800002291DD0042918BF092919D098B1002336
:1097900032463946FFF750FF0DE0122918BF132952
:1097A0001CD0212918BF2229F0D120B10023B21CDE
:1097B0003946FFF741FF03B0BDE8F04F00F050BB62
:1097C0002178012902D95A492E780F780028F2D041
:1097D00000233246394600F05DFBECE7F8F7DFF98D
:1097E000F8F71AF90090002818BFF8F764FB207802
:1097F000012888BF2E78F8F7D8FA10F0040F18BFA8
:10980000761CDFF830919AF80100A0F111089AF85F
:10981000000040F2DB1148433D4901EB8004DAF8D7
:109820001000B84238BF0746DAF81400B04238BF1B
:109830000646F8F789FB01900020F8F7A3FE002503
:10984000002E39DD4FF0000A002FC4BF05EB4500A4
:1098500000EB051B29DD019810F90A00262824BF1A
:10986000002024F81A001CD200F0010109EB41315C
:1098700000EBD07001EB8B014010B8F1000F51F8F4
:1098800020104FF0FF301DD0B8F1010F08BFC8B253
:1098900005D0B8F1020F04BF0846F8F779FE24F8A6
:1098A0001A000AF1010ABA45D5DB1A486D1CB54207
:1098B000006904EB4004C5DB0098002818BFF8F7E6
:1098C000FDFA78E711F4803FC1F3072018BF40424A
:1098D000E5E7104801214172407980F0010000EB7A
:1098E0004001C1EB4010084901EB80007047094876
:1098F000C279002132B1027A22B9427982F00102A2
:109900004271C171417270472CBB001014BC001031
:1099100054AC00103C8500104AFCFFFFCD840010C1
:10992000D3840010CE840010D0840010CC840010AA
:10993000CF84001000800030F9491E288A79887190
:1099400008BF002003D01F2808BF012000D14871A4
:1099500010467047F248407980F0010000EB40016A
:10996000C1EB4010EF4901EB800070472DE9F04F4B
:10997000ED4985B0012291F80080EC4991F8009002
:10998000E7490A728979E74C11291CBF122913296A
:1099900029D090B1E249497901EB4102C2EB411172
:1099A00004EB8102002119EB080306D030F811C046
:1099B00022F811C0491C8B42F8D8F9F797FC00F047
:1099C00008050820F9F78DFCD54C607A002818BFEF
:1099D00001217CD0E1712846F9F77EFC002020723D
:1099E00005B0BDE8F08FF8F7DAF8F8F715F8019050
:1099F000002818BFF8F75FFAC9488179A1F111056D
:109A0000C1690091407900EB4001C1EB401004EBCB
:109A10008006F7F7E2F9C64FC6494FF0110A002851
:109A200004BF8B46012004D0BB4650460F464FF082
:109A3000010AF8F7A7FDF8F785FA00240390B9F1B9
:109A4000000F28D900984C214843029003980057F2
:109A5000262824BF002026F8140019D200F00101A6
:109A60000BEB413200EBD0700299401001EB80000B
:109A7000002D11584FF0FF3049D0012D08BFC8B25A
:109A800004D0022D04BF0846F8F782FD26F8140022
:109A9000641C4C45DAD306EB49065046F8F772FDD4
:109AA000F8F752FA00248246B8F1000F29D900983D
:109AB0004C2100FB01F94FF0000B1AF90400262895
:109AC00028BF26F814B019D200F0010100E02CE004
:109AD00000EBD070401007EB413109EB80000958D2
:109AE0004FF0FF30D5B1012D08BFC8B204D0022D10
:109AF00004BF0846F8F74CFD26F81400641C4445E2
:109B0000DBD30198002818BFF8F7D8F955E711F40E
:109B1000803FC1F3072018BF4042B7E711F4803FF0
:109B2000C1F3072018BF4042E6E7607980F00100EA
:109B3000607100214EE77A4801218173807A80F0BC
:109B4000010000EB4001C1EB40107B4901EB8000BC
:109B500070477348027B002132B1427B22B9827A7E
:109B600082F0010282720173817370476C491E2872
:109B7000CA7AC87208BF002003D01F2808BF01207E
:109B800000D18872104670476548807A80F00100E5
:109B900000EB4001C1EB4010674901EB80007047CA
:109BA0002DE9F04F5E4987B001224A73C97A624DB0
:109BB000624C11291CBF1229132930D0C8B1584951
:109BC000897A237801EB4102C2EB411105EB810256
:109BD00094F801C0002113EB0C0F0AD030F81130BB
:109BE00022F81130237894F801C0491C63448B4259
:109BF000F4D8F9F77BFB00F008060820F9F771FBB1
:109C0000474CA07B002500281CBF012121737DD07B
:109C10003046F9F761FB657307B0BDE8F08FF7F7E1
:109C2000BEFFF7F7F9FE0490002818BFF8F743F9D4
:109C30004348059020786178394A00EB0108D07AD2
:109C4000917AA0F11109D06901EB4103C3EB4111F5
:109C500005EB810B9169414538BF8846022102918D
:109C600012210391002500EB40012E4601EB001A62
:109C700002AC54F82600F8F785FC54F826000021C1
:109C8000F7F712FC009054F826000121F7F70CFCBE
:109C9000019006EB4600059900EB0610002401EB4D
:109CA000C0072EE0E01704EBD060421120F01F0047
:109CB0005DF82210221A01209040014220D004F0C9
:109CC000010007EB403004EBD47100EB8A0049102F
:109CD00000EB810141F64860B9F1000F09584FF0DF
:109CE000FF302FD0B9F1010F08BFC8B205D0B9F1CC
:109CF000020F04BF0846F8F74BFC2BF815006D1C4B
:109D0000641C4545B8BF262CCCDB00E021E0761C66
:109D1000022EADDB0498002818BFF8F7CFF868E7EB
:109D20003C8500102CBB0010D1840010D2840010A0
:109D3000B09D0030189D003014BC0010D484001079
:109D40000080003011F4803FC1F3072018BF40426B
:109D5000D3E7A07A80F00100A072257358E770B5B0
:109D60000D466F490122CA706E4A497816786E4ACC
:109D7000212914781EBF2229232970BD002818BF6D
:109D8000002D11D0002322463146FFF755FC631CFD
:109D9000012221462846FFF74FFC05EB4400A31C97
:109DA00001223146FFF748FCBDE8704000F058B88A
:109DB00070B55B4D0446687868B9E06858B15B4996
:109DC0000978012994BF584959490B78594901220A
:109DD000097800F05FF8E87A112804BF0020FFF747
:109DE000DFFEE87A122804BF0020FFF7D9FEE87AE8
:109DF000132804BF0020FFF7D3FE6878002804BFB3
:109E0000A068FFF7A8FC6878112804BF0020FFF7BE
:109E1000A2FC6878122804BF0020FFF79CFC687839
:109E2000132804BF0020FFF796FC206920B1A97910
:109E3000002908BFFFF79AFDA879112804BF002068
:109E4000FFF794FDA879122804BF0020FFF78EFDCC
:109E5000A879132818BF70BD0020BDE8704085E5C3
:109E600070B5F9F743FA00F008060820F9F739FA57
:109E70002B4C20790025002801BF207880F00100BC
:109E80002070A5701CBF0120A0703046F9F724FA9D
:109E9000E57070BD2DE9F047994616460D4604461B
:109EA000F8F757F85FEA000C1CD01D49087840F21B
:109EB000DB125043204AD1F8108002EB800009FBEE
:109EC00008F200EB4200454594BF2F4647464969DA
:109ED000A1EB0901B14238BF0E460021002E09D87E
:109EE000BDE8F0874B46324629462046BDE8F0479C
:109EF000FFF7A2BB0023002F08D91CF9032034F878
:109F0000122020F813205B1C9F42F6D8491C00EB5E
:109F1000480004EB4504B142ECD3BDE8F0870000F3
:109F20003C850010CC840010CD840010CE8400103D
:109F3000D0840010D384001054AC0010594900287C
:109F400014BF002001200870704756480078002890
:109F50000CBF0120002070475248017829B14FF012
:109F600040214A6942F001024A610021416081605A
:109F7000C1600161416170474A48017829B14FF0E1
:109F800040214A6942F001024A610021416081603A
:109F9000C16001614161704770B50446F9F7A6F9E7
:109FA00000F008050820F9F79CF93E4A3E490023D5
:109FB000106901EBC001401C1061B0F5807F28BF23
:109FC00013612078087060784870A0788870E07815
:109FD000C8702079087160794871A0798871E0793A
:109FE000C8715069B0F5807F3CBF401C506116D3EA
:109FF0001D20087001204870207888706078C87033
:10A00000A0780871E0784871207988716079C8710A
:10A01000D068401CD060B0F5807F28BFD360506806
:10A0200040F001005060107828B14FF040204169A5
:10A0300021F0010141612846F9F74EF9012070BD78
:10A0400000B50178427883B0890141EA82018DF838
:10A050000010418809098DF80110818809098DF8DF
:10A060000210817801F00F02017962F31F118DF85F
:10A070000310017A8DF80410417A8DF8051081796A
:10A08000C27901F03F0102F00C0241EA02118DF8A1
:10A090000610C07980018DF807006846FFF77CFF45
:10A0A00003B000BD5C8500105CBD0010194A0021A2
:10A0B00012684FF0402312F0804F26D0164AD2F893
:10A0C00000C05FEA1C4C04D011686FF30F0141F02F
:10A0D0000101D2F800C01CF47F4F0CD011684FF082
:10A0E000020C01F47F414CEA0121DFF830C0DCF8BA
:10A0F00000C0C3F874C0D2F800C01CF0FF0F04D039
:10A1000011680322C9B242EA014199678069D867A0
:10A11000FEE700002CED00E028ED00E038ED00E067
:10A1200070B50E460446FBF769F8042811D1A4F572
:10A130009C7050280DD2A019A0F23910502808D2D6
:10A1400065020024002E04D92846F8F7CBFC01282C
:10A1500001D0002070BD641C05F50075B442F3D336
:10A16000012070BD70B50D460446FBF747F8042882
:10A170000AD1A4F59C70502806D260022946F8F74F
:10A1800053FD012808BF70BD002070BD10B5074CFD
:10A19000FEF73BFF012808BF10BD206800F082FDDC
:10A1A000002818BFFBF782F8F2E70000D485001002
:10A1B000E34A0028516814BF41F0010021F001007A
:10A1C00050607047DE4B59680A0E120721F07F413C
:10A1D00042EA0060084358607047D9484068C0F3BD
:10A1E00003607047D6484068000F7047D448006944
:10A1F0007047D349012008617047D14900200861A8
:10A2000070472DE9F043AFB000270EF0BCFD0646C5
:10A21000A02102A812F051F8002425464FF00308AF
:10A220004FF00109305D10F0800F17D0601CC1B2F3
:10A230008DF8A9108DF8AF508DF8A880ADF8AC500E
:10A24000ADF8AA508DF8AE503555CDE900910022F9
:10A2500001272AAB114602A8F6F743F9601CC4B2E5
:10A260000A2CDFD3012F06D1102302AA06210120D8
:10A27000009510F0E9FD0EF0A1FB2FB0BDE8F083D2
:10A280002DE9F04FDFF8BC8287B0D8F80000B0F9B4
:10A290000E11B0F90C0112F06AF80120FAF7A9F9D1
:10A2A0000020F7F718FE0EF04FFD042000F010F923
:10A2B000FAF783F9FAF7A2FF05285ED1DFF888B232
:10A2C0009F4F4FF000094FF0402A7868C7F8089078
:10A2D000C0F30366C7F80C90D8F80000B100D0F8BE
:10A2E000F80020FA01F101F00F04C0F30321C0F3DC
:10A2F00003358C4222D10F2D20D003F0C4FC20B1B5
:10A3000009F0A5FC082818BF2C467869A04215D092
:10A3100009F09DFCAC420CBF0121002141EA00255F
:10A3200009F08AFC45EA004509F09DFC45EA006217
:10A3300000238421072003F021F87C6131460520A9
:10A3400003F09AF8002E7DD0022E1FD0042E7AD072
:10A3500078680A2E4FEA106120F07F404FEA0171C1
:10A3600018BF41F0007108437860FEF74EFE0128E7
:10A3700003D0FAF743FF0528A7D00EF01FFBFAF72A
:10A3800037F907B0BDE8F04F0EF0E3BC0D212046D1
:10A39000FBF736F80028E8D012F007F812F00AF8B8
:10A3A000FAF7C6F8040065D1F6F76FFF6748F7F7CC
:10A3B0007CFB0120F7F76EFBF8F7BAFF6448F9F76A
:10A3C0006CF8F9F753F8F9F77CF8D8F8001040006A
:10A3D000B1F80621B0FBF2F0401CC0F34F007880CA
:10A3E00091F80811397059B1F9F76BF8D8F80010E5
:10A3F0004000B1F80411B0FBF1F0401CC0F34F0075
:10A40000F8F7D0FF5348CAF81800F7F7C8FBF7F77A
:10A4100019FD387838B1401E10F0FF00387004BFC5
:10A420007888F8F7BFFF7868C0F3036529460520F0
:10A43000F5F75BFFFEF7E9FD012809D07868C0F366
:10A44000036001E03CE03FE0A84208BF002C18D0C8
:10A45000CAF818B0F8F7DEFFF9F713F80020F9F79B
:10A460001CF8F8F76EFFF7F79AFBF7F7D7FA00201A
:10A47000F7F71BFB11F09EFF11F0A1FFFBF72FF97F
:10A4800073E76846F7F7E0FE70B16846FFF790FCA7
:10A490000198F9F7E8FB684611F096FF0446F7F7D4
:10A4A00030FFFAF724FFC5E7D8F80000406E10F03F
:10A4B000704F02D0FAF7FAFEBCE7FAF71FFFB9E7D0
:10A4C000204611F086FF50E7204603F0ACFD4CE734
:10A4D00070B51C4980000968D1F8F81021FA00F025
:10A4E00000F00F04C1F30320C1F30335844224D1EB
:10A4F0000F2D22D003F0C7FB20B109F0A8FB0828DC
:10A5000018BF2C460E4E7069A04216D009F09FFB72
:10A510000146AC420CBF0120002040EA012509F0B1
:10A520008BFB45EA004509F09EFB45EA00620023EB
:10A530008421072002F022FF7461204670BD0000D4
:10A5400074850010D485001000005FA0EB39001066
:10A55000A733001007005FA07047002808BF7047AE
:10A5600080220146014811F0A3BE70475CC500106F
:10A57000704708283CBFFE49087070470020FC491E
:10A5800088604860FB48006890F88100082838BF60
:10A59000087070470020F64948607047F44800781A
:10A5A000704770B5F34D0024286890F86C0010F0E7
:10A5B000020F0BD0FAF722FE022807D1EC482968D7
:10A5C000007801EB8000B0F8840084B2204670BDB2
:10A5D00070B5E84D4FF48054286890F86C0010F086
:10A5E000020F0DD0FAF70AFE022809D1E0482968C7
:10A5F000007801EB8000D0F88400000CC0F3130455
:10A60000204670BDDA488078002818BF01207047C6
:10A610002DE9F041FAF7F2FD022803D103F0A4FA84
:10A62000022803D04FF48050BDE8F0814FF48055EC
:10A630002E4603F0B7FADFF83C830446CC4FD8F837
:10A64000000090F86C1011F0010F0CD0B0F87600FB
:10A65000B9684042814206DC2CB10020641EB8601B
:10A66000204603F0A2FAD8F8001091F86C0010F020
:10A67000040F18BF002C0AD0B1F87C00621E904075
:10A68000B1F87E20824238BF1046C0F31306D1F8DD
:10A69000A40010F0020F1CBFB978002902D0000CF2
:10A6A000C0F31305B54298BF35462846BDE8F08192
:10A6B0002DE9F04FDFF8BCA287B0DAF8001091F86E
:10A6C0006C2012F0020F0DD0A94A91F88090DFF8AB
:10A6D000A8B21778002809DB484503D2B84218BF52
:10A6E000064643D107B00020BDE8F08F3E464FF04C
:10A6F000FF38F7F793F9F7F7B0FF0025B9F1000F2E
:10A7000034D9DAF80000002400EB8500B0F88400AA
:10A7100081B22046F6F7D8FDF7F794FB6846F7F7C5
:10A7200093FD002866D0029878B1014693489BF8C3
:10A73000002000785043421E07D331F9020B002855
:10A74000B8BF40420444521EF7D2F7F7DAFDF7F7DC
:10A7500065F9002322469221072002F00FFEA04552
:10A7600084BF2E46A0466D1C4D45CAD3B74244D087
:10A77000082E3CBF7E490E70DAF80000B0F8821057
:10A7800039B300EB870200EB8600B2F88420B0F802
:10A79000840092B280B2801A484340F30F34F9F734
:10A7A000D2FA774B9BF80020002193F800C002FBFF
:10A7B0000CF2002A0DD930F81120224420F8112083
:10A7C0009BF8002093F800C0491C02FB0CF28A425F
:10A7D000F1D84FF0806003F022FBDAF8000000238C
:10A7E00000EB86008021B0F8840082B2072002F0DE
:10A7F000C5FD09E0FAF75AFD90E703F0D3F9032805
:10A800003CBF401C03F0D1F9012007B0BDE8F08F38
:10A81000584857490068B0F876004242886882423A
:10A82000BCBF401E886070472DE9F04F93B093463F
:10A830000E4604464FF0000A03F0B4F9DFF8348105
:10A840004B4F0500D14610D111F0C8FDD8F80010CB
:10A85000B1F87810884208D30120C7F8089003F0B7
:10A86000A4F913B00120BDE8F08F002E1FDDB868F9
:10A870000028B8BFC7F8089007DBD8F80010B1F877
:10A8800074108842BCBF401CB860D8F80000B9689A
:10A89000B0F87400884215DC032D13D2681CC7F889
:10A8A000089003F082F913B00120BDE8F08F09D1C0
:10A8B000D8F80000B0F876004142B8688842C4BFBA
:10A8C000401EB860B87850B1D8F8000090F8A400E5
:10A8D00010F0040F1EBF002013B0BDE8F08FD8F8B1
:10A8E0000000B0F972108C420EDD79682144796065
:10A8F000B0F86E00884210DC4FF0FF30C7F80490CB
:10A90000FFF7D6FE824608E07868002805DD002CB7
:10A91000D4BF01212146401A7860DFF8689099F889
:10A92000000007283BD11848594600784200684685
:10A9300011F0CDFCADF80040ADF80260ADF8045068
:10A940003889ADF80600B888ADF80800D8F80000DE
:10A95000B0F87210ADF80A10B0F87410ADF80C1021
:10A96000B0F86E10ADF80E10B0F876000EE00000F2
:10A97000C0850010D4850010CC840010D084001055
:10A98000CD8400103D850010D3840010ADF8100078
:10A9900099F80000072804BF6846FEF7C0FE50463D
:10A9A00013B0BDE8F08F3E4810B50068D0F8A400A1
:10A9B00010F4807F06D0C0F30330012101FA00F0CB
:10A9C000F8F701FA374900204870887010BD70B55B
:10A9D000344D0024A878002814BF0126002668788A
:10A9E00028B903F0EEF8002808BF002100D00121AB
:10A9F0008E4225D00A1C18BF0122AA702848006880
:10AA0000D0F8A43013F0040F0ED021B1C3F303101B
:10AA1000082808D206E00021A960696090F881004A
:10AA2000082800D22870012413F0020F18BF012457
:10AA3000002A18BF012200238221072002F09EFC79
:10AA4000204670BD164900200968D1F8A41011F401
:10AA5000807F08BF7047DFF84CC09CF80120131CB2
:10AA600018BF012330B4104CC1F30332E46B01254D
:10AA700005FA02F2224011F4007F01D00AB102E08F
:10AA80000AB1002100E001218B4204BF30BC7047B5
:10AA9000081C18BF01208CF8010030BC97E70000AB
:10AAA000D4850010C085001000100040694800786F
:10AAB00070476848406800F54070704765484068D6
:10AAC00000F58070704770B5624C4FF41C326249DB
:10AAD00062601068884204BF5068B0F5087F26D1D4
:10AAE000D2F808C0BCF5084F21D85C49D06888422C
:10AAF0000DD0002311461846B3EB9C0F07D251F836
:10AB0000045B401C6B40B0EB9C0FF8D37BB9012574
:10AB100002F5807000F0C6F848B1606800F540703A
:10AB200000F0CFF800281EBF2570012070BD002066
:10AB300070BD4849002008704FF41C30F7F7D2BFB1
:10AB40004448017841B14068434A0168914202BFDC
:10AB50004168B1F5087F7047002070473D4B5B6846
:10AB600003F580731844F8F7B3B83A4B5B6803F504
:10AB700040731844F8F7ACB836484068006970472D
:10AB8000344949680A6982429CBF00207047C0EB83
:10AB9000C00001EBC00000F5806070472D4A52688C
:10ABA00002EB80035B6A1A442D4B53F820C04033FC
:10ABB00033F810000CEB0003401E5B1E23EA00007C
:10ABC00000FB012070472DE9F003224B244F0022A7
:10ABD0005C6807F140069046831893F928C0BCF1E1
:10ABE000000FB8BF41F8228012DBD3B204EB83051B
:10ABF00057F8239036F813306D6A99445B1EA9F11B
:10AC00000109254429EA030303FB0C5341F82230D0
:10AC1000521C102AE0D3BDE8F00370470029B8BFEA
:10AC2000704730B494460B4A0E4C526802EB8003D6
:10AC30005B6A13440A4A52F8202034F810001418B2
:10AC4000401E641E24EA000001FB003030BC614657
:10AC5000F8F73EB8CC85001054465053EFBEADDE39
:10AC60009CE90100DCE9010010B5FFF72CFFA8B159
:10AC7000FFF71FFF0146D022174811F019FBFFF71D
:10AC80001DFF164C01464FF4E272206811F010FBD4
:10AC90002068406DBDE8104002F00DBF0220FAF7B9
:10ACA00071FBE2E758B10E4A0168914207D1406852
:10ACB00020F00F00B0F5107F04BF01207047002086
:10ACC000704730B1006820F00F00602804BF0120F9
:10ACD0007047002070470000E8FC0010D485001089
:10ACE00041505352B34810B5806810F0020F15D090
:10ACF000F6F792FE90B1F6F752FE0402FAF77EFAEA
:10AD000044EA0044FAF780FA44EA00604EF2AF01E8
:10AD100008434FF04021C867012010BD002010BD3E
:10AD200010B572B60120F7F7E1FDF8F785FCF8F7EA
:10AD3000AFFC4FF0FF30F8F7D4FA9F4880234FF470
:10AD40000052002152F821C040F821C0491CB1EB4B
:10AD5000930FF7D3F8F7D7FAF8F7FAFEF8F71CFFD6
:10AD60009648F8F735FF0120F8F7F3FEF7F752FEA3
:10AD70001E20F8F7E3FEF8F7A7FCF8F72FF8F8F72E
:10AD80009FFEF8F7E7FCF8F7CFFAF8F79FF8F6F729
:10AD900058FEFFF769FFF8F74EFAF8F719FAFEF7D1
:10ADA000B5F8FBF701FDFFF7E7F862B684480DF050
:10ADB000E5FD844C2068B0F90C010DF0BDFFF5F7FE
:10ADC0007AFAFFF7D5FBF8F71FFFFAF7C0FC206807
:10ADD000018BC1F30722418A008AFEF7DAFB206863
:10ADE000806E000C02F0C7FAFFF7B6FB11F0FBFA19
:10ADF000FAF7FCFA206890F8640000F00F00F7F70B
:10AE00009BFC206890F8200010F0010F04BF002187
:10AE1000032003D002F0AEFE01460220FAF703FA47
:10AE20004FF040242069002300F0700219460220F0
:10AE300002F0A4FA206910F0200F17D0226F00232F
:10AE40000521072002F09AFA626F002305210720EE
:10AE500002F094FAA26F00230521072002F08EFA77
:10AE6000E26F00230521072002F088FAFFF79BFD1F
:10AE7000F9F7E1FD0020206710BD534CFEF7C5F83F
:10AE8000012806D0FAF7BAF9032802D102F021FB13
:10AE900040B3002C05DC02F06DFE01460220FAF7FB
:10AEA000C2F9DFF82C810127484E4FF04025A8F168
:10AEB0000309FAF7A3F90446FAF7A6F90146204672
:10AEC00002F0DAFAFAF7A0F901462046F5F70DFA92
:10AED000FEF758F8072C68D2DFE804F0671A082458
:10AEE00027172A00641E002CC8DCD4E7307848B944
:10AEF000FBF7F8FB30B900231A462021072002F0A7
:10AF00003DFA377003F047FBD3E7FFF7B9F9D0E715
:10AF1000FBF706FBFAF772F9012804BF0220FAF7E3
:10AF20007FF9C6E702F04FFDC3E7FFF72FF9C0E74F
:10AF30000024C5F81880FEF768F8012806D1FAF752
:10AF40005DF9062802D0C5F81890B2E7FAF759F96A
:10AF500040B3002C04DCFAF7BFF943F22054EAE7CF
:10AF6000641E00BF00BF00BF00BF00BF00BF00BF26
:10AF700000BF00BF00BF00BF00BF00BF00BF00BFD9
:10AF800000BF00BF00BF00BF00BF00BF00BF00BFC9
:10AF900000BF00BF00BF00BF00BF00BF00BF00BFB9
:10AFA00000BFC8E7FAF782F9C5E70220FAF7EAF925
:10AFB0007FE70000008000400000011095CC0000F9
:10AFC000E8FC0010D4850010FF700200D885001046
:10AFD00003005FA0FE490860704710B44FF4403092
:10AFE000FC4A016891421CD14168B1F5007F18D339
:10AFF000836800228446B3F5056F88BF4FF405636C
:10B000000021B1EB930F24BF10BC70475CF82140C6
:10B01000491C2244B1EB930FF8D3002A04BF10BCA3
:10B020007047002010BC704770B54FF440310446A3
:10B03000E84D0868A84217D14868B0F5007F13D3DF
:10B040008B6800228C46B3F5056F88BF4FF405630B
:10B050000020B0EB930F08D25CF82060401C324413
:10B06000B0EB930FF8D302B1002149B18A68B2F571
:10B07000056F88BF4FF40562204611F019F91CE0F6
:10B08000FF224FF40561204611F044F94FF4087097
:10B09000C4E900504FF40560A0600020E06084F82F
:10B0A000200084F8210084F8220084F8230040F274
:10B0B000FF71C4E90410A061E061012070BD70B5AA
:10B0C0000021C160D0F808C00B460446BCF5056FEE
:10B0D00088BF4FF4056C0022B2EB9C0F06D254F8E7
:10B0E0002250521C2B44B2EB9C0FF8D35942C16042
:10B0F0004FF440304FF405622146F7F7E9FD01288F
:10B1000018BF002070BDFF2270B500250446056100
:10B110004FF40061503011F0FDF8A584E584E5623C
:10B12000A56265632563E563A56365642564E564DD
:10B130000120A56470BD70B402684FF408715160BD
:10B14000016801F1500291F821C091F820300CFB08
:10B1500003F102EB41010022BCF1000F08D900EB22
:10B160004204521CB4F8EA4021F8024B9445F6D848
:10B170000022002B08D900EB4204521CB4F8124103
:10B1800021F8024B9342F6D80468002294F822403A
:10B19000002C0BD900EB4204521CB4F8BE4321F83A
:10B1A000024B046894F822409442F3D804680022C9
:10B1B00094F82340002C0BD900EB4204521CB4F845
:10B1C000CE4321F8024B046894F823409442F3D80C
:10B1D0000022BCF1000F08D900EB4204521CB4F865
:10B1E000704021F8024B9445F6D80022002B08D974
:10B1F00000EB4204521CB4F8984021F8024B9342F1
:10B20000F6D8B0F8E62021F8022BB0F8E82021F8B3
:10B21000022BB0F8E42021F8022B00240022BCF11C
:10B22000000F0ED904EB440505EB041500EB850572
:10B2300005EB4206521CB6F85E6121F8026B6245CE
:10B24000F6D30022002B0ED904EB440505EB0415C0
:10B2500000EB850505EB4206521CB6F88E6221F81C
:10B26000026B9A42F6D3641C042CD7D30023D0F887
:10B2700000C000229CF822C0BCF1000F88BF00EB88
:10B28000031C0BD90CEB4204521CB4F8DE4321F82A
:10B29000024B046894F822409442F3D8D0F800C0DE
:10B2A00000229CF823C0BCF1000F88BF00EB031CF8
:10B2B0000BD90CEB4204521CB4F8FE4321F8024BAC
:10B2C000046894F823409442F3D85B1C022BCED33D
:10B2D00070BC70472DE9F74F88B000250A992C46BD
:10B2E0002E460968049101F150030999002984BF91
:10B2F0003949D1F800801CD90022002888BFB8F94C
:10B30000CE700DD933F9021B0029B4BFC1F1000C76
:10B310008C46BC45BCBF0D44641C521C8242F1D318
:10B320000999761C8E42E7D3002CC8BF95FBF4FA2E
:10B3300008DC4908414301EB5002049901EB42014A
:10B34000B1F950A00021029101910499503100916E
:10B35000002103910999002975D91F49009E06967D
:10B3600009684FF0000B4FF00109B1F9C0E0D1F8C6
:10B37000B4105F46C1F30741D846CDF814B0079129
:10B38000002830D9B6F900204FF0000C06999344FC
:10B39000634600280DD9B1F90040A51A48BF151B16
:10B3A0007545B8BF0CF1010C01EB49015B1C8342F0
:10B3B000F1D307998C4503D305997F1C114405915E
:10B3C00008F1010806EB49068045DBD3002F05E0B4
:10B3D000DC85001053454C46D4850010C4BF059948
:10B3E00091FBF7F101DC9BFBF0F1039B0A9A09B298
:10B3F00002EB4302A2F87010FE4A1268B2F9BA30AA
:10B40000AAEB030399420ADDB2F9B82052448A42FA
:10B4100005DD019A114401910299491C029100999C
:10B42000099A01EB400100910399491C0391914253
:10B4300093D30299002906DDDDE9011291FBF2F1B7
:10B44000019103E0FFE75146CDF804A00A9AA2F863
:10B45000E6100021029103910499503100910021DE
:10B460000491002868D9E349009F069709684FF0C6
:10B47000000B099EB1F9BCE0D1F8B410D846090E12
:10B48000D946CDF814B00791002E2BD9B7F900207A
:10B490004FF0000C069993446346002E0DD9B1F984
:10B4A0000040A51A48BF151B7545B8BF0CF1010C2B
:10B4B00001EB40015B1CB342F1D307998C4504D3E7
:10B4C000059908F101081144059109F1010907EBFB
:10B4D0004007B145DAD3B8F1000FC4BF059991FB1D
:10B4E000F8F101DC9BFBF6F1049B0A9A09B202EB2E
:10B4F0004302A2F89810BF4A1268B2F9BA30AAEB18
:10B50000030399420ADDB2F9B82052448A4205DDAC
:10B51000039A114403910299491C02910099891CD4
:10B5200000910499491C049181429CD302980028FF
:10B53000C4BF039991FBF0FA0A98A0F8E8A001981B
:10B540000A99504400B200EBD0704010A1F8E4001A
:10B550000BB0BDE8F08F2DE9F04F146889B01546A7
:10B560000E460746A1F12008202928BF4FF0FF3AD8
:10B5700005D24FF0010000FA06F0A0F1010A38BF31
:10B580004FF0000B05D34FF0010000FA08F0A0F1D6
:10B59000010B202F3DBF0120B840401E4FF0FF306F
:10B5A00038BF002207D3A7F120024FF0010101FAB2
:10B5B00002F1A1F10102C6F12009202E34BF20FAC8
:10B5C00009F100FA08F1B2401143B040CDE90001A1
:10B5D000206920F4FE6020618748007810F0010F98
:10B5E0007ED02A463146384601F08AFC0020A86108
:10B5F0006861002F84BFDFF8FCE101221BD905EB55
:10B600004001B1F998100029B8BF494209B2DEF8EB
:10B610000030B3F9CC308B420ADD410905EB8101E2
:10B6200000F01F0C4B6902FA0CFC43EA0C034B615F
:10B63000401CB842E3D30020012F18BFA7F1010E30
:10B640003BD005EB4001B1F99A30B1F99820991A35
:10B6500048BFD11A09B2DFF89CC1DCF800C0BCF9C0
:10B66000C4C08C4526DAB5F9E810B2EB010C48BF2E
:10B67000A1EB020C0FFA8CFC5A1A48BFCA1A11B27D
:10B680008C450BDB420905EB820100F01F0C012207
:10B690004B6902FA0CF21A434A610BE0411C4B0958
:10B6A00005EB830201F01F0C0121536901FA0CF133
:10B6B00019435161401C7045C3D36969E869B140C1
:10B6C00008432063A969286AB1400143616368693E
:10B6D000202E34BF20FA09F000FA08F0084300E0F9
:10B6E00000E0606344480068079010F0040F00F029
:10B6F000BC8100202863E862002E88BFDFF8F4E0F8
:10B700001BD9DEF8002005EB4001B1F95E11B2F95A
:10B71000D8308B4203DCB2F9DA208A420ADA4209D5
:10B7200005EB820100F01F0C0122CB6A02FA0CF239
:10B730001A43CA62401CB042E3D30020A862686288
:10B74000002F88BFDFF8ACE01BD9DEF8002005EB46
:10B750004001B1F98E12B2F9D8308B4203DCB2F954
:10B76000DA208A420ADA420905EB820100F01F0C56
:10B7700001224B6A02FA0CF21A434A62401CB84298
:10B78000E3D300202864E863002E88BFDFF864E07C
:10B790001BD9DEF8002005EB4001B1F9AA11B2F97E
:10B7A000DC308B4203DCB2F9DE208A420ADA42093D
:10B7B00005EB820100F01F0C0122CB6B02FA0CF2A8
:10B7C0001A43CA63401CB042E3D30020A8636863F5
:10B7D000002F88BFDFF81CE020D9DEF8002005EB41
:10B7E0004001B1F9DA12B2F9DC308B4208DCB2F96F
:10B7F000DE2003E0D4850010DC8500108A420ADADE
:10B80000420905EB820100F01F0C01224B6B02FA8A
:10B810000CF21A434A63401CB842DED3002028656C
:10B82000E864A8646864002E88BFDFF844E71CD988
:10B83000DEF8003005EB4001B1F9F611B3F9E02074
:10B840008A4203DCB3F9E2208A420BDA410905EBB4
:10B85000810C00F01F030121DCF84C2099401143BA
:10B86000CCF84C10401CB042E2D30020002F88BF1F
:10B87000DFF8FCE61BD9DEF8002005EB4001B1F94A
:10B880002613B2F9E0308B4203DCB2F9E2208A429F
:10B890000ADA420905EB820100F01F0C01224B6C11
:10B8A00002FA0CF21A434A64401CB842E3D3696AB4
:10B8B000E86AB14040EA010EC4F838E0A96A286B92
:10B8C000B1400843E063696A202E34BF21FA09F1D0
:10B8D00001FA08F141EA0000E0630590696BE86B4A
:10B8E00001FA06F140EA01022264A96B286C01FA10
:10B8F00006F140EA01006064696B34BF21FA09F186
:10B9000001FA08F141EA000161646B6CE86C03FA2A
:10B9100006F340EA0300A0640490AB6C286D03FAC0
:10B9200006F340EA0300E0646B6C34BF23FA09F3CA
:10B9300003FA08F343EA0000E0640290059832EA53
:10B940000E0521EA000C4EEA05022564069240EA43
:10B950000C00C4F844C006EB0701039008BFBCF11B
:10B96000000F42D000231A461846002988BF01273D
:10B970003BD94FEA501804EB880800F01F09D8F8AB
:10B98000408007FA09F918EA090F03D0864294BFEC
:10B99000521C5B1C401C8142EBD8012B0FD105EAE5
:10B9A0000A0040EA0E00A06305980CEA0B03184356
:10B9B000E06325EA0A0020642CEA0B006064012A97
:10B9C00013D1226C0098A36B10401843A063606CE5
:10B9D000019BD4F83CC0034043EA0C03E363009BA3
:10B9E0009A432264019A90436064069A049830EA6C
:10B9F0000202A264069840EA020CDDE9020320EA92
:10BA00000300E064039B43EA000508BF002821D03F
:10BA100000231A461846002988BF012717D94FEA84
:10BA2000501804EB880800F01F09D8F8488007FA7E
:10BA300009F918EA090F03D0864294BF521C5B1C17
:10BA4000401C8142EBD8002B18BF002A02D10020F5
:10BA5000A064E064079810F0010F06D0206B20EA84
:10BA60000C002063606BA8436063206B0099084260
:10BA700003D1626B01990A4203D0216941F01001A0
:10BA8000216110EA0A0F04BF606B10EA0B0F03D0AC
:10BA9000206940F020002061A06B0099084203D18A
:10BAA000E26B01990A4203D0216941F04001216112
:10BAB00010EA0A0F04BFE06B10EA0B0F03D02069F5
:10BAC00040F080002061206C0099084203D1626C34
:10BAD00001990A4203D0216941F48071216110EA81
:10BAE0000A0F04BF606C10EA0B0F03D0206940F40A
:10BAF00000702061A06C002804BFE06C002803D017
:10BB0000206940F48060206109B00120BDE8F08F19
:10BB10002DE9F04FBDB016460D460446F5F77EFF01
:10BB2000F5F75BF901004FF011001DBF02900120F5
:10BB30000390012108BFCDE90210CDE93854F6F792
:10BB400001FA0022002D88BF04A904D9835C8B541C
:10BB5000521C9542FAD8F6F7F7F90021002C88BF5D
:10BB600004AA07D9435C02EB010C491C8CF8203075
:10BB70008C42F7D8F6F719F93190FE48007810F0AA
:10BB8000200F5DD0F5F729F9FB49FC4A00280CBFCE
:10BB9000CDE90021CDE9001206F1EA003A90283003
:10BBA0000025EA460DF1E8090DF1E00B3B9002A8F3
:10BBB0005BF8257050F82500F6F7E4FC0024002F10
:10BBC00084BF04A800EB451818D918F904002628EA
:10BBD00028BF00200BD2C10700EBD070890C4010A9
:10BBE00001EB80005AF825104058F6F7D1FC59F8BF
:10BBF000251021F81400641CBC42E6D36D1C022DF4
:10BC0000D5D3DF4805781D2D1AD100210A4614AB83
:10BC10005BF822400020002C88BF59F822C007D9C9
:10BC20003CF8107023F81170401C491C8442F7D86E
:10BC3000521C022AECD31D2D04BF1846FDF796FEB8
:10BC4000CC4D287810F00C0F00F0CB82F5F7C5F83A
:10BC5000CC49CD4A00280CBFCDE91421CDE91412FE
:10BC6000CA48F5F784FF0120F5F71EFB2D9001204F
:10BC7000F5F76AFB2B900120F5F744FE1B90029824
:10BC8000F5F78FFB28900398F5F78BFB17900120B1
:10BC9000F5F71CFC2E901120F5F718FC27900120D9
:10BCA000F5F754FC2C901120F5F750FC1D9024A8BA
:10BCB000009022AB20AA1EA90298F5F76AFD25A8DC
:10BCC000009023AB21AA1FA90398F5F762FD029803
:10BCD000F5F7E1FD26900298F5F7DDFDA44C019003
:10BCE0002068B0F8E4100120F5F7EEFA00210120F9
:10BCF000F5F7F0FD206890F8E6100298F5F763FB81
:10BD0000206890F8E6100398F5F75DFB002101200C
:10BD1000F5F7F5FB00211120F5F7F1FB00210120DB
:10BD2000F5F72DFC00211120F5F729FC2068B0F86B
:10BD3000E8100298F5F75DFD2068B0F8E810039868
:10BD4000F5F757FD00210120F5F7F6FD2990894808
:10BD5000007810F0040F00F047812068B0F8EC1074
:10BD6000009190F8EB3090F8EA200B210298F5F75B
:10BD7000E2FC2068B0F8EC10009190F8EB3090F8FD
:10BD8000EA200B210398F5F7D6FC00210120F5F7F6
:10BD9000D3FD32A801F09FF83699002238AD00207B
:10BDA00055F822C0BCF1000F0ED902EB420303EBA1
:10BDB000021306EB031331F8027B03EB4008401C2F
:10BDC000A8F85E718445F6D8521C022AE7D302987F
:10BDD000F4F72FFD1C900398F4F72BFD1A90002127
:10BDE0000298F5F761FB189001210298F5F75CFBCA
:10BDF000169000210398F5F757FB2A90012103982C
:10BE0000F5F752FB5A4C19902068B0F8EE100091EB
:10BE100090F8EB3090F8EA200B210298F5F78BFCB4
:10BE20002068B0F8EE10009190F8EB3090F8EA201E
:10BE30000B210398F5F77FFC00240DF1080B00217E
:10BE40000120F5F779FD00210298F4F7DAFC0021D2
:10BE50000398F4F7D6FC5BF824000121F4F7D1FC39
:10BE600038A8002550F8249014A8B9F1000F50F814
:10BE700024002F9049D904A800EB4410009004EB53
:10BE8000440000EB041006EB001A00980022114653
:10BE900010F905801046F5F75DFDB8F1200F06DBBF
:10BEA0000027A8F12001012000FA01F804E0012098
:10BEB00000FA08F74FF000085BF824003A4600212A
:10BEC000F5F7E0FA5BF8240042460121F5F7DAFACB
:10BED0006FEA0802F9430920F5F73CFD32AFF5F7A8
:10BEE000B1FFFDF792F8012804D03846F6F7ACF917
:10BEF00000287CD0F5F792FD2F9800880AEB4501C9
:10BF00006D1CA1F8AA014D45BFD300221146104671
:10BF1000F5F720FD641C022C91D31C990298F4F7CC
:10BF200070FC1A990398F4F76CFC0021189A029897
:10BF3000F5F7A8FA0121169A0298F5F7A3FA00215D
:10BF40002A9A0398F5F79EFA0121199A0398F5F7B2
:10BF500099FA074C2068B0F8F010009190F8EB3097
:10BF600090F8EA200B210298F5F7E5FB20680FE036
:10BF7000D4850010DC850010B09D0030189D003085
:10BF800042850010CC0E0030CC09003001000E00BC
:10BF9000B0F8F010009190F8EB3090F8EA200B2107
:10BFA0000398F5F7C8FB01210846F5F7C5FC32A850
:10BFB00000F091FF3699002238AC002054F822306E
:10BFC000002B0ED902EB420C0CEB021C06EB0C1CF6
:10BFD00031F8025B0CEB4007401CA7F8F651834296
:10BFE000F6D8521C022AE8D3FE48007800E049E067
:10BFF00010F0080F7DD0FC4D2868B0F8F2100091C9
:10C0000090F8EB3090F8EA200B210298F5F793FBBB
:10C010002868B0F8F210009190F8EB3090F8EA2020
:10C020000B210398F5F787FB00210A4638AF002063
:10C0300057F821C0BCF1000F0CD901EB410303EB11
:10C04000011306EB031303EB4004401CA4F8422247
:10C050008445F8D8491C0229E9D32868002490F8BF
:10C060002401B4EB400F7CDA286890F82401A04248
:10C07000D4BF012100210120F5F75EFC32AFF5F7B6
:10C08000E1FE02E0F9F712F92BE7FCF7BEFF012809
:10C0900003D03846F6F7D8F860B3F5F7BFFC369909
:10C0A0004FF000090DF1E00E00225EF829701046F5
:10C0B000002F05D931F91030401C1A448742F9D8B5
:10C0C000B2FBF7F2781E3ED009EB490303EB0913EC
:10C0D00006EB031A31F9103001EB400C3CF9028CED
:10C0E000B3EB080348BF5B4231F91080B8EB02089C
:10C0F00001E036E01CE031F910804CBFA2EB0808EB
:10C10000A8EB02083CF902BC3CF902CCBBEB020BE9
:10C110004CBFA2EB0C0CACEB020CE0450AEB400C64
:10C1200009DDBCF942824345C8BFACF8423208E0A1
:10C13000F9F7BCF8A9E7BCF940829845B8BFACF85C
:10C140004032401EC6D109F1010901EB4701B9F1A6
:10C15000020FA9D32868641C90F82401B4EB400FA7
:10C1600082DB01202D99F5F7AFF801202B99F5F727
:10C17000F6F801201B99F5F7ADFB28990298F5F721
:10C1800022F917990398F5F71EF901202E99F5F772
:10C19000B6F911202799F5F7B2F901202C99F5F796
:10C1A000EEF911201D99F5F7EAF924980090229BE9
:10C1B000209A1E990298F5F7BEFA25980090239BC5
:10C1C000219A1F990398F5F7B6FA26990298F5F780
:10C1D00010FB01990398F5F70CFB01202999F5F75D
:10C1E000ABFB3198F5F7C3FC3DB0BDE8F08F2DE90E
:10C1F000F04FABB091460D460446F5F70FFC022216
:10C20000209212222192CDE90C45F5F7CEFD19902E
:10C2100074484FF00107007810F0210F6CD073487C
:10C220000E9073480F9000212098F5F73DF9089083
:10C2300001212098F5F738F9099000212198F5F7A8
:10C2400033F90A9001212198F5F72EF900250B907A
:10C250000CA850F825B020A850F82500F6F792F960
:10C26000002408A8264609EB051A00EBC50819E0CA
:10C27000600904F01F0158F8200007FA01F1084294
:10C280000FD0E007800C610800EB81010EA850F888
:10C2900025004058F6F77CF90AEB4601761CA1F818
:10C2A000BE03641C5E4538BF262CE1D36D1C022DF5
:10C2B000CED3504805781D2D1ED100210A466C466C
:10C2C0000CAE002056F822C0BCF1000F88BF09EB6D
:10C2D000021309D903EB4008401CB8F8BE8324F8C8
:10C2E0001180491C8445F5D8521C022AE9D31D2D22
:10C2F00004BF2046FDF754FC3A48007810F0040FC4
:10C3000000F0C6813C4816903C4817900220F4F794
:10C31000CBFF27900220F5F717F825900220F5F7BC
:10C32000F1FA1B902098F5F73CF81A902198F5F750
:10C3300038F818900220F5F7C9F826901220F5F782
:10C34000C5F81F900220F5F701F924901220F5F7A7
:10C35000FDF81D900EA8009006AB04AA02A9209833
:10C36000F5F717FA0FA8009007AB05AA03A92198C3
:10C37000F5F70FFA2098F5F78EFA22902198F5F745
:10C380008AFA194D01902868B0F8E4100220F4F7F9
:10C390009BFF00210220F5F79DFA286890F8E6102F
:10C3A0002098F5F710F8286890F8E6102198F5F72E
:10C3B0000AF800210220F5F7A2F800211220F5F773
:10C3C0009EF800210220F5F7DAF800211220F5F797
:10C3D000D6F82868B0F8E8102098F5F70AFA286827
:10C3E0000EE00000DC850010D4850010489E00306F
:10C3F000E09E0030478500104C1800304C1D003086
:10C40000B0F8E8102198F5F7F4F900210220F5F7CB
:10C4100093FA23902868B0F8EC10009190F8EB3074
:10C4200090F8EA200B212098F5F785F92868B0F8F4
:10C43000EC10009190F8EB3090F8EA200B21219855
:10C44000F5F779F900210220F5F776FA10A800F047
:10C4500042FD159900220CAC002054F822C0BCF11A
:10C46000000F88BF09EB421308D931F8026B03EBC8
:10C470004008401CA8F8DE638445F6D8521C022A06
:10C48000EAD32098F4F7D5F91E902198F4F7D1F962
:10C490001C9000212098F5F707F8089001212098BA
:10C4A000F5F702F8099000212198F4F7FDFF0A90B2
:10C4B00001212198F4F7F8FF0B902868B0F8EE10EE
:10C4C000009190F8EB3090F8EA200B212098F5F7D6
:10C4D00032F92868B0F8EE10009190F8EB3090F83F
:10C4E000EA200B212198F5F726F900250DF1800BA4
:10C4F00000210220F5F720FA00212098F4F781F9B5
:10C5000000212198F4F77DF95BF825000121F4F76B
:10C5100078F90CA8002450F82500299016A8264682
:10C5200050F82500289008A800EBC50009EB451A33
:10C53000009044E0009861094FF0010850F8210094
:10C5400004F01F0108FA01F1084237D00022114619
:10C550001046F5F7FFF9202C23BF0027A4F1200097
:10C5600008FA00F808FA04F738BF4FF000085BF843
:10C5700025003A460021F4F785FF5BF82500424686
:10C580000121F4F77FFF6FEA0802F9430920F5F76C
:10C59000E1F910AFF5F756FCFCF737FD012804D0A0
:10C5A0003846F5F751FE002879D0F5F737FA289884
:10C5B00000880AEB4601761CA1F8EE03641C29985A
:10C5C000864238BF262CB5D3002211461046F5F717
:10C5D000C1F96D1C022D8BD31E992098F4F711F927
:10C5E0001C992198F4F70DF90021089A2098F4F786
:10C5F00049FF0121099A2098F4F744FF00210A9A83
:10C600002198F4F73FFF01210B9A2198F4F73AFFA4
:10C6100002202799F4F758FE02202599F4F79FFE8F
:10C6200002201B99F5F756F91A992098F4F7CBFEDA
:10C6300018992198F4F7C7FE02202699F4F75FFFB6
:10C6400012201F99F4F75BFF02202499F4F797FF5B
:10C6500012201D99F4F793FF0E980090069B049A00
:10C6600002992098F5F767F80F980090079B059AB4
:10C6700003992198F5F75FF822992098F5F7B9F812
:10C6800001992198F5F7B5F802202399F5F754F9A7
:10C690001998F5F76CFA2BB0BDE8F08FFFE7F8F7C3
:10C6A00005FE79E72DE9F04FADF6844DFF224FF4FA
:10C6B000056168460FF02EFEFF224FF484610DF5F0
:10C6C00005600FF027FECDF850D86846FEF7ACFCA9
:10C6D000FE4C208810F4804F15D00025FF224FF427
:10C6E000006114A804950FF015FEADF82450ADF8C4
:10C6F00026500B950A950D950C950E950F95119555
:10C70000109513951295DDF85018DDF85008DDF8F6
:10C71000503891F8211090F82000503301FB00FCB4
:10C7200003EB4C030DF505624FF0000C002909D90D
:10C7300002EB4C0633F8025B0CF1010CA6F8EA5050
:10C740006145F5D84FF0000C002809D902EB4C06E2
:10C7500033F8025B0CF1010CA6F812516045F5D8D4
:10C7600015684FF0000C95F82250002D0CD902EB03
:10C770004C0633F8025BA6F8BE5315680CF1010CA9
:10C7800095F822506545F2D815684FF0000C95F8E1
:10C790002350002D0CD902EB4C0633F8025BA6F8AF
:10C7A000CE5315680CF1010C95F823506545F2D86D
:10C7B0004FF0000C002909D902EB4C0633F8025B5C
:10C7C0000CF1010CA6F870506145F5D84FF0000C43
:10C7D000002809D902EB4C0633F8025B0CF1010C7E
:10C7E000A6F898506045F5D833F802CBA2F8E6C019
:10C7F00033F802CBA2F8E8C033F802CBA2F8E4C0C9
:10C8000000254FF0000C00290FD905EB450606EB7B
:10C81000051602EB860606EB4C0833F8027B0CF19A
:10C82000010CA8F85E718C45F5D34FF0000C002880
:10C830000FD905EB450606EB051602EB860606EB5F
:10C840004C0833F8027B0CF1010CA8F88E72844579
:10C85000F5D36D1C042DD4D3002516684FF0000CC1
:10C8600096F82260002E88BF02EB05160CD906EB65
:10C870004C0833F8027BA8F8DE7317680CF1010C42
:10C8800097F822706745F2D816684FF0000C96F8BA
:10C890002360002E88BF02EB05160CD906EB4C086E
:10C8A00033F8027BA8F8FE7317680CF1010C97F8B7
:10C8B00023706745F2D86D1C022DCED3FEF70AFD1A
:10C8C00082480125046814F4004F7DD10746804852
:10C8D0000DF505660025006890F8B40000F00F081B
:10C8E00000F0FDFD012809D00F214046F8F788FD32
:10C8F000012812D0002000F0EFFDB2E00021084630
:10C90000F5F758F9F4F74FFA50B17248D0F84013E0
:10C9100041F48031C0F8401302E0012000F0DCFD5A
:10C920006D4890F800806D4890F80090B9F1000FC4
:10C9300018BFB8F1000F7CD0DDF85058002085F802
:10C94000208085F8219085F8220085F82300F5F7EE
:10C9500058FEF5F72AFA0023824614F0030F18BF99
:10C960004FF4817314F0200F1CBF40F201200343E9
:10C9700014F0100F1EBF387810F0210F43F48463B9
:10C9800063B10AEA0300F5F7F2F8FF210F20F8F788
:10C99000E2FEF5F743F85046F5F7E9F814F0100F0A
:10C9A00009D04F493246087885F82200497885F841
:10C9B0002310FFF71CFC14F02C0F04D0324649461C
:10C9C0004046FFF7A5F800E04BE014F0030F45D018
:10C9D000DDF850B8CDF8706C0BF15005F5F7B4FAEE
:10C9E0008246F5F71BF80020F5F7CCFD0026B9F1DB
:10C9F000000F25D906EB4600002400EB061716E0D1
:10CA00001AF90400262811D2C107890C00EBD07056
:10CA100001EB8701401001EB800000F1405000F570
:10CA200000400068F5F7B4FD25F8020B641C44458E
:10CA300000E014E038BF262CE2D3761C4E45D9D353
:10CA4000284800781D2804BF0BF15000FCF783FE36
:10CA500049464046DDF8702CFEF73CFC0125F5F711
:10CA600065F99DF82000CDF8740C9DF82100CDF8F3
:10CA7000780C002D1FBFDDF8740C0028DDF8780C51
:10CA8000002804BF0DF6844DBDE8F08F0F48006804
:10CA9000CDF87C0C10F0020F00F01A81DDF8504840
:10CAA000DDF8786CDDF8741C206947F6FF7920F01A
:10CAB0000F00206100200DF5056504F150076FEAB5
:10CAC0000908CDF86008CDF85C080DE0DC850010A1
:10CAD000D485001000500040CC840010CD8400109C
:10CAE000D48400103D850010CDF858088246CDF85A
:10CAF0005408002E4ED90AFB01F04FF0010C37F913
:10CB00001020002093465B46CDF8700C01291BD9FC
:10CB10000AFB01C037F910009042C8BF0246984294
:10CB2000B8BF0346B0EB0B0E48BFABEB000E0FFADD
:10CB30008EFBDDF870ECF345C8BFCDF870BC8346C2
:10CB40000CF1010C8C45E3D34245C8BF90464B45E0
:10CB5000B8BF9946D01A48BF981A02B2FE4800687A
:10CB6000B0F9C030934205DBB0F9C220DDF8700C9B
:10CB700090420BDD4FEA5A1005EB80000AF01F0CC3
:10CB80000122C36802FA0CF21A43C2600AF1010AD8
:10CB9000B245B0D34FF0000A00294CD937F91A201A
:10CBA000002093465B464FF0010CCDF8700C012E2F
:10CBB0001BD90CFB01A037F910009042C8BF0246F8
:10CBC0009842B8BF0346B0EB0B0E48BFABEB000E6C
:10CBD0000FFA8EFBDDF870ECF345C8BFCDF870BCE2
:10CBE00083460CF1010CB445E3D34245C8BF9046DF
:10CBF0004B45B8BF9946D01A48BF981A02B2D648DA
:10CC00000068B0F9BC30934205DBB0F9BE20DDF816
:10CC1000700C90420BDD4FEA5A1005EB80000AF0D1
:10CC20001F0C0122436802FA0CF21A4342600AF117
:10CC3000010A8A45B2D3E868002804BF28690028A1
:10CC400003D0206940F0080020616868002804BF14
:10CC5000A868002803D0206940F0040020616968BA
:10CC6000E868B1400843A062A9682869B14001435F
:10CC7000E1626868202E39BFC6F12002D040A6F1DB
:10CC8000200290400843E062A4F82490A4F8268093
:10CC9000B5F9E410B8EB010048BFA1EB0800AE49BC
:10CCA0000968B1F9B820904203DD206940F0020024
:10CCB0002061B5F9E420B2EB090048BFA9EB0200FE
:10CCC000B1F9BA10884203DD206940F0010020610B
:10CCD000DDF87C0CA14D10F0050F07D00DF50562B5
:10CCE000DDF8781CDDF8740CFEF735FCD5F8008013
:10CCF00018F0080F7CD0DDF85028DDF8783CDDF81E
:10CD0000749C11694FF0000A21F4C05111610DF5B6
:10CD10000560CDF8B0A85146CDF8ACA8002B84BF73
:10CD2000DFF834B2012418D9DBF8006000EB410CC5
:10CD3000BCF942C2B6F9266166450BDA4E0900EB32
:10CD4000860C01F01F07DCF85C6004FA07F73E432D
:10CD5000CCF85C60491C9942E6D3C0F858A0002189
:10CD6000C0F854A0B9F1000F84BF7B4C012618D93C
:10CD7000276800EB410CBCF972C3B7F9267167450F
:10CD80000CDA4F0900EB870C01F01F0ADCF8547035
:10CD900006FA0AFA47EA0A07CCF85470491C4945D2
:10CDA000E6D3916BD0F85CC041EA0C01D0F854C0D6
:10CDB0000CFA03FC41EA0C019163D16BD0F860C01E
:10CDC00041EA0C01D0F858C00CFA03FC41EA0C0C03
:10CDD000C2F83CC0416D202B39BFC3F12003D940BC
:10CDE000203B994041EA0C01D163416D002900E0EC
:10CDF00011E004BF816D002903D0116941F4006185
:10CE00001161C16D002904BF006E002803D01069B4
:10CE100040F48050106118F0100F18BF18F0050F83
:10CE200007D09DF823109DF822000DF5056200F053
:10CE300080F9287810F0400F2FD10598401C0590FC
:10CE40000498002814BF0798069800F1010014BF49
:10CE5000079006900DF50560FEF76DF9002002467B
:10CE60000390029869468C46B0F5056F94BF03465F
:10CE70004FF405630020B0EB930F06D25CF820401E
:10CE8000401C2244B0EB930FF8D35042C8604FF4DB
:10CE900040304FF40562F5F71BFF41208DF8700C10
:10CEA0009DF810008DF8710C9DF811008DF8720C32
:10CEB0009DF812008DF8730C9DF813008DF8740C1A
:10CEC000002305220DF54761072000F087FA0DF6D3
:10CED000844DBDE8F08F70B505460024F4F7B2FF2D
:10CEE000FCF793F8012804D02846F5F7ADF920B1F6
:10CEF0000124F4F793FD204670BDF8F7D7F9EFE76A
:10CF00002DE9F74F84B04FF00008C2F82080C2F836
:10CF10001C80059B104E01274146002B23D902EBB4
:10CF20004103B3F97030002BB8BF5B421BB2D6F897
:10CF300000C0BCF9CCC09C450CDD4B0902EB83035F
:10CF400001F01F04D3F81CC007FA04F44CEA040CE7
:10CF5000C3F81CC0491C03E0D4850010DC85001018
:10CF6000059B9942DBD30021012B1CBF059BA3F13C
:10CF7000010940D002EB4103B3F97240B3F970C02C
:10CF8000B4EB0C0348BFACEB04031BB23568B5F936
:10CF9000C6509D422CDAB2F9E630BCEB030548BF1F
:10CFA000A3EB0C052DB2B4EB030C48BFA3EB040CB0
:10CFB0000FFA8CF39D420DDB4B0902EB830301F06A
:10CFC0001F04D3F81CC007FA04F44CEA040CC3F89D
:10CFD0001CC00DE04B1C4FEA531C02EB8C0C03F001
:10CFE0001F03DCF81C4007FA03F32343CCF81C3082
:10CFF000491C4945BED3316891F8CA30002B7DD019
:10D0000091F8CB1014688B4288BF19460023DDF8D5
:10D0100014C0BCF1000F84BF491C00916ED94FF0C1
:10D02000010EDDF800C04FF000090121CA46BCF135
:10D03000010F52D9DFF828C303FB0005DCF800C05C
:10D04000CDF80CC0BCF9CEC002950EFB00050195D1
:10D0500003FB001504EB4505B5F95080B8F1000F4E
:10D06000B4BFC8F100054546AC4536DB0EFB0015E4
:10D0700004EB4505B5F95070002FB4BF7D423D4625
:10D08000AC452ADB029D6D1A04EB4505B5F94E60EF
:10D09000002EB4BF75423546AC451EDB019D6D1AAE
:10D0A00004EB4505B5F94E50002DB4BFC5F1000B9A
:10D0B000AB46E34511DCA7EB0808039FB7F9C8703E
:10D0C0004745B8BF09F10109AD1BBD42C8BF0AF110
:10D0D000010A491C009DA942BAD3BAEB090148BF15
:10D0E000A9EB0A01DFF878C2DCF800C09CF8CAC0DE
:10D0F00061450FDB590902EB810100E015E003F007
:10D100001F064FF0010CCD690CFA06FC45EA0C0C29
:10D11000C1F81CC005995B1C8B4206D2002B18BFBE
:10D12000A3F1010E7FF47DAF79E707B00120BDE8E0
:10D13000F08F2DE9F04FD2F800C083B04FF0010816
:10D14000DCF8103023F4E023CCF81030854BD3F812
:10D1500000E0834B1EF0010F1B6827D000245466AB
:10D1600025462746CDE900015DF827B00024BBF134
:10D17000000F88BF02EB071A15D90AEB4406B3F972
:10D18000D490B6F9BE63B14503DCB3F9D690B1458E
:10D1900005DA566E08FA05F946EA09065666641C71
:10D1A0006D1CA345E9D87F1C022FDDD31EF0040FB0
:10D1B00071D00024946625462746CDE900015DF82C
:10D1C00027A00024BAF1000F88BF02EB471915D938
:10D1D00009EB4406B3F9D8B0B6F9DE63B34503DC16
:10D1E000B3F9DAB0B34505DA966E08FA05FB46EAFC
:10D1F0000B069666641C6D1CA245E9D87F1C022FA5
:10D20000DDD30024D46625462746CDE900015DF82C
:10D2100027A00024BAF1000F88BF02EB471915D9E7
:10D2200009EB4406B3F9DCB0B6F9EE63B34503DCB1
:10D23000B3F9DEB0B34505DAD66E08FA05FB46EA67
:10D240000B06D666641C6D1CA245E9D87F1C022F14
:10D25000DDD34418D2E91A5030EA050343EA050643
:10D26000D36612D000210846002C0ED908FA00F728
:10D270003B4218BF491C401CA042F7D3012904D1EE
:10D2800045EA030090660020D0661EF0010F02D030
:10D29000506EB04350669CF820009CF821101EF0A0
:10D2A000010F08441CBF516E00291AD0DCF8101081
:10D2B00041F48031CCF81010536EDCF8301083400C
:10D2C0001943CCF83010516E202839BFC0F120032B
:10D2D000D940A0F120039940DCF834301943CCF850
:10D2E0003410916ED1B1DCF8101041F40031CCF85B
:10D2F0001010936EDCF8381083401943CCF83810C6
:10D30000916E202827BFA0F120039940C0F120038F
:10D31000D940DCF83C301943CCF83C10D16ED9B17F
:10D32000DCF8101041F48021CCF81010D36EDCF83A
:10D33000401083401943CCF84010D16E202827BFFD
:10D34000203801FA00F0C0F1200021FA00F0DCF8EA
:10D3500044100843CCF8440003B00120BDE8F08F2E
:10D36000D4850010DC85001070474FF0FF30704707
:10D3700055484068704754494860704710B582B0BE
:10D3800007280BD14FEA111C012404FA0CFC4E4C67
:10D3900064681CEA040F04BF02B010BD9B0100F0DA
:10D3A0000F0043EA800040F001008DF800008DF886
:10D3B00001108DF80220100A8DF80300100C8DF872
:10D3C0000400100E8DF8050000208DF806008DF881
:10D3D000070068460FF00CF802B010BD10B59B01B5
:10D3E00000F00F0082B043EA800040F001008DF8A9
:10D3F0000000072A88BF072200206B46002A09D9AF
:10D4000011F800C01C18401C84F801C09042F7D3EA
:10D41000072805D200211A18401C51700728FAD39A
:10D4200018460EF0E5FF02B010BD10B59B0100F0EC
:10D430000F0082B043EA800040F002008DF8000047
:10D44000072A88BF072200206B46002A09D911F855
:10D4500000C01C18401C84F801C09042F7D3072874
:10D4600005D200211A18401C51700728FAD318461B
:10D470000EF0BEFF02B010BD70B5134E40EA01259C
:10D4800002283488224618BF052803D1002918BF76
:10D49000022900D12C46A24209D051B17088002344
:10D4A00044EA004290210720FFF768FF348075802E
:10D4B00070BDF6F706F844EA0042002390210720E9
:10D4C000FFF75CFFF2E70000E0850010FE490870FE
:10D4D0007047FD4800787047FB4948707047FA482C
:10D4E000407870472DE9F04FF848F74E95B0006846
:10D4F0007178836D0229C3F303201AD0726812F485
:10D50000007F1EBFC3F303310F29084612F0800FBE
:10D510001EBFC3F303110F29084602F00701F7F7F6
:10D520006FFF012814BF00200220707040F0468277
:10D530000DE000210846F4F73DFBF3F734FC30B171
:10D54000E348D0F8401341F48031C0F84013F4F7B9
:10D550002CFC1090307910F0100F18BFF5F730F850
:10D56000307910F0080F03D1FF210F20F8F7F3F8FE
:10D57000D848DC4900780590D74800781190D74802
:10D580000478D74805780878009048780190119879
:10D5900000281CBF0598002816D00EF006FF0EF0DC
:10D5A00009FF0020F7F7B6F80020F7F7ECF80020A5
:10D5B000F7F708F9C448007910F0100F0AD00120DD
:10D5C000F7F712F9012009E0002D18BF002CE4D173
:10D5D00000F0F4B90020F7F707F90020F7F704F995
:10D5E000F3F7E1FB10F0010F04BF0120F3F74DFE4C
:10D5F000F4F7EFFB1E20FCF706F800210846FBF7C6
:10D6000081FF834601210020FBF77CFF119A0599D9
:10D610008246002001FB02F6002E84BFB2494A0C6C
:10D6200006D92BF810102AF81020401C8642F8D892
:10D630001E20FCF781F900210120FBF763FF012187
:10D6400012900846FBF75EFF8146002065191CBF5B
:10D65000A54A510C07D0129B23F8102029F810106E
:10D66000401C8542F7D81E20FCF780FA00210220DA
:10D67000FBF748FF804601210220FBF743FFDDE96D
:10D680000012074600208C181CBF97494A0C06D090
:10D6900028F8101027F81020401C8442F8D80020E9
:10D6A000139089484088002840F2DA80601C4008C6
:10D6B000691C0C9048080E90FBF7A7FC012800F0AD
:10D6C000CF8006A8F4F7C0FD00287CD00798F6F7B5
:10D6D000CAFA0898002845D07B48007910F0100F4E
:10D6E00008D0089801900EF088FE01990EF08AFE8D
:10D6F000019015E000200023019002900390049017
:10D7000000901A46194608980EF081FE01906E4866
:10D71000007910F0200F03D00EF06FFE01900AE0A8
:10D72000F6F711FB119A0092019A01461046059BEB
:10D730000EF072FE019800281CBF0020002E11D9A7
:10D7400001993BF9102031F910108A42B8BF2BF82B
:10D7500010103AF910208A42C8BF2AF81010401C55
:10D760008642EDD8109810F0010F1CBF0A980028CF
:10D7700033D05548007910F0400F0A9809D00023A3
:10D780001A4619460EF04DFE0EF050FE0F9020B3D3
:10D790000AE00F90F6F7A0FA02220092DDE90E32BD
:10D7A000014610460EF038FE0020002D15D90F99C5
:10D7B000129A31F9101032F910208A42BCBF129A25
:10D7C00022F8101000E043E039F910208A42C8BF67
:10D7D00029F81010401C8542E9D8109810F0200F4D
:10D7E0001CBF0B9800282DD03748808810F4807F0C
:10D7F0000B9807D000210EF01EFE0EF021FE0D90BA
:10D8000000B30AE00D90F6F74DFA02220092DDE92E
:10D810000C32014610460EF0FFFD0020002C11D9FD
:10D820000D9938F9102031F910108A42B8BF28F844
:10D83000101037F910208A42C8BF27F81010401C7A
:10D840008442EDD8F4F75DFD1398401C139002E07C
:10D85000F7F72CFD13981C4949888842FFF42CAF38
:10D86000F4F7DCF80EF0A6FD0EF0A9FD16491398AA
:10D87000498888427DD3109810F0020F3AD00022D8
:10D880004FF6FF731046002E0ED93BF910103AF9EF
:10D8900010C0A1EB0C019142C8BF0A469942B8BF23
:10D8A0000B46401C8642F0D842208DF80000100A3A
:10D8B0008DF80100180A8DF802208DF8043000233D
:10D8C0008DF80300052211E0E8850010D4850010D2
:10D8D00000500040CC840010CD840010D184001092
:10D8E000D2840010D48400100080FFFF6946072016
:10D8F000FFF774FD109810F0010F28D000224FF6AA
:10D90000FF731046002D0FD9129939F910C031F963
:10D910001010A1EB0C019142C8BF0A469942B8BF52
:10D920000B46401C8542EFD843208DF80000100ABA
:10D930008DF801008DF80220180A8DF803008DF88B
:10D9400004300023052269460720FFF747FD1098A1
:10D9500010F0200F29D000224FF6FF731046002C44
:10D9600010D938F9101037F910C0A1EB0C01914211
:10D9700000E01AE0C8BF0A469942B8BF0B46401CF7
:10D980008442EED844208DF80000100A8DF8010082
:10D990008DF80220180A8DF803008DF8043000235A
:10D9A000052269460720FFF719FDFF20FBF72BFE34
:10D9B000FF20FBF7C1FFFF20FCF7D8F8F4F7B6F91A
:10D9C00015B0BDE8F08F70B5224C00206070F4F700
:10D9D000B3FAF4F786FA05460020F4F77CFAFBF771
:10D9E00014FB012803D1F7F709FC03281BD1207889
:10D9F00010F0010F07D0FEF755FE207820F001004F
:10DA00002070FBF7BBFA207810F0020F07D0FFF769
:10DA100069FD207820F002002070FBF7AFFAF7F7DD
:10DA2000EDFB032807D02846F4F755FABDE870400F
:10DA30000120F4F781BAF7F739FCD0E705494860CF
:10DA4000002048707047034840687047014948808B
:10DA500070470000E8850010FE4908707047FD48D7
:10DA600000787047FB48007A7047FA48002101723D
:10DA7000C1717047F74948727047F648407A70475D
:10DA8000F448808BC0F300207047F24910B5898BB1
:10DA90000020C1F3002151B106F0CEF864280FBF79
:10DAA0004FF0C040012101FA00F040F08040BDE895
:10DAB000104006F0C4B8E74A10B5C0F3074381B27E
:10DAC0005361D161C0F30360507090700020C1F3C6
:10DAD0000021906151B106F0AFF864280FBF4FF0FC
:10DAE000C040012101FA00F040F08040BDE8104044
:10DAF00006F0A5B8D74840797047D64A0028D169C2
:10DB000014BF41F0020021F00200D0617047D148FB
:10DB1000007FC0F340007047CE4A10F0010FD0697B
:10DB200014BF40F0020020F00200D0617047C949E4
:10DB30000020097FC1F34001002918BF0120704770
:10DB40000028C44AD16914BF41F0010021F001004E
:10DB5000D0617047BF48007F00F001007047BD49A9
:10DB60004A788A7048707047BA4840787047B94818
:10DB700080787047B8480068406DC0F30360704714
:10DB800001218140B3484269114041617047012140
:10DB90008140B048426922EA010141617047AD48C5
:10DBA00040697047AB4880697047AA4910B58C69D5
:10DBB00088610246002381210720FFF7DFFB204612
:10DBC00010BDA448808BC0F380207047A14901207C
:10DBD000486270479F49C872704710B59D4C60B944
:10DBE00006F035F808281CBFE07A022805D001208D
:10DBF000E072F4F76DF9206210BD0020E07210BDF4
:10DC00002DE9F041934D0024E87A012802D0204606
:10DC1000BDE8F081F7F7F2FA8046F7F7F5FA00264B
:10DC20000746B8F1020F1CBF0124EE72EFD1F4F7E2
:10DC30004FF90146286A88429CBF081AB0F5966FD2
:10DC4000E5D30124022F14BFEE720024DFE78148E0
:10DC5000C07A012818BF002070477E48007FC0F3BB
:10DC6000800070477B48007FC0F3C0007047794850
:10DC7000808BC0F3402070477648007FC0F3C0100F
:10DC80007047FCF7BFBC7348818B11F4005F04D16F
:10DC9000C07A01281CBF00207047012070476D48E2
:10DCA000808BC0F3C02070476A48808BC0F300307F
:10DCB000704770B5674E0546C0F34020F469C4F361
:10DCC000403188420CD0F0B905F0C1FF08281CBFD4
:10DCD000F07A022817D00120F072F4F7F9F83062D8
:10DCE00015F4807F14BF44F4806124F4806115F43E
:10DCF000007F14BF41F4005021F40050F061BDE8F2
:10DD00007040FCF764BE0020F072E9E770B551493D
:10DD1000044610F0040FCD69284614BF40F480700B
:10DD200020F4807014F0080F14BF40F4007020F449
:10DD3000007014F0100F14BF40F4006020F4006075
:10DD400014F0400F14BF40F4805020F4805014F0C1
:10DD5000200F14BF40F0800020F08000C861002137
:10DD6000C0F3002050B105F067FF64280FBF4FF0EB
:10DD7000C041012101FA00F040F08041084605F061
:10DD80005EFFC4F38000C5F30021884208BF70BD68
:10DD90000120F6F72EFC05F0F4FE10F4817F0CBF95
:10DDA00001200020F4F797F805F0EBFE10F0020FC9
:10DDB00004D0BDE87040002002F06FBF274890F803
:10DDC0006C00BDE87040C00802F067BF2148C1691F
:10DDD000002011F0040F18BF012011F0080F18BF28
:10DDE00040F0020011F4807F18BF40F0040011F4ED
:10DDF000007F18BF40F0080011F4006F18BF40F01A
:10DE0000100011F4805F18BF40F0400011F0800F47
:10DE100018BF40F0200070470E48006B70470D4956
:10DE20008A6A10438862704770B50A4EB06A40F43F
:10DE300000640020B062F56915F0040F18BF44F0CB
:10DE4000010415F0080F18BF44F0020415F4807F98
:10DE500006E00000F0850010D4850010E8FC0010FA
:10DE600018BF44F0040415F4007F18BF44F0080400
:10DE7000FCF7C8FB002818BF44F4807415F4006F49
:10DE800018BF44F0100415F0800F18BF44F02004B0
:10DE900015F4805F18BF44F0400415F4005F02D110
:10DEA000F07A012801D144F40074B16944EA0140D8
:10DEB000002918BF40F4805070BDF749C862704710
:10DEC000F54890F82C0000F001007047F24890F8F7
:10DED0002C00C0F340007047EF4890F82C00C0F3CE
:10DEE00080007047002818BF0120EB494873704735
:10DEF0002DE9F047002586B02E46F7F77FF9E74970
:10DF0000052808680CBF90F8F80090F8580000F059
:10DF10000F094846FCF734FEDF4F4FF0000A4FF080
:10DF20000108002808BF54460FD0446A05F029FEB6
:10DF300010F4C06F08BF87F80CA006D014F0020FD1
:10DF400018BF24F0010487F80C8014F0010F14BFEF
:10DF50000224042444F400314846F7F751FA00281B
:10DF600004BF06B0BDE8F08714F0040FCC4C07D016
:10DF7000F2F741FC01462078814288BFF2F733FC7A
:10DF80000120F3F782F9F3F75DFFFBF73EF8012874
:10DF90003BD06846F4F758F9002832D06846FBF7C2
:10DFA00007FF0198F5F75FFE029880B1BD48217820
:10DFB0000078400000FB01F2BB4802990EF087F99F
:10DFC000BA480078492804BFB748FBF7C4FB049857
:10DFD00088B1B748B749049C0078097842185200C4
:10DFE0002146B5480EF073F9B44A1278492A04BFA5
:10DFF0002046FBF7BBFC87F80D80F4F782F9012679
:10E0000003E0F7F753F9002DBFD0F3F707FDF7F75B
:10E0100066FB06B03046BDE8F0879F48407B00288D
:10E0200018BF012070472DE9F04F4FF0000A87B06C
:10E030000446D146F7F7E2F80746F7F7E5F8DFF8C8
:10E0400058B20690052F07D1FCF7D0F8002804BF7E
:10E0500000208BF80D0002D09BF80D0008B9FFF7E7
:10E0600047FF052F0CBFDFF85882DFF858820F21D9
:10E070002046F7F7C5F9002804BF07B0BDE8F08FC8
:10E080000EF093F9F6F754FA04007DD10125F2F76A
:10E090008AFE06460020F3F7F8F82846F3F7B2FEAA
:10E0A0007D480564F5F710FAA5F1010BFAF7ADFF0D
:10E0B00001280AD0F7F7A2F8B84206D1F7F7A4F87A
:10E0C0000699884208BF002C09D0F3F7A7FC724FCD
:10E0D00016F0010F7D7834D0012C27D031E068464E
:10E0E000F4F7B2F8F8B116F0010F03D00120F5F7FC
:10E0F0002FFC82466846FBF75BFE0198F5F7B3FDFF
:10E100006846C0470446F4F7FCF8002CCED115B998
:10E1100001985845CAD1F3F77FFC002804BF284670
:10E12000F3F770FEC2E7F7F7B6F8BFE70120F5F79F
:10E130000FFC504505D2AAEB00010120F5F718FCB1
:10E140008146F5F7E6F916F0010F29D0012C27D109
:10E15000B9F1000F24D0F2F7DFFF0446F2F734FEE6
:10E1600000EB800004EB40004844002144F2090227
:10E17000904284BFA0F580400938002D08BF43F6C7
:10E18000390105D0022D00E00AE008BF41F6F9018F
:10E19000884205D2091A0120F5F719FC0120B8724E
:10E1A0000EF00DF9F7F79BFA07B0BDE8F08F2DE9F7
:10E1B000F14F88B000260396049606960296F7F76C
:10E1C0001DF801903748B046C146047834482346CC
:10E1D00035490578089804FB05FA00EB4A07024622
:10E1E000009538460EF018F9DFF8C0B09BF8000033
:10E1F000492804BF2C48FBF7AEFA2C4800784C287D
:10E2000004BF3846FBF7A7FA07EB4A0293464FF0E4
:10E21000000C002D25D90020611E13D007EB410E04
:10E2200037F811303EF802ECA3EB0E031BB2002BC3
:10E23000B8BF5B421BB222F811308342C8BF1846F8
:10E24000491EEBD10199022919D0108007EB440730
:10E2500002EB44024045C8BF80460CF1010CAC45BE
:10E26000D9D30D48B0F9100005908045A4BF012610
:10E270000396002E04BF019802285ED124E002EB31
:10E28000440131F9023C142BB9BF31F9041C1429A3
:10E2900001260396D9E70000F0850010D485001010
:10E2A000CD840010CC840010800001103D8500104A
:10E2B000D2840010D1840010700601104285001035
:10E2C000A531001019360010FA48007B00281CBF49
:10E2D0000022002D88BF6B462FD902FB04F00BEB08
:10E2E0004000018EADF80010818EADF80210018F54
:10E2F000ADF80410B0F93C70ADF80670002003EBE7
:10E30000400C33F81010BCF802C06144DDF814C0B2
:10E3100009B2614503DB0126884602960AE0401CEB
:10E320000328ECDB36B9142F04DB0126BDF9068087
:10E33000029602E0521CAA42CFD30BEB4A034FF0E5
:10E34000000C002D25D90021601E022812D90BEBEC
:10E3500040023BF8107032F802EC32F8042C77449B
:10E360003A4412B223F810208A42C8BF1146401E18
:10E370000228ECD800201980588098800BEB440BC1
:10E3800003EB44034945C8BF89460CF1010CAC4579
:10E39000D9D3C84BB3F912209145A4BF01260496E6
:10E3A000002E14BF986CD86C00F1010014BF986463
:10E3B000D864C1480078FF2842D008980127002E71
:10E3C00020F83A600898039900EBCA00418004994C
:10E3D00081800299C18006990181996C4FEAE17CA4
:10E3E00001EB1C5C6FF30B0CA1EB0C014181D96CB0
:10E3F0004FEAE17C01EB1C5C6FF30B0CA1EB0C0111
:10E400008181A0F80E80A0F81090197B41820599B7
:10E410008182C2824FF00208089907EB85032246E9
:10E42000CDF800800CBF4E204D20FBF736F907EBEE
:10E4300085032246CDF8008047200899FBF72DF987
:10E4400009B03046BDE8F08F9C4870472DE9F84F81
:10E45000834698489C490025B0F91080994809786E
:10E460002E460078964CAA464718F3F79EFC00907B
:10E470009648A4F174090078492804BF4846FBF780
:10E4800075FA0020002F09D93BF8101039F8102038
:10E49000891A24F81010401C8742F5D8DFF82C9216
:10E4A00099F800004C2804BF2046FBF75FFA00985B
:10E4B00010F4007FA7F1010012D000281CBF7D4995
:10E4C000B1F9123026D034F910100029B4BF4A42F5
:10E4D0000A469A42BCBF0D44761C401EF3D119E097
:10E4E00000281CBF7349B1F9123013D004EB40026D
:10E4F00034F8101032F8022C891A09B224F81010DE
:10E500000029B4BF4A420A469A42BCBF0D44761C59
:10E51000401EEBD1002EC8BF95FBF6F52EB226802B
:10E5200099F800004F2804BF2046FBF71FFA00258A
:10E53000781E0ED034F81010891B09B224F8101080
:10E540000029B8BF494209B28D42B8BF0D46401EEE
:10E55000F0D1258005F015FB10F4817F18BF4FF036
:10E560000508454506DD99F800004FF0010A4D28E1
:10E5700007D103E099F800004E2802D12046FBF7AE
:10E58000F5F999F80000472804BF2046FBF7EEF99B
:10E590005046BDE8F88F2DE9F04F87B0FBF7EEFF4E
:10E5A0004B4D2868B0F93610B0F934000DF0DFFE9D
:10E5B0000120F6F71EF805F0E4FA10F4817F14BF8D
:10E5C00000200120F3F787FC3A4C207D10F0100F5B
:10E5D00006D0042000F018F90F2818BFF5F7EDFF5A
:10E5E000FF20A07108F0B4FDF6F708FE022840F005
:10E5F000FD80DFF8E0B0A1464FF0000A99F8016015
:10E600003348C9F838A0C9F83CA00068B100806D53
:10E6100020FA01F101F00F04C0F30328C0F3033521
:10E62000C0F30317444536D10F2D34D0B9F81C0080
:10E6300010F4005F03D199F80B00012803D105F015
:10E6400006FB082808D105F09CFA10F4817F03D15D
:10E6500005F009FB022800D12C46D9F85000A04251
:10E6600019D005F0F4FAAC420CBF0121002141EAB7
:10E67000002505F0E1FA45EA004505F0F4FA45EA1F
:10E680000062002384210720FEF778FE0020C9F8ED
:10E690005040F5F7AEFFF6F791FE20B1444502D1A8
:10E6A0000F2F18BF3C4631460220FEF7E5FE052E2F
:10E6B00064D211E0F08500103D8500107006011055
:10E6C000E4060110D2840010D184001042850010AD
:10E6D000D485001088840010DFE806F0740303037B
:10E6E000780099F801600F212046F6F789FE00288E
:10E6F0006FD00DF05AFE0DF05DFEF5F719FF050025
:10E7000036D199F8000000281CBF0001F2F718FD6F
:10E710000024F3F74AFB0690F2F745FB10F0010FD7
:10E720000FD0F2F7ACFD02280BD399F80A0040B1E4
:10E73000069840F40030F3F71AFA0124F3F782FB4D
:10E7400001E0F3F746FB89F80AA089F803A0DFF897
:10E75000BC814FF0E027FAF758FC012808D0F6F703
:10E760004DFD022802BF99F80100B042002D06D0ED
:10E770000DF020FE0DF023FEF6F7B1FF29E068460C
:10E78000F3F762FDD8B12CB1641E0698F3F7EFF9E8
:10E79000F3F71FFB6846FBF70BFB0198F5F763FAED
:10E7A00068460DF052FE054698F8000020B1B869A1
:10E7B000CBF80000C7F810A0F3F7A3FDCBE7F6F7FE
:10E7C00075FDC8E720460DF004FE02E02046FFF785
:10E7D0002AFCFAF71AFC012803D1F6F70FFD0228EC
:10E7E00004D1F6F70BFD02283FF408AF0AF0E6F873
:10E7F000F5F7FEFE07B0BDE8F04FFBF7BFBE4A00DD
:10E80000014643480DF063BD2DE9F04141498000C8
:10E810000968896D21FA00F000F00F04C1F30327A5
:10E82000C1F30335C1F30316BC4239D10F2D37D0E4
:10E83000DFF8E480B8F81C0010F4005F03D198F80A
:10E840000B00012803D105F002FA082808D105F0D1
:10E8500098F910F4817F03D105F005FA022800D160
:10E860002C46D8F85000A0421AD005F0F0F9014625
:10E87000AC420CBF0120002040EA012505F0DCF984
:10E8800045EA004505F0EFF945EA006200238421DE
:10E890000720FEF773FD0020C8F85040F5F7A9FEE9
:10E8A000F6F78CFD20B1BC4202D10F2E18BF3446C2
:10E8B0002046BDE8F08110B58168044679B117485B
:10E8C000174A007812784000424316480DF0FFFCCA
:10E8D00015480078492804BF1248FAF73CFF24691C
:10E8E00084B112480178124800780A185200214673
:10E8F00007480DF0ECFC0F4A1278492A04BF204665
:10E90000FBF734F801200449487310BD208400103F
:10E9100070060110D4850010F0850010CC84001022
:10E92000CD840010800001103D850010D2840010BD
:10E93000D184001042850010404A30B4146894F825
:10E940006CC01CF0040F1ABF012222EA0C050CF067
:10E950000105B0F90030B1F900201DB1E58AAA1A0D
:10E96000521E12B21CF0020F03D0A48AE31A5B1EDF
:10E970001BB21CF0040F19BF02800B8003800A80B9
:10E9800030BC70474FF6FF71A0F8B010A0F8B2107D
:10E99000A0F8B410A0F8B61070472DE9F05F164645
:10E9A0008A46834605F0B8F8074605F0ADF800F151
:10E9B0005009002E18BF002588BF4FF6FF780FD0F2
:10E9C00098BFBDE8F09FC5EB051007EB001494F865
:10E9D000E000012804BF94F89300002812D103E05E
:10E9E000BDE8F05F02F0C2B8A4F8B080A4F8B2802D
:10E9F000A4F8B480A4F8B68023464A465146584647
:10EA000002F0F6FD94F8ED00022812BF032894F8F6
:10EA1000930000280DD0B4F8B000A4F8B400B4F806
:10EA2000B200A4F8B600681CC5B2B542CBD3BDE8AD
:10EA3000F09F204601F0CBFEF5E70000F0860010C5
:10EA4000FE484078002818BF01207047FC48006845
:10EA500090F8700000F001007047F94909680A6FEA
:10EA600060F300020A6770472DE9F001F4491025B0
:10EA700040268024F14A09684FF0200C670010B34B
:10EA800001284ED002281CBFBDE8F0017047488A1B
:10EA9000322300FB03F84B8BB8FBF3F808FB08F8B4
:10EAA000C2F8108000EB001808EB4010B0FBF3F048
:10EAB00040435061486F000F062821D2DFE800F084
:10EAC000201C2025292D488A4B8B4FEA0018C000B6
:10EAD000B8FBF3F8B0FBF3F008FB08F84043C2E9D9
:10EAE0000480B1F87400C0F30330062808D2DFE8D0
:10EAF00000F00703070C10145580BDE8F0017047C3
:10EB0000A2F802C0BDE8F00170475680BDE8F001F0
:10EB100070475480BDE8F00170475780BDE8F001B0
:10EB20007047488A498BC0EB00135B00B3FBF1F3DD
:10EB30005B43136100EB4003C3EB4010B0FBF1F00B
:10EB4000404350615480BDE8F001704710B5BC48A7
:10EB5000BA4C006890F87C20418A408B4A43B2FB53
:10EB6000F0F201EB81014900B1FBF0F04043E260BB
:10EB7000A0610020FFF778FF04F120014FF6FF703D
:10EB800008804880091F4FF0FF300880488000202F
:10EB9000207010BD2DE9F04F8DB01F46DDE91686BF
:10EBA0000D46044604F0B0FF029004F0C9FF0B903C
:10EBB000A2484FF4A051A24AB0F802A0CDF8288094
:10EBC00001910169049140690390029890F80C80CA
:10EBD0001068B8F1000F418A26D0408BC900B1FB04
:10EBE000F0F04043089010686421428A438B5143FF
:10EBF000B1FBF3F14943079102EB8201B1FBF3F161
:10EC00004943099194F899C08E491CF801900A3142
:10EC1000B9F1000F10D0B9F1010F11D0B9F1030F04
:10EC200008BF1CF801100FE0408B01EB4101B1FB64
:10EC3000F0F040430890D6E71CF8011021B904E039
:10EC40001CF8011001292FD001210091DFF8F88173
:10EC500094F8ED10A8F10A03A3F10A0902291CBFD8
:10EC600094F8BB10012934D0784901EBCC0252E969
:10EC70000212B5F800C0CDF818C0B5F802C0CDF842
:10EC800014C094F8CCC0BCF1000F57D094F89AC0CF
:10EC9000CCEB0C1BDDF82CC00CEB0B1C9CF8CCC097
:10ECA000BCF1000F39D06CE001210091B8F1000FE8
:10ECB000CCD002EBC20101EB0211B1FBF3F14943ED
:10ECC000049102EB4201C900B1FBF3F14943039106
:10ECD000BCE729886A884FF0000B0CF809B094F85B
:10ECE00099C00CF803B094F899C00CF808B094F8E7
:10ECF00099E0DFF85CB1DDF804C00BEB4E0B2BF8AC
:10ED000002CC94F899C0BCF1010FB2D1DFF82CB15C
:10ED10004FF0000C8BF801C0ABE794F899B0DFF826
:10ED200030C10CEB4B0C3CF802BCB34529D92CF894
:10ED3000026C94F8CCC0BCF1000F22D1DDF81CC0ED
:10ED4000674594F8EDC015D3BCF1020F12D0DDF881
:10ED50001CC0674515D394F899E0DFF8F4B094F837
:10ED6000CCC00BEB4E0B3BF802ECB64588BF2BF842
:10ED7000026C08E04FF4A06B4FF0020CCDF804B029
:10ED800001E094F8CCC0DDF820B05F4538BF4FF00B
:10ED9000020CDFF8A8B09BF801E0BEF1000F01BF44
:10EDA00094F899E0BEF1010F94F8CCE0BEF1030FA6
:10EDB0000DD14FF0010E8BF801E0DFF894B0BBF8F5
:10EDC00000B0B34584BFDFF888B0ABF80060DDF871
:10EDD00010B05F451DD3BCF1020F1CBFDDF800B0C1
:10EDE000BBF1000F15D094F899E04FF0000B0EF82E
:10EDF00003B094F899E00EF808B094F899B01BF8B5
:10EE000009E0BEF1640F3CBF0EF1010E0BF809E002
:10EE100053E0DDF80CB05F4502D2BCF1020F37D1F0
:10EE2000DDF800B0BBF1000F32D0DDF80CB05F456B
:10EE300024BFDDF810B0BB453CD90BE04486001080
:10EE4000F0860010D9070110BB0701105807011008
:10EE5000C6070110BCF1020F51D094F899B01BF80D
:10EE600008E0BEF1000F28D04FF0000E0BF809E0CB
:10EE700094F899B00BF808E094F899B01BF803E007
:10EE8000BEF1640F19D20EF1010E0BF803E014E08D
:10EE900094F899E04FF0000B0EF809B094F899E05F
:10EEA0000EF808B094F899B01BF803E0BEF1640FB7
:10EEB00003D2E8E7BCF1020F21D094F899B01BF817
:10EEC000033093B3DFF8DC9406EB460309EB4B0801
:10EED00038F802BC9B4508D9DDF808B09BF80CB0A7
:10EEE000BBF1000F08BF28F8023C94F8993009EBF9
:10EEF000430838F8023CB34230D365D94DE094F86A
:10EF000099E04FF0000B0EF809B094F899E00EF874
:10EF100003B094F899B01BF808E0BEF1640F3CBF51
:10EF20000EF1010E0BF808E0C7D30BF0FF0313F846
:10EF30000990B9F1000F33D0DFF8689409EB43086A
:10EF400038F8023CB34206D9DDF808B09BF80CB0A3
:10EF5000BBF1000F06D00A9EB3421DD2534428F8DD
:10EF6000023C31E0A3EB0606A3EB66039BB228F854
:10EF7000023C94F899604FEA132309EB46064FF6DA
:10EF8000FF7826F8023C94F8996008EA032309EB1D
:10EF9000460626F8023C17E016D9A3EB0A03DEE783
:10EFA00013F80860012E0FD9FE4EDDF8048006EB41
:10EFB000430636F8023C434588BFA3EB0A0338BF3B
:10EFC000534401D026F8023C94F89930F54E009352
:10EFD00006EB430333F8023C002B08BF00207AD035
:10EFE0001E46B3F5807F3CBF4FF480763346BCF1BC
:10EFF000020F1CBFDDF824C067456DD81F0A029BB5
:10F00000360A93F84230022B1CD3B0F818A0069BA6
:10F01000B0F810900AFB03F3B3FBF9F3B0F81AE071
:10F02000DDF814C0B0F812800AFB01FA0EFB0CFCEC
:10F03000BAFBF9F9BCFBF8FC0EFB02FABAFBF8F8D4
:10F040008B461BE0B0F814A0069BB0F810900AFBAA
:10F0500003F3B3FBF9F3B0F816E0DDF814C0B0F831
:10F0600012800AFB01FA0EFB0CFCBAFBF9F9BCFB9F
:10F07000F8FC0EFB02FABAFBF8F88B46A6F1010A7F
:10F080000AFB0933B3FBF6F6A7F1010303FB08C340
:10F09000B3FBF7FC078A07FB06F308D3078BB0F82E
:10F0A00012A0B3FBF7F30AFB0CF7408B07E0878A4B
:10F0B000B0F812A0B3FBF7F3C08A0AFB0CF7B7FB5A
:10F0C000F0F04E4518BFC44535D14E4508BF5B46EC
:10F0D000C44508BF10462EE0B0F81480078ADDF85A
:10F0E00018C008FB01F108FB0CFCBCFBF7F9B0F8F9
:10F0F00016C0B1FBF7F1408AA6F5807B0BFB01F14E
:10F1000001EB0921DDF814A0B1FBF6F10CFB02F2D2
:10F110000CFB0AFAB2FBF0F2BAFBF0FAA3F5807628
:10F12000724302EB0A22B2FBF3F279435043B1FB84
:10F13000F8F3B0FBFCF09C49009A01EBC20242F8E4
:10F14000083C94F8992001EBC20141F8040CAB8013
:10F15000E8800DB0BDE8F08F2DE9F84F9349944B4E
:10F1600001444FF0000E01F801EC0344012103F8C3
:10F17000011C9049744601EB401100918E49724682
:10F1800001EB401B01F5A07101EB40190098002133
:10F190000BEB041809EB041700EB0416002008EB36
:10F1A000C10307EBC10C06EBC10503EB800A4AF86B
:10F1B000202C0CEB800A4AF8202C05EB800A401C1E
:10F1C00000B24AF8202C0228EFDB481C01B20229C9
:10F1D000E4DB601C04B2022CD8DB7848784E0021B6
:10F1E000D0F800C0A6F110070BEB0E1809EB0E1AB1
:10F1F000002006EBC10908EBC1050AEBC10407EBCF
:10F20000C103814207D1BCF87A2043F82020BCF822
:10F21000782049F8202053F8202005EB800B02EBE2
:10F22000820252004BF8202C04EB800B401C00B2F1
:10F230004BF8202C0228E4DB481C01B20229D7DB62
:10F24000BDE8F88F10B490F899C05E4C00230CF81C
:10F25000043090F899C00A340CF80430574B90F8F9
:10F2600099C01B6893F87430C3F303131B02153461
:10F2700004EB4C0C2CF8023C90F899C0A4F16E03FE
:10F2800003EBCC0C4CF8081C90F8991003EBC1016F
:10F2900041F8042C90F8990010BC5DE710B50446C5
:10F2A00004F04EFC01464848C26894F8ED0002287C
:10F2B00004BFB4F8B410B4F8B60009D094F89A00BA
:10F2C000C0EB001001EB0010B0F8B410B0F8B600BD
:10F2D00094F8CC30022B18BF10BDB4F8B4C0BCEB0E
:10F2E000010348BFA1EB0C03934228BF10BDB4F843
:10F2F000B6C0BCEB000348BFA0EB0C0393423CBF7D
:10F30000A4F8B410A4F8B60010BD2DE9F04F83B0F6
:10F31000044604F015FC2948B4F8B690B4F8B4A03B
:10F320000068DFF8A8B0B0F81880078A468B458AD5
:10F3300009FB06F292FBF5F00AFB08F191FBF7F1ED
:10F3400094F8ED20ABF1200E022A68D09EF800C0A0
:10F35000BCF1000F00F0EF80BCF1020F7ED2BBF8D1
:10F360000020019202FB08F292FBF7F9BBF80220A1
:10F37000009202FB06F292FBF5FAB1EB090348BFDB
:10F38000A9EB0103B0EB0A0248BFAAEB0002142B61
:10F39000B8BF142A7EDADFF838B0BBF900E0AEF56A
:10F3A0007F4B17E0C607011058070110F80C011039
:10F3B000020D0110B80B011038090110F086001081
:10F3C000A0860010A7070110448600106486001074
:10F3D00060860010BBF1FF0B6CD04945FC4981FBF6
:10F3E00003314FEA6103A3EBE1730199D4BFC91A5A
:10F3F0001944F84B5045F648198080FB02104FEA3B
:10F400006001A1EBE0710098CCBF0844401AF149BB
:10F41000488008460188A4F8B410408875E0BBF81D
:10F4200000C00CFB08F292FBF7F7BBF8028008FB68
:10F4300006F292FBF5F5CA1B48BF7A1A431B48BF78
:10F440002B1A142AB8BF142B30DAACF57F46FF3ED6
:10F450002CD0B942DE4981FB022100E034E04FEAC2
:10F460006102A2EBE171D4BFACEB01016144D94A66
:10F47000A842D748118080FB03104FEA6001A1EB3E
:10F48000E070CCBF4044A8EB0000D2494880084659
:10F49000018800E00EE0A4F8B4104088A4F8B6009B
:10F4A00001208EF8000003B0BDE8F08F00208EF838
:10F4B000000040E0C84ABCF1010F04BF02231370F2
:10F4C00003D003B0BDE8F08F2FD1DFF80893B9F96E
:10F4D0000020B9F9023002FB08F2734392FBF7F205
:10F4E00093FBF5F3B1EB020C48BFA2EB010CC11A80
:10F4F00048BF191ABCF1060FB8BF06290ADAB9F8D5
:10F500000000A4F8B400B9F80200A4F8B60003B0F3
:10F51000BDE8F08FB4F8B400A9F80000B4F8B60064
:10F52000A9F8020003B0BDE8F08FBCF1000F1CBFCA
:10F5300003B0BDE8F08FABF800A0ABF8029003B0C9
:10F54000BDE8F08F2DE9F04F90F899C08FB04FF4DF
:10F55000806300290CBFA14CA14C04EB4C14A14DBD
:10F56000029205EB4C1705F5A5756544203C15F88E
:10F57000015C07EB051606EBC10858F8206C921BDE
:10F58000039290F8ED20022A1CBF90F8BB000128DE
:10F590007DD058F81C8C04EB051206EB0809CDF859
:10F5A0003890D2F80490D6689568106809EB060286
:10F5B000DFF8349228441044D9F800A03544504470
:10F5C000D9F804A0DFF824B25244D9F808A0D9F839
:10F5D0000C9055444E44DDF808A0DDF83890AAEBB5
:10F5E0000909CDF82090DDF80C90A9EB0809CDF8B9
:10F5F0002C90DBF800908144CDF82890DBF8049043
:10F6000009EB020ADBF80890DBF80CB0A9440BEB1D
:10F61000060EDDF828B00BFB0EFB0AFB19BB9BFBAB
:10F62000F3FBBBF1000F08BF4FF0010B4FEA8E2E2A
:10F630004FEA8A2A9AFBFBFA4FEA892999FBFBF9E0
:10F640009EFBFBFECAF1000ACDF834A0DDF828A02D
:10F65000C9F100094FEA8A2A9AFBFBFB00FB0EFA6C
:10F6600002FB09AA9AFBF3FACDF828A0DDF834A032
:10F6700000FB0AFA02FB0BAA9AFBF3FACDF824A0CE
:10F6800005FB0EFA06FB09A999FBF3F900E05BE024
:10F69000DDF834A0CDF8309005FB0AF906FB0B9994
:10F6A00099FBF3FBDDF828A0DDF820900AFB09FEAA
:10F6B000DDF824A0DDF82C900AFB09EEDDF820A08F
:10F6C000DDF830909EFBF3FE09FB0AFADDF82C9082
:10F6D0000BFB09A999FBF3F9DDF838A0C844F24403
:10F6E000CDE900A8DDF828A0CBF5806ECAF58068CA
:10F6F00008FB00FBDDF824A0DDF83090CAF1000A19
:10F70000C9F100090AFB05BB08FB02F809FB00F080
:10F710000AFB06880EFB05009BFBF3FB98FBF3F846
:10F7200090FBF3F0CDF810B0CDE9058009FB02F0B5
:10F730000EFB060090FBF3F007902D480022E846F0
:10F7400004AE00EB0C0315E0294A0020624403904C
:10F7500012F8012C02AB07EB021202EBC10253F8C4
:10F76000204002EB8005401C00B245F8204C0228E6
:10F77000F5DB20E013F8015C58F8220007EB0515D3
:10F7800005EBC10505EB820545F8200C002006EBD2
:10F79000C20513F801AC55F8209004EB0A1A0AEBE5
:10F7A000C20A4AF82090401C00B20228F1DB501C2B
:10F7B00002B2022ADEDB0E48604410F8010C07EBAF
:10F7C000001000EBC10050F8200C0FB0BDE8F08F26
:10F7D000676666666086001044860010380901106E
:10F7E000780A0110B80B011090860010A086001056
:10F7F000F80C01100288438862F30F01808863F3DC
:10F800001F419A4284BF63F30F0162F31F410A0C48
:10F81000824288BF60F31F4188B20A0C904284BFC5
:10F8200062F30F0160F31F41080C704730B51546B5
:10F83000024690F8EDC090F89900FE4B2C8869883C
:10F8400000EB400003EB8000BCF1020F1CBF92F8FC
:10F85000BB20012A20D0844630F80A0C2CF8080C72
:10F860003CF80C0C2CF80A0C2CF80C4C3CF8040C52
:10F870002CF8020C3CF8060C2CF8040C2CF8061C96
:10F88000ACF10C00FFF7B6FF0446ACF10600FFF741
:10F89000B1FFAC80E88030BD20F8084C20F80A4C5D
:10F8A00020F80C4C20F8021C20F8041C20F8061C40
:10F8B0000846EEE730B4002488B0A44601EB0011FE
:10F8C00001EB4C0030F8100C04440CF101001FFA5D
:10F8D00080FCBCF1080FF3D3E4081C600023184639
:10F8E0006D4601EB400C3CF810CCACEB040C0CFB6F
:10F8F0000CFC45F820C0401C80B263440828F0D3BB
:10F90000D80831F80A3C31F8101C591A49431160E3
:10F9100008B030BC7047C84A0021024402F8011CFC
:10F92000C64A024402F8011CC54A024402F8011CFE
:10F93000C44A02EB800242F8041CC34A02EB800274
:10F9400042F8041CC14A02EB800242F8041CC04A7F
:10F9500002EB800242F8041CBE4A02EB400020F891
:10F96000021C418070472DE9FF4FE1B053B20022E5
:10F970005792B94A1F461268B2F812C0528BCCEBAC
:10F980000C1CBCFBF2F25092AD4ADFF8B0C202444C
:10F9900012F8016C0CF10202844402441CF8015C70
:10F9A00012F8014C00EB800C01EB0C1C002E7DD0FA
:10F9B0000CEB450131F8505C5495B1F8501053915F
:10F9C00012F8011C143949B20029BCBF283149B2D0
:10F9D0000CEB410131F8502C5292B1F850101E221C
:10F9E00051910CEB4401052A31F8504C5994B1F86F
:10F9F0005010589140F2E6819249EE4601EB8001A9
:10FA000051F8044C90495E9401EB8000012150F8BC
:10FA1000040C5B90844268DD649800885A90501E04
:10FA200058BF744612D40CEB430544F8201004EB85
:10FA300080065B1E35F8505C5BB2C6F8A050002B08
:10FA4000B8BF2723401E00B20028ECDA00210C4684
:10FA5000B846501E58BF754616D40CEB480355F8EF
:10FA60002060B3F850307343A8F1010659184FFADB
:10FA700086F844EBE374B8F1000FB8BF4FF02708E5
:10FA8000401E00B20028E8DA00252E46501E58BF5E
:10FA9000F1467DD40CEB470309EB8008B3F85030F6
:10FAA000D8F8A0807F1E03FB08F300E00BE05D198F
:10FAB0007FB246EBE376002FB8BF2727401E00B287
:10FAC0000028E7DA67E0611CCAB23CF8501C549188
:10FAD000BCF85010539125F00101614431F8505C9D
:10FAE0005295B1F8501051917BE76E9800885A906A
:10FAF000501E58BF744612D40CEB430544F8201036
:10FB000004EB80065B1EB5F850505BB2C6F8A050FF
:10FB1000002BB8BF2723401E00B20028ECDA0021DA
:10FB20000C46B946501E58BF754616D40CEB490317
:10FB300055F8206033F8503C7343A9F10106591879
:10FB40004FFA86F944EBE374B9F1000FB8BF4FF0F8
:10FB50002709401E00B20028E8DA00252E46501E74
:10FB600058BFF14617D40CEB470309EB800833F874
:10FB7000503CD8F8A0807F1E03FB08F35D197FB2CC
:10FB800046EBE376002FB8BF2727401E00B200E007
:10FB900001E00028E7DA0027B8463846002AC8BF47
:10FBA000F4460ADD5CF8203000F101005B43DF1908
:10FBB00048EBE37800B28242F4DC0023CDE9553310
:10FBC0001846002AC8BFF44615DD0CEB80095CF826
:10FBD0002030D9F8A09003FB09F3DDE955A94FEADD
:10FBE000E37B13EB09034BEB0A09401CCDE955936A
:10FBF00000B28242E9DC4FF0000AD1465046002AAA
:10FC0000C8BFF34610DD0BEB80035BF820C0D3F8D0
:10FC1000A03000F1010003FB0CF313EB0A0A49EBDF
:10FC2000E37900B28242EEDC4FF0000CE34660461E
:10FC3000002A13E00C0D01104A86001048860010BF
:10FC40004C860010808600108886001068860010A0
:10FC50007086001078860010F08600100EDD6B466E
:10FC600003EB800300F10100D3F8A03000B25B4346
:10FC700013EB0C0C4BEBE37B8242F0DCA7FB0C326A
:10FC8000CDE95CCB08FB0C2207FB0B2CDDE95520F2
:10FC9000A0FB0ABECDE95F2002FB0AE200FB0922BD
:10FCA000B3EB0B006CEB0202CDE95520104304BF0F
:10FCB0004FF0000B594632D0DDE95C03A0FB012C6C
:10FCC0005C9103FB01C100FB0411DDE95F30A0FB87
:10FCD00005CB03FB05B300FB0633B2EB0C0061EB75
:10FCE0000301DDE955320CF0F7FA8346A7FB050165
:10FCF00008FB051107FB06125C99AAFB013C09FBF6
:10FD000001C10AFB0411C01A62EB01010904DDE91B
:10FD1000553241EA104100040CF0DEFA01465A98CF
:10FD200048431BEB204048BF00205B9B5E9A9A42F1
:10FD300024DD549A539B4A430BEB2242D31A44BF0F
:10FD4000539B9B1A509A93423CD2529A5143519AD8
:10FD50000BEB21418A1A44BF519A521A50998A4298
:10FD600030D25899091A44BF5899411A509A914271
:10FD700028D26E9908800120579023E0539A549B13
:10FD80004A430BEB2242D31A44BF549B9B1A509A0E
:10FD9000934217D2519A5143529A0BEB21418A1A3E
:10FDA00044BF529A521A50998A420BD25999091A51
:10FDB00044BF5999411A509A914203D264990880DC
:10FDC00001205790579865B0BDE8F08F2DE9FF4F9F
:10FDD0008DB09A468B46054603F096FE0190007B57
:10FDE000D8B1142002900220009095F89940022C7E
:10FDF00094BF4FF001094FF0000995F876000128F3
:10FE00001CBFFE48806914D0039095F8ED00FC4BB0
:10FE10004FF00008022846D115E03C2002900198DE
:10FE200090F8420002282EBF03200F200090DCD360
:10FE3000DAE7F44864220068418A408B5143B1FB01
:10FE4000F0F04043E0E71819B9F1000F00F8018C19
:10FE5000ED48204400F8018C80F80980EB482044EC
:10FE600000F8018C80F80980E94800EB440020F894
:10FE7000028CA0F81280E7488BF8CC80204485F8EB
:10FE8000CC8000F8018CE448204400F8018CE34861
:10FE9000204400F8018CE248204400F8018C1CBF8B
:10FEA0002046FFF738FD0F981919B9F1000F0288A5
:10FEB000DC48059100EB0410079011F8011C049137
:10FEC00000EB410020F8102CBAF80010A0F89010B8
:10FED00072D0D548D54900EB040E21441EF8010C20
:10FEE00001F8010CD2492144069111F8011C01B31B
:10FEF000411CC9B2282927D3CE4904EB840201EB67
:10FF0000021101EB400231F850CC32F8503CACEB1E
:10FF1000030CC94B03EB840343F804CCB2F8502024
:10FF2000B1F850108A1AC54901EB840141F8042C3C
:10FF300025E0C14901EB840141F8048CBF4901EB84
:10FF4000840141F8048C1AE0BA4A04EB840302EB02
:10FF5000031202EB410131F8502C31F8523CD31A14
:10FF6000B54A02EB840242F8043CB1F85020B1F8E3
:10FF70004E10521AB14901EB840141F8042C0F993B
:10FF800004EB840327280A88AA4901EB031101EB3B
:10FF9000400121F8502CBAF80020A1F8502003D1DC
:10FFA000069A012102F8011C401CC0B20EF8010C97
:10FFB000282828BF0EF8018C95F8ED00022800F0E3
:10FFC000898104980799C01D4FF0000E00F00700CA
:10FFD0000F9ACDF818E001EB4000128830F8101CA1
:10FFE000B0F89000511ABAF80020101AB9F1000FB9
:10FFF00036D08F4A224412F801CC914ABCF1000F4E
:020000021000EC
:1000000002F108034AD002EB840C00295CF8046C6E
:10001000ACBF0A464A42164403EB84034CF8046C16
:1000200053F8047C0028B4BF424202463A4443F8E5
:10003000042C1746804A02EB840252F8042C002A52
:10004000B8BF5242B21A4CF8042C7C4A02EB84022C
:1000500052F8042C002AB8BF5242BA1A43F8042CB2
:10006000684A1268138B5943138A91FBF3F6518B3C
:100070004843518AB9F1000F90FBF1F704D06C4866
:10008000204410F8010C08B3002E3DDD60484FF00D
:10009000020100EB440020F8028C4DE002EB8402E8
:1000A000002952F8046CB4BFC1F1000C8C46B44472
:1000B00042F804CC03EB8402002852F804CCB4BF0D
:1000C00043420346634442F8043CC9E75D48002EBE
:1000D00000EB440030F8022CB4BF714231468A4232
:1000E00005DA002EACBF3146714220F8021C42886E
:1000F000002FB4BF794239468A42C5DA002FACBF1F
:10010000394679424180BFE706DA4148012100EBD8
:10011000440020F8028C0FE03C48204410F8011CF9
:100120003B4800EB440030F8022C642A04D2521CF5
:1001300020F8022C4FF0010E002F07DD344A4FF05B
:10014000040002EB4402A2F8128015E007DA304AFC
:100150004FF0030002EB4402A2F812800CE02C4A9C
:100160002A4802EB44022044538A407A642B03D28B
:100170005B1C538201220692244A224412F8013C5D
:1001800013B38B4221D1224B03EB440333F802CC4F
:10019000029B9C451C4B234496BF13F801CC03F8EB
:1001A000018CBCF1640F51D2BEF1000F4ED10CF1A5
:1001B000010C0CF0FF0C03F801CCBCF10A0F45D385
:1001C000144B234403F8018C40E00F4B234413F8F5
:1001D00001CCBCF1050FDFF83CC0A44436BF1CF8CD
:1001E00001EC0CF8018CBEF1640F05D20A2EA4BFFD
:1001F0000EF1010E0CF801EC26E000004486001020
:10020000C40E0110F0860010E20E0110CE0E011097
:10021000F60E01101E0F0110280F0110320F0110F1
:100220002E090110840D0110488600104A86001026
:100230004C860010EE0701106886001070860010D2
:10024000808600107886001003F8018C537A23B35F
:10025000834223D1FD4B03EB4403B3F812C0029B4E
:100260009C45FB4B234496BF93F809C083F8098053
:10027000BCF1640F2BD2DDF818E0BEF1000F26D1DF
:100280000CF1010C0CF0FF0C83F809C0BCF10A0F53
:100290001DD3F04B234403F8018C18E0EC4B2344AE
:1002A00093F809C0BCF1050FDFF8A8C3A44436BF1A
:1002B0001CF801EC0CF8018CBEF1640F05D20A2F7A
:1002C000A4BF0EF1010E0CF801EC83F8098002F8CE
:1002D000011C507204980599401CC0B201F8010C31
:1002E00008280AD3059800F8018C9BF8CC00002858
:1002F00004BF01208BF8CC0006E09BF8CC0000285E
:1003000008BF85F8CC8037D00AAB08AAD24920466E
:10031000FFF7D0FA83460BAB09AAD0492046FFF776
:10032000C9FA03998B4598BF88420CD9032085F8F8
:10033000CC00CB480121204400F8018CC94820445E
:1003400000F8011C14E0C248204410F8011C0829E0
:100350009CBF407A08282AD9032085F8CC00C048E1
:10036000C0492044214400F8018C012001F8010C0F
:1003700095F8CC00032807D0BB48204400F8018C36
:10038000B448204400F8018CB8480221204402906F
:1003900000F8011CB648B9F1000F00EB040B0BF894
:1003A000011C26D095F8CC0003281CD01EE0AC48D8
:1003B000204410F8011CC8293CBF491C00F8011C4E
:1003C000A849214411F8011C012908D110F8011C89
:1003D000009881429CBF032085F8CC00D4D902202C
:1003E00085F8CC00C8E703F058FC88B12046FFF739
:1003F00092FA95F8CC0003281EBF042811B0BDE87E
:10040000F08F0120019981F8200511B0BDE8F08F2F
:100410009848204410F8010C012808D00028E8D1A1
:100420009548204410F8010C401C0728E1D3282EE1
:10043000D8BF282F09DC914800EB440030F8021C9B
:1004400028299CBF408828280AD90198007B0028C9
:10045000CFD00299032001F8010C0BF8010CC8E77A
:100460008548CDF800A02044854910F8012C20468D
:100470000F9BFFF778FA012805D0029800F8018C4D
:100480000BF8018CB5E70299012001F8010C0BF87B
:10049000010CAEE7B0F8B030B1F8B0C0B3EB0C026D
:1004A00048BFACEB0302B0F8B230B1F8B210581A42
:1004B00048BFC81A02FB02F100FB0010704770B57C
:1004C0000D46044603F020FB94F8ED006D4E022823
:1004D0001DBF94F8BB000128012DB4F8B4000FBF74
:1004E000B4F8B62094F8990006EBC00151E9020275
:1004F00032213125B4F8B4C0B4F8B63005FB00C0E1
:10050000B0FBF1F005FB0232B2FBF1F194F8992057
:1005100006EBC20242F8080C94F8992006EBC202DE
:1005200042F8041CA4F8B400A4F8B61070BD2DE97C
:10053000F007554CDDE9078C24681F8890F8ED30F2
:10054000658A648BC5EB0515AD00B5FBF4F90E8823
:100550001588B8F80040032B3BD190F89930DFF8AC
:100560002CA10AEB430333F8028CB8F1050F30D20B
:10057000B8F1000F1AD0A1F800C02B1B1480002B7B
:10058000B8BF5B424B459CBFBDE8F007704767456D
:100590001CBFBDE8F0077047052190F899000AEBF1
:1005A000400020F8021CBDE8F00770474FF001083A
:1005B00023F8028C2B1B1C04A6EB070894FBF8F411
:1005C0007443A5EB2445A1F800C005EB244111803C
:1005D000D5E7A1F800C0BDE8F00770472DE9F04766
:1005E00086B00C46074603F0ABFA804600F0B8FA36
:1005F000064600F0B8FADFF890A0054694F89A0095
:10060000DAF80010C0EB001008EB0010B1F812800F
:10061000B1F810903988ADF808107988ADF80C1051
:10062000B0F8B410ADF81010B0F8B600ADF8140082
:1006300000F02DFB60B3BDF80800B04238BF304673
:10064000ADF80800BDF80C10A94222E0F60E01102A
:10065000E20E0110280F0110840D0110240E01106C
:10066000320F01102E0901101E0F0110DA070110C0
:10067000E40701104C8600104A86001078860010AE
:10068000EE0701103C0F0110F08600108C0F0110D6
:100690001CE038BF2946ADF80C10A9EB0602531E2A
:1006A0008342B8BF1846ADF80800A8EB0500421E0B
:1006B0008A42B8BF1146ADF80C10BDF80800B880EA
:1006C000BDF80C00F88006B0BDE8F08794F8ED00A6
:1006D00002281CBF94F8BB0001281ED16078FE4A96
:1006E00060B1DAF800108B795B1E98421CBF20784D
:1006F000002803D0C979491E884207D194F899107F
:10070000052002EB410121F8020C06E094F8991053
:10071000002002EB410121F8020CBDF80800B042B4
:1007200008D205A8CDE9000604AB03AA02A9204619
:10073000FFF7FDFEBDF80C00A84208D204A8CDE9E1
:10074000000505AB02AA03A92046FFF7F0FEA9EBBE
:100750000600BDF80810401E884209DA80B205A9DB
:10076000CDE9001004AB03AA02A92046FFF7DFFE83
:10077000A8EB0500BDF80C10401E88429DDA80B23F
:1007800004A9CDE9001005AB02AA03A92046FFF792
:10079000CEFE92E730B490F8ED20052490F890104A
:1007A000DFF838C390F89930022A1BBF90F8BB20BD
:1007B000012A0A4613F80C20042505FB021191FBBF
:1007C000F4F103F80C1080F8901030BC70472DE95C
:1007D000F04F87B0044600F0C3F9824600F0C3F939
:1007E000814603F0ADF9059003F08EF90746007BD2
:1007F00094F89980DFF8E8B200281CBF387D012802
:10080000DBF800107ED0086FC0F3C0420192C0F345
:100810004042C0F3804004920090486FC0F303410F
:100820000E02B049414411F8011C02290EBF4FF4D9
:100830004075C0F3035005020220FEF715F9A848E1
:10084000006890F8700010F0010F00F0798194F8C2
:100850009A00B4F8B010ADF80810B4F8B210ADF8C2
:100860000A10C0EB0011059802AA00EB011B5946C3
:100870002046FEF7DBFF019838B1BDF80C00ADF85B
:100880000800BDF80E00ADF80A0094F8ED0002284B
:1008900019BF94F8BB0001284046FEF75DFCBDF887
:1008A000082000212046FEF74DFE0190BDF80A20E9
:1008B00001212046FEF746FE01990029B8BF00211C
:1008C0000028B8BF0020DFF818C2DCF80020B2F919
:1008D0001030A3F1010E8E45B8BF7146B2F9122057
:1008E000531E8342B8BF184689B283B27E48ADF822
:1008F0000C1000EB0802ADF80E300A3012F801CCF3
:10090000404400E027E010F801EC02F801EC00F8A8
:1009100001CC009800281CBFADF80810ADF80A30D3
:100920000DF10E0303AA59462046FFF74FFAB4F81B
:10093000B000BBF8B020811A48BF111AB4F8B22039
:10094000BBF8B230D01A48BF981A494300FB0013D5
:10095000387BC0B34EE091F87000C0F3C002019242
:10096000C0F34002C0F3800004920090387D01285B
:1009700011D003F006F910F4817F14D0DBF80000E9
:10098000B0F8740001070E0DC0F30320000200F55B
:100990008075012051E7B1F87400C0F3032006020E
:1009A0003546002049E703F094F9002818BF03F00A
:1009B0004EF9DBF8000090F8740001070E0DC0F34B
:1009C00003100502EDE7FFE74848404410F8010C2A
:1009D000012807D070B94648404410F8010C401C6B
:1009E000282807D9BDF80C00ADF80800BDF80E00A6
:1009F000ADF80A00CDE9006597F8422002A920462B
:100A0000FEF7C8F8049868B1BDF80C00ADF808000E
:100A1000BDF80E10ADF80A10A4F8B400BDF80E0031
:100A2000A4F8B60003F039F9012804BF94F8E500F2
:100A3000012807D1B4F8B000A4F8B400B4F8B200AB
:100A4000A4F8B600264D286890F8700010F0200F2A
:100A50000FD097F8421001296ED026484FF0FF3191
:100A600001804180080C24490880488000202039FA
:100A70000870B4F8B400ADF80800B4F8B600ADF8EA
:100A80000A00214602A8FFF7A9FDBDF80C00ADF849
:100A90000800BDF80E10ADF80A1094F8ED1005230B
:100AA0000E4A02291BBF94F8BB10012994F890103C
:100AB00094F8991018BF895C94F890C0042606FB3E
:100AC00001C191FBF3F194F899305045995484F8A1
:100AD0009010BDF80A1011E08C0F01109F0F01104B
:100AE000F0860010DA070110F80C01104C86001097
:100AF0004A8600106086001064860010B8BF504619
:100B00004945B8BF49462B68B3F91020A2EB0A0249
:100B1000A2F1010C8445B8BF6046B3F91220A2EBE4
:100B20000902531E8B42B8BF1946A4F8B400A4F8BA
:100B3000B61007B0BDE8F08F2046FEF7E6FB98E759
:100B4000B4F8B000A4F8B400B4F8B200A4F8B60049
:100B500007B0BDE8F08F0000FE487047FE487047C0
:100B6000FE4800787047FD4840787047FB481421E4
:100B700081801221C180704703460020024600296F
:100B8000D8BF704753F822C0521C60449142F9DC30
:100B900070472DE9F05F0E46054602F0E1FF04467E
:100BA00002F0DAFF310291FBF0FC290291FBF4F331
:100BB000DFF8A8A30021DFF8A893BAF80480BAF8F8
:100BC00006704FEA6C264FEA632B002CC8BFE24D3B
:100BD0000BDD01FB03F20BEB222245F8212049F843
:100BE0002120491C09B28C42F3DC0021DFF874B3E8
:100BF0000028C8BFD74D0BDD01FB0CF206EB22220B
:100C000045F821204BF82120491C09B28842F3DC29
:100C10000CFB08FC4FEA6C317B43CAF808105A13EE
:100C20009AF802504FEA6C3C5B13CDB1D9F8003012
:100C30000BEB80009B1AC9F8003009EB840353F8D2
:100C400004CC624443F8042CDBF80020521ACBF8A1
:100C5000002050F8042C114440F8041CBDE8F09F1B
:100C6000D9F800500BEB8000AA1AC9F8002009EB54
:100C7000840252F8044C234442F8043CDBF8002080
:100C8000511ACBF8001050F8041C6144E4E7B34853
:100C90008078012818BF002070472DE9F047DFF861
:100CA000C89204461226D9F80000AC4D478AB0F825
:100CB00010801420142C03D2A4F10F01052902D2B4
:100CC000A880EE801BE0A4F10A0105293CBFA880A2
:100CD000E88014D3611F052903D21620A880E8807C
:100CE0000DE0052C28BFA88008D202F0D6FF00280E
:100CF0001DBF1820A880E880AE8000D1EE800021C2
:100D0000002C06BF0120A870A970D9F80000428A03
:100D1000408B6243B2FBF0F0287069704146384660
:100D2000BDE8F04735E710B5012907BF8F4C142106
:100D30008F4C1221142803D2A0F10F02052A01D2F0
:100D4000218010BDA0F10A02052A38BF14200CD35F
:100D5000421F052A38BF162007D30528F0D202F01B
:100D60009CFF002814BF18201220208010BD7E494F
:100D70007A4A0128096807D0488B5278498A50433B
:100D8000B0FBF1F0C0B27047088B1278098A50436B
:100D9000B0FBF1F0C0B27047734810B502684FF075
:100DA000140C92F86C30508A118ADB08528B434342
:100DB000B3FBF2F3694A137000235370A2F804C026
:100DC0004FF0120CA2F806C09370FFF7E2FE6949DB
:100DD00000204FF6FF7221F8202001EB8003401C19
:100DE00080B25A800A28F6D310BD2DE9FF4FADF529
:100DF000037D1C461646982168460BF05EFA50218A
:100E00004CA80BF05AFA982126A80BF056FA50215C
:100E100060A80BF052FA02F093FE814602F074FED5
:100E2000074602F083FE7890503081900A2080902F
:100E300002F092FE054602F093FE80464A480068A2
:100E4000418A7591008A7690607800281BBFA8F1CE
:100E500001018842424840487790207800281BBF13
:100E6000691E88423F483B48749002F08AFEDFF8D2
:100E7000ECA010F0020F0CD01820AAF80400DDE955
:100E80007501FFF786FE3748DAF80820C16B114478
:100E9000C1639AF802007F90012803D1304877900F
:100EA0009838749094F8EBC0DFF8CCA0BCF1000F38
:100EB0000FD1E088401DAAFB0010C00800FB05F11F
:100EC000A088401DAAFB002006EBD000085C00F0C3
:100ED0003F0C94F89A0094F899202649C0EB001032
:100EE00001EB820309EB001033F8049CA9F57F4164
:100EF000FF391DBF33F8022CA2F57F41B1F1FF018C
:100F000081880CBFC2884946B4F804B0CDF8E8B176
:100F10000BF1050BAAFB0BEBCBF3CF0BCDF8F8B124
:100F2000B4F806B0CDF8E4B10BF1050BAAFB0BEB5E
:100F3000CBF3CF0BCDF808B201F1050BAAFB0BEBFD
:100F4000CBF3CF0E02F1050BAAFB0BBACAF3CF0A03
:100F500014E00000AC0F011044100110B086001026
:100F60002C11011094100110F0860010B4860010AE
:100F7000B68600107C110110CDCCCCCCCDF8ECE1C4
:100F8000DDF8E8B14CF6CD4E0BFB0EFB4FEADB4B28
:100F9000CDF8F0B1DDF8E4B10BFB0EFB4FEADB4B13
:100FA000CDF8F4B101FB0EFB4FEADB4BCDF8E8B115
:100FB00002FB0EFB4FEADB4BCDF8E4B1DDF8ECE1D0
:100FC000DDF8F8B1F34504BFDDF808B2D3450BD026
:100FD000DDF8E8B1DDF8F0A1DA4515D1DDF8F4B1BE
:100FE000DDF8E4A1D3450FD197F842A0BAF1020F82
:100FF0000AD3DDF8E0B19BF842B0D34504BF94F8C2
:1010000098A0BAF1020F4CD04FF6FF7023F8040CF1
:10101000F94994F8992001EB820121F8020C207B18
:101020007990607B7890A27B94F80F907898EB464B
:1010300048452AD800FB05F189B27A917999914205
:101040001FD87A9B03EB010A839B33F91A3016F8F9
:101050000AA00AF03F0AE2450FD1DDF800A253458D
:101060000BDB5BF821A09A444BF821A00DF5987A90
:101070005AF820E073444AF82030491C89B2914262
:10108000DFD9401C80B24845D4D9387B00287DD0B8
:1010900097F82E05002804BF97F83304012852D092
:1010A0008CE0DFF854A34FF6FF7BD94504BF33F83B
:1010B000029CD94507D123F8041C94F899100AEB37
:1010C000810121F8022C017B227B914238BF2173E0
:1010D000417B627B914238BF6173817BA27B9142ED
:1010E00088BFA173C17BE27B914288BFE173217B02
:1010F000799194F80DA0CDF8E0A194F80F90A27B1F
:1011000090F8EBB0CA4591D80AFB05F080B27A900E
:101110007998904210D87A99819B01445B5C03F0E6
:101120003F0EDE4504D123F03F0343EA0C03735422
:10113000401C80B29042EED90AF101001FFA80FAF9
:10114000CA45E1D972E794F8E860012E07D835D195
:1011500097F84C13849830F911001E282EDD502189
:101160004CA80BF0AAF807EB460197F8422091F83B
:10117000E20391F8E313012A13D10A1A521C0A2A36
:101180000FDD07EB860292F8483300E016E0DA1E26
:10119000DB1C8242C8BF1046C0B29942C8BF194684
:1011A000C9B2884298BF4CAB08D8849A32F9102053
:1011B00043F82020401C80B28842F6D900216A46BC
:1011C0000846002D40F3F68052F82030401C1944A8
:1011D000A842F9DB002940F3ED8000214CAB084622
:1011E000B8F1000F40F3E68053F82020401C114472
:1011F0008045F9DC00297ADD002026AE002D88BF6D
:1012000059460BD9749A51F8203052F820205A438D
:1012100046F82020401C80B28542F3D80020B8F167
:10122000000F84BF4CA960AA0CD9779B51F820C04D
:1012300053F820300CFB03F342F82030401C80B2FE
:101240008045F2D8002132460846002D05DD52F8CF
:101250002030401C19448542F9DC00226B461046C0
:10126000002D05DD53F820C0401C62448542F9DCA6
:1012700091FBF2F094F87610012904BF7F990029C0
:101280006AD1DFF878C1F0280CEB8503DCF8007038
:1012900053F8044CBCBF8020CCF800002EDBA0F13A
:1012A000F001DC2938BFC02007D3A0F5E671B1F505
:1012B000967F38BF4FF4807002D2CCF800001DE05A
:1012C000A0F5B8413039B1F52F7F3CBF45F6E0605D
:1012D00043F8040C12D3A0F5BC41EC39642938BFA3
:1012E00045F6407008D345F65071884200E061E051
:1012F000A8BF4FF4BF4001DB43F8040C0020002DD1
:1013000088BF59460CD9749A51F8209052F8202081
:1013100009FB02F246F82020401C80B28542F2D838
:10132000002132460846002D05DD52F82060401CA1
:1013300031448542F9DC00226E461046002D05DD61
:1013400056F82090401C4A448542F9DC91FBF2F0AB
:10135000CCF8007043F8044C002260AB1146B8F1A1
:10136000000F05DD53F821C0491C62448845F9DCB3
:1013700000230DF5987C1946B8F1000F05DD5CF8E7
:101380002140491C23448845F9DC92FBF3F10028F5
:10139000B8BF00200029B8BF0021769A521E9042A3
:1013A000C4BF7698401E759A521E9142C4BF75996B
:1013B000491E01E000200146909A1080919801801A
:1013C0000DF5077DBDE8F08F2DE9F84F1D46164657
:1013D0000C46834602F0B4FB014694F89A000022C2
:1013E000C0EB001001EB00130548BBF1010F09D061
:1013F000BBF1080F27D049E07C11011094100110B7
:10140000F086001000686E2140F2D34AB0F812C096
:10141000078B0CFB01F8418B008AB2FBF7F900FB4C
:101420000AF0B0FBF7F0B8FBF1F840F231570CFBD3
:1014300007FCBCFBF1F11FFA80FA80B21FFA88F8B2
:101440008FB2009022E001684FF448700F8AB1F823
:1014500018C07843B0FBFCF01FFA80F9488A07EB0C
:101460008717C0EB40187F0108EB8018498BB7FB4A
:10147000FCFC1FFA8CFA40F2415C00FB0CF0B8FB5C
:10148000F1F8B0FBF1F01FFA88F887B2A4F8B06069
:10149000A4F8B2504E4538BFA4F8B09003D3B2457B
:1014A00038BFA4F8B0A0454538BFA4F8B28003D334
:1014B000AF4238BFA4F8B2700120BBF1080F15D0BD
:1014C000BBF1010F18BFBDE8F88F4E4522BF009950
:1014D000B142454503D3BD4298BFBDE8F88F94F8AB
:1014E000ED10022918BFBDE8F88F1CE04E4528BF5B
:1014F000B24504D3454524BFAF42BDE8F88F94F808
:10150000ED1002290FD084F8E50093F8E5100129C9
:1015100018BFBDE8F88F84F8E40084F8E02084F870
:10152000ED20BDE8F88F84F8E40084F8E02084F82A
:10153000ED2084F8E520BDE8F88F2DE9F04385B073
:101540001C4616460F46804602F0DEFA02F0EEFA1E
:1015500002F0F6FA94F89A10C1EB011100EB0115B4
:1015600002F0FEFA814602A903A8CDE90001234654
:10157000324639464046FFF738FCBDF80C00A4F867
:10158000B000BDF80800A4F8B20002F0FAFA10F4B6
:10159000817F08D002F050FBBDF80830BDF80C2068
:1015A0002146FFF711FF95F8BB00032807BF2878F5
:1015B000002805B0BDE8F083687800281CBFA9F1B9
:1015C00001018842A4BF05B0BDE8F08394F8BB00D8
:1015D00001281CBF05B0BDE8F083B5F8B000A4F841
:1015E000B000B5F8B200A4F8B20005B0BDE8F083D1
:1015F000A3E700002DE9F04114460D46074602F02E
:1016000083FA02F0A9FA064602F0AAFAD5E907130E
:1016100080462869002510B301EB81018900400054
:10162000B1FBF0F203EB83018900B1FBF0F1FE485E
:10163000A0FB02C34FEAD30CA0FB0130C308701E0D
:1016400084459CBFA8F10100834208D803FB06C073
:101650002280618037F81000A080BDE8F0812580ED
:101660006580A580BDE8F0812DE9F0410446DDE903
:101670000606089F0D4600281CBF002081F829009F
:1016800002D00020BDE8F081286820606868E06032
:10169000106851686060A1608422194604F114004A
:1016A0000AF006FEA86820612869A061A889A082C6
:1016B000A88CA4F8700095F8280084F8E10095F84B
:1016C0002A0084F8E200012084F8E00095F82B005D
:1016D00084F8E70084F8E37095F82C0084F8E800BB
:1016E00095F82D0084F8E90095F82E0084F8EA00BA
:1016F00095F82F0084F8EB003078401CC0B23070B1
:101700000A2828BF0120BCD3BDE8F0810028DCBF37
:10171000002070474FF480714FEA002C00200B121C
:101720009CFBF3F30A46991801EBD1714910531A47
:1017300048BF8B1A802B02DB401C6428EFD30812B1
:1017400070472DE9FF4F85B01F4616460D46002411
:1017500002F002FA0190B6F900E0B6F90200029038
:10176000287903906A79E87995F806A0A446654639
:1017700066460090824229DC0398504521DC02999C
:1017800002EB8203C1EB430303FB03FB019902FB62
:101790000108059931F918100A290EDD00EB8008BF
:1017A000CEEB480808FB08F903FB08F809FB01CC5D
:1017B0000BFB015508FB01660C44401C00B2504570
:1017C000E4DD501C02B200988242D5DDDFF85C8275
:1017D00088FB0C104111A1EBE07188FB0520421140
:1017E000A2EBE07288FB06304311A3EBE0734CB12F
:1017F000080211021A0290FBF4F091FBF4F192FB43
:10180000F4F202E000200146024600FB01F302FB75
:1018100012320844C0F1000C1412A0000CFB0CF1B1
:10182000C0EB2120001241000029D8BF002014DDA8
:101830000D024FF480700021031295FBF3F3024672
:10184000981800EBD0704010131A48BF831A802BF1
:1018500002DB491C6429EFD30012000200EBD070B8
:10186000DCEB60010CEB6000C0F100027C6148BF62
:101870004942F960002AB8BF524201EB81004000A2
:1018800088FB0030C310A3EBE0703A61FF28C8BFAB
:10189000FF2049115211FF2988BFFF21FF2A88BF6D
:1018A000FF22002912BF002A01210A46002808BF92
:1018B000012087F87C0087F87D1087F87E2009B02A
:1018C000BDE8F08F70B5044602F046F9054602F017
:1018D00047F92178024600291CBF681E814206D0C4
:1018E000607800281FBF511E8842002070BD012073
:1018F00070BD2DE9F05F9A4690460E46054602F00F
:1019000003F9044602F012F983464FF0000902F091
:1019100023F9074694F84A030023012842D1207B8B
:1019200000283FD0D4F82805DBF82815404A884223
:1019300006D2D2F800C0C94361440844106003E0F5
:10194000401A11680844106094F82605012808D050
:1019500094F8300400281CBF94F8180500281DD105
:101960000AE094F8300400281ABF94F818050028FB
:101970004FF0010912D1EBE7BAF1030F24BF207D2C
:1019800000280BD194F8240594F82215401A072852
:1019900004DB012084F82605136056E01068B0F5DA
:1019A000616F02D984F8263502E0B9F1000F4CD1FD
:1019B00002F08FF918B102F04AF9082803D102F0B9
:1019C00052F902282BD1737996F807B04FF000092D
:1019D0009B453AD3B07996F804A0441E5046844201
:1019E00016DB03FB070235F9121005EB4202B2F9D0
:1019F0000220B1EB020C48BFA2EB010CBCF1230F9B
:101A000002DD4FF0010903E0401C80B28442E8DAB5
:101A1000581C83B29B45E1D2B9F1000F15D0B6F93D
:101A200002005A2814DA05E0CDCCCCCC1F85EB514E
:101A3000BC860010B0898C289CBF98F87D00FA28DD
:101A40003CBF98F87E00FA2802D30120BDE8F09F41
:101A50000020BDE8F09F2DE9FF4F89B017460C46E6
:101A6000FE48D0E90012CDE90212D0E90210CDE91A
:101A7000041000200090019002F046F850300690CB
:101A800002F06AF8804602F06BF8B4F90210079190
:101A9000237861784FF000094A465C1EA1F1010CE1
:101AA0004D46A8F1010EA0F1010BEA4602A925F06E
:101AB0000100095A21440CB204A9002C085A6044C0
:101AC0000FFA80FCA8BFA64534DBBCF1000FA8BF0D
:101AD000E3452FDB0CFB0840069900B2095C49B3D3
:101AE000099931F91060002ED8BF012616980321FC
:101AF00020F8126006EB09000FFA80F903E0481E97
:101B000010F0FF0105D00AEB410030F9020C8642CB
:101B1000F5DC0223022909D20AEB430030F8020C5B
:101B20002AF81300581EC3B29942F5D3501C2AF864
:101B30001160C2B2681CC5B2082DB7D3BDF8000051
:101B4000BDF80210BDF8043001441944A7F87A101A
:101B50000C990A7007990844A7F84A00A7F87890EA
:101B60000DB0BDE8F08F2DE9F04186B014460D466A
:101B70008046002701F0C8FF02A8009001AB224672
:101B800029464046FFF767FF002084F85A7084F822
:101B90005F00687840B101F0E3FF6978401E884239
:101BA0001CBF06B0BDE8F081012084F8760006B0C5
:101BB000BDE8F0812DE9F04117460E4601F0A4FF83
:101BC000044601F0B3FF217D002599B9B1891E2992
:101BD00081BF97F87D104B29F18C072906D897F81B
:101BE0007D10642984BFF18C062903D9217B01254E
:101BF000022907D002F072F8002808BF0025284605
:101C0000BDE8F08194F82D15012919BF90F8420024
